:020000021000EC
:10F000000000012071BA020099BA02009BBA020006
:10F010009DBA02009FBA0200A1BA020000000000DF
:10F02000000000000000000000000000A3BA020081
:10F03000A5BA020000000000A7BA0200A9BA0200A7
:10F04000A9A80200ABBA0200B1B00200ABBA02003C
:10F05000ABBA0200ABBA0200ABBA0200ABBA020014
:10F06000ABBA0200ABBA0200959A0200ABBA02003A
:10F07000ABBA0200ABBA0200ABBA0200ABBA0200F4
:10F08000ABBA0200CDF70100ABBA0200ABBA020086
:10F0900091F80100ABBA020021BF0200ABBA020036
:10F0A000ABBA0200ABBA0200ABBA0200ABBA0200C4
:10F0B000ABBA0200ABBA0200000000000000000082
:10F0C000ABBA0200ABBA0200ABBA0200ABBA0200A4
:10F0D000ABBA0200ABBA0200ABBA020000000000FB
:10F0E0000000000000000000000000000000000020
:10F0F0000000000000000000000000000000000010
:10F1000000000000000000000000000000000000FF
:10F1100000000000000000000000000000000000EF
:10F4000010B5054C237833B9044B13B10448AFF35E
:10F4100000800123237010BD4C5D0020000000001F
:10F4200064C4020008B5034B1BB103490348AFF3A2
:10F43000008008BD00000000505D002064C4020090
:10F44000154B002B08BF134B9D46A3F5803A0021B6
:10F450008B460F461348144A121A00F063F80F4BFC
:10F46000002B00D098470E4B002B00D0984700206F
:10F47000002104000D000D48002802D00C48AFF315
:10F48000008000F02BF8200029000BF085FF00F031
:10F4900011F800BF0000080000000120000000007B
:10F4A000000000004C5D0020F482002000000000FD
:10F4B0000000000008B5074B044613B10021AFF36C
:10F4C0000080054B1868836A03B19847204600F016
:10F4D00031F800BF0000000024C0020070B50D4EDE
:10F4E0000D4CA41BA4100025A54209D10B4E0C4CB9
:10F4F0000CF08CFDA41BA4100025A54205D170BD05
:10F5000056F8253098470135EEE756F825309847EC
:10F510000135F2E7445D0020445D0020445D002099
:10F52000485D002002440346934200D1704703F82F
:10F53000011BF9E7FEE700BF00B585B0002303908B
:10F54000194601AA44F20100ADF80430029309F013
:10F5500065FA05B05DF804FB12F0030315D1F0B4B1
:10F560004C1CE4000A4D0B4E0B4F3370A4B21444F4
:10F570002C600A4E0A4D3A600A4C0B4A28803370C0
:10F58000218013801846F0BC70470720704700BFE9
:10F590006C5D00206A5D0020705D0020785D0020B9
:10F5A000745D0020765D0020685D0020094A0A4BEA
:10F5B00010781B78094A9842128806D9511C0B44CE
:10F5C000181A80B2101A80B270471B1A98B2101A1B
:10F5D00080B27047785D00206A5D0020765D002073
:10F5E0002DE9F047364F3B888B4282B04BD305461E
:10F5F00002A84FF0000800F8018D16460C4600F0F6
:10F60000FBFCDFF8D0C02F4B2F499CF800E01A78A4
:10F6100009889DF80700D2B28A4238BF01325FFAEA
:10F620008EFE38BF5FFA82F8C64530D093F800806E
:10F630001A78D2B2914286BF0132D2B200221A7039
:10F640009CF800201B789A4284BF01315B189B1AFA
:10F650001E4A11889BB299425FFA88F81DD3DFF8E1
:10F66000789000F0EFFCD9F800300FFA88F24FEAFA
:10F67000C20A43F83260534405B184B9002098802F
:10F6800002B0BDE8F087092002B0BDE8F08700F0C5
:10F69000D9FC042002B0BDE8F0871380DFE70C4BF3
:10F6A00038881B68294608FB003022460CF0A3FC72
:10F6B000D9F800309A440020AAF80440E0E700BFDF
:10F6C000745D00206A5D0020765D0020685D00208A
:10F6D0006C5D0020785D0020705D002000B583B077
:10F6E00002A8002300F8013D00F086FC064A9DF8C0
:10F6F00007001368591C1CBF0133136000F0A2FC03
:10F7000003B05DF804FB00BF7C5D002000B583B052
:10F7100002A8002300F8013D00F06EFC054A1368C2
:10F720000BB1013B13609DF8070000F08BFC03B0A8
:10F730005DF804FB7C5D00202DE9F84F1C4D2B6823
:10F74000002B32D11B4C1C4E227833789A422CD09D
:10F75000DFF868A0DFF86890DFF86880DFF868B04D
:10F7600003E0227833789A421FD02378DAF8002019
:10F77000B8F80000D9F80070DBB20FFA83FE02EB94
:10F78000CE0103FB0070898852F83E3098472378F9
:10F79000BBF80020DBB29A4203F101032A688CBF58
:10F7A000DBB200232370002ADBD0BDE8F88F00BF56
:10F7B0007C5D0020785D00206A5D0020705D002087
:10F7C0006C5D0020745D0020765D00202DE9F8431B
:10F7D000274A284B0024C2F84041C2F84441C2F8ED
:10F7E0004841C2F84C41C2F80041C2F804411B68CC
:10F7F0001BB32149D2F804550A68204FAD1A1A6884
:10F8000025F07F45AA42A04609D8197CDE69AD1AC9
:10F810001444A1B91EB133461A68AA42F5D9184951
:10F82000184A0B7812789A4217D01749174A41F8AC
:10F8300023404FF48013C2F80031BDE8F88383F809
:10F840001080D3E905933A684846194662B190475B
:10F850000028DFD0FFF770FEDCE7531CDBB2022B81
:10F8600008BF00230B70E0E71846C847D2E700BF87
:10F8700000100140A05D00209C5D0020805D002004
:10F88000995D0020985D0020905D002000E100E07F
:10F890002DE9F04FA74AA84913780978A74899425B
:10F8A00089B0D0F8008000F068810133DBB2022B10
:10F8B00008BF00231370A24A52F823109F4A08EB96
:10F8C000010B2BF07F4303931360012304939D4AA4
:10F8D0009D4BD2F800909D4A93F800E012785C7836
:10F8E000D3F804B09B7807924FF0000C0193059277
:10F8F00076464B46E2466246A6421AD006EB4600E2
:10F90000019F1BF830500136F6B2BE4208BF0026F8
:10F91000022D0BEBC00000F09780032DECD1002BE3
:10F92000EAD01A74DB69002BFBD1A6424FF0010C20
:10F93000E4D1BAF1000F40F08982BCF1000F40F031
:10F940008282804B049A1B680593002A40F019813B
:10F95000B9EB030318BF0123049300240023CDE96E
:10F9600002339C46754BDFF8F0A1D3F80080059F69
:10F970004FF001092CB3D4E901212346E469A2EB3D
:10F98000080020F07F4050454AD801441960C3E97F
:10F9900001CC83F81090C3F81CC0002F50D03A68F7
:10F9A0008A427BD23D4603E002688A427DD2054608
:10F9B000E869891A0028F7D11960D861EB61002C39
:10F9C000D9D103990EEB4E030EF1010276450BEBF4
:10F9D000C3005FFA82FE73D01BF83350019B73455E
:10F9E00008BF4FF0000E012D65D14368197C002936
:10F9F000E8D182685A600391C168996006950569EB
:10FA0000DD60406998610798002856D0039A5A60D3
:10FA100000220390A2EB080020F07F405045B4D9AB
:10FA2000A8EB020222F07F428A422BD2891A196087
:10FA3000C3E901CC83F81090C3F81CC0002FAED1ED
:10FA40001F460123029395E74768002B3FF454AF0C
:10FA50009F4200F083801D4600E00546E8690028CB
:10FA60003FF44AAF8742F8D1AF42029578D0F869A7
:10FA7000029D3F68E86100283FF43EAF05683D44C1
:10FA8000056039E7C3E900CCC3F808C083F81090DB
:10FA9000C3F81CC0002FD3D03A680021511A0122AC
:10FAA00039600292DF611F4664E7521A02601960F2
:10FAB000D861EB6183E7012184E7069803905EE754
:10FAC000002940F0CE81029B002B40F0C7811D4BE6
:10FAD000059A1B68934201D1049A2AB3002B00F0C7
:10FAE00021811B4A1B48D2F804151C680578A1EB3C
:10FAF000080323F07F430333002D00F0B0809C42C5
:10FB00002CBF08EB04034344114823F07F43C0F8A3
:10FB10004035D0F80425521A5B1A22F07F4223F0B8
:10FB20007F4303329A4250D8084A0023137009B029
:10FB3000BDE8F08F985D0020995D00209C5D00205D
:10FB4000905D0020A05D0020845D00208C5D002081
:10FB5000001001408D5D0020FEFF7F0002931F46D4
:10FB6000DB694FF0010C002B81D16948E246C0F8F7
:10FB700008C0CDF814C0039379E70021CDE90381D3
:10FB8000A5E600209146044602468446B3B11D68AE
:10FB90008D4200F2B680D868C3F800C0491B2A44E1
:10FBA000DD6938B108EB020727F07F47C3E9017030
:10FBB000DC611C462B464846002BE8D100283FF468
:10FBC000CDAE544A05931360C8E6D0F80435524AC6
:10FBD000C0F84035126851492F2300BF00BF00BF55
:10FBE00000BF00BF00BF00BF00BF8A422FD000BFD0
:10FBF00000BF00BF00BF00BF00BF00BF00BF00BF0D
:10FC000000BF00BF00BF00BF00BF00BF00BF00BFFC
:10FC100000BF00BF00BF00BF00BF00BF00BF00BFEC
:10FC200000BF00BF00BF00BF00BF00BF00BF00BFDC
:10FC300000BF00BF00BF00BF00BF00BF00BF00BFCC
:10FC400000BF00BF00BF00BF00BF00BF00BF013B3F
:10FC5000C3D1334B4FF40032C3F8002164E7304D79
:10FC6000DFF8B4C02D4F4FF48036C2F84463C2F8B9
:10FC700004634FF40036C5F880612E6001251560DD
:10FC8000DCF800602F2200BF00BF00BF00BF00BF34
:10FC900000BF00BF00BFBE422FD000BF00BF00BFEB
:10FCA00000BF00BF00BF00BF00BF00BF00BF00BF5C
:10FCB00000BF00BF00BF00BF00BF00BF00BF00BF4C
:10FCC00000BF00BF00BF00BF00BF00BF00BF00BF3C
:10FCD00000BF00BF00BF00BF00BF00BF00BF00BF2C
:10FCE00000BF00BF00BF00BF00BF00BF00BF00BF1C
:10FCF00000BF00BF00BF00BF00BF013AC3D1057005
:10FD0000FDE6002840F0B080691A196026E600BFC1
:10FD100000100140A05D0020405D00200024F400A0
:10FD200000E100E05249534A534E544C4FF48030A6
:10FD30004FF400370125C2F88070C1F848032F2224
:10FD4000C1F808034D603068164600BF00BF00BF11
:10FD500000BF00BF00BF00BF00BFA0422FD000BF48
:10FD600000BF00BF00BF00BF00BF00BF00BF00BF9B
:10FD700000BF00BF00BF00BF00BF00BF00BF00BF8B
:10FD800000BF00BF00BF00BF00BF00BF00BF00BF7B
:10FD900000BF00BF00BF00BF00BF00BF00BF00BF6B
:10FDA00000BF00BF00BF00BF00BF00BF00BF00BF5B
:10FDB00000BF00BF00BF00BF00BF00BF00BF013ECB
:10FDC000C3D18D602E490B6000BF00BF00BF00BFD4
:10FDD00000BF00BF00BF00BFA0422FD000BF00BFC8
:10FDE00000BF00BF00BF00BF00BF00BF00BF00BF1B
:10FDF00000BF00BF00BF00BF00BF00BF00BF00BF0B
:10FE000000BF00BF00BF00BF00BF00BF00BF00BFFA
:10FE100000BF00BF00BF00BF00BF00BF00BF00BFEA
:10FE200000BF00BF00BF00BF00BF00BF00BF00BFDA
:10FE300000BF00BF00BF00BF00BF00BF013AC3D179
:10FE4000104A137070E6104A13607AE50F48059A5D
:10FE500002700B48039C046007926EE50A4B1F601A
:10FE600035E60B4B1E702EE6074A059313604BE7F1
:10FE70000010014000E100E0405D00200024F4009B
:10FE80009C5D00208D5D0020A05D00208C5D002029
:10FE9000845D002010B50478012C82B00BD0022CB8
:10FEA0001DD034B902A8032300F8083D134B1B688A
:10FEB000984702B010BD43681149124804228DF8DA
:10FEC00000201B788DF8043022460AF0A9FF0E4A64
:10FED0000A4B14701B686846984702B010BDC3688F
:10FEE00007490848019301228DF800400AF098FF65
:10FEF000024B68461B68984702B010BDA45D002005
:10FF0000A85D0020205D0020A95D00202DE9F041C2
:10FF1000254D264E804617469E460FCD8AB002AC30
:10FF20000FC495E80F0098F810C098F8115037608A
:10FF300084E80F00D8E900431CF1000CD8E90267FF
:10FF400018BF4FF0010C002D14BF0E2000200193AC
:10FF5000174DD8F814308DF824E08DF81D00089363
:10FF60004FF0000E8DF81CC0CDE9047602A9039471
:10FF7000104A019B1048029385F800E00AF03AFD10
:10FF800058B9D8F80030013307D09DF825303BB17F
:10FF900001220A4908480AF043FF0AB0BDE8F0818F
:10FFA00005480BF05FF8F3E728C00200A45D0020CD
:10FFB000A95D002095FE0100205D0020A85D0020C5
:10FFC000074908B50122087006480AF07FFE11288B
:10FFD00004D0002814BF0320002008BD042008BD61
:10FFE000AC5D0020205D002008B502480AF0EAFD63
:10FFF000002008BD205D002070B4EFF3108472B6BD
:020000022000DC
:100000000D4B9A68AAB90D490D4E01259D60D1F896
:10001000805035401D60C1F88060D1F884505D602B
:100020004FF0FF33C1F88430027004B962B670BC7F
:10003000704701230370F8E7307E002000E100E004
:10004000FC06FFBC094B9A687AB170B910B4EFF3A3
:10005000108172B6064A1C6814605C68546098602F
:1000600001B962B65DF8044B70477047307E0020DE
:1000700000E100E00346BAB11088A1B1194401398A
:100080005A1E12F8013F40BA80B24340C3F3031036
:10009000584080EA003000B2430103F4FF53584057
:1000A0008A4280B2EDD170474FF6FF70E5E700BF9E
:1000B00070B582B002AB002503F8015D0446184616
:1000C0000E46FFF799FF2268A368506883421368C1
:1000D00088BF451CAB420BD05560E2686568531E73
:1000E000072B3DD8DFE803F028343C383C3C3C107B
:1000F000217C00293AD155602368A5681A68AA4274
:1001000000D2511C1960E8E7D6E9002305EBC000D6
:10011000C0E900232268D2E90030984213D3C31A01
:1001200091689DF80700994238BF9360FFF78AFFF6
:100130000024204602B070BD33782B542268D2E9E7
:1001400000309842EBD2A16801310144CB1AE7E7B5
:10015000338825F81030DDE7336845F82030D9E7DB
:10016000314600FB02500BF046FFD3E79DF8070035
:10017000FFF768FF0424204602B070BD70B582B05E
:1001800002AB002403F8014D044618460E461546FE
:10019000FFF732FF2368D3E9001291424BD025B913
:1001A000A268914238BF4D1C1D60E2686068531E12
:1001B000072B33D8DFE803F0121C32273232320427
:1001C00000EBC101D1E900239DF80700C6E9002337
:1001D000FFF738FF0024204602B070BD435C337047
:1001E0009DF80700FFF72EFF0024204602B070BDE7
:1001F00030F8113033809DF80700FFF723FF00240B
:10020000204602B070BD50F8213033609DF80700E1
:10021000FFF718FF0024204602B070BD01FB020169
:1002200030460BF0E8FE9DF80700FFF70BFF0024B7
:10023000204602B070BD9DF80700FFF703FF0524BC
:10024000204602B070BD00BF30B583B002AB0024C1
:1002500003F8014D05461846FFF7CEFE21460C2255
:100260002868FFF75FF99DF80700FFF7EBFE03B082
:1002700030BD00BF10B582B002AB002203F8012DE3
:1002800004461846FFF7B8FE2268D2E9000383420D
:100290000AD2A46801341C44241A9DF80700FFF711
:1002A000D1FE204602B010BD1C1A9DF80700FFF7D2
:1002B000C9FE204602B010BDD0B130B50C4685B0A5
:1002C00011B10378602B02D0072005B030BD134672
:1002D00004AA012542F8045D064D009506F0B6FC1F
:1002E0000028F2D1039BA34218BF092005B030BDFE
:1002F0000E207047B168020013460A46014660208E
:1003000005F0A6BF80B3F0B50C4685B0B9B106784C
:10031000692E14D101260396A2B19BB11E688EB13D
:1003200015461F4603AA2B46064605F0CBFF38B9F3
:100330002B685A1E022A08D9203B062B05D9072014
:1003400005B0F0BD0E2005B0F0BD002100913B4688
:1003500003AA3046214606F079FC0028F0D1039B21
:100360009C4218BF0920EBE70E207047F0B585B01E
:10037000CDE9003039B332B316680020144669273E
:100380000390324603AB0DF10B000D468DF80B7058
:1003900005F0DAFF08B105B0F0BD03AB32462946DF
:1003A00001A805F06DFF0028F5D1019B002B71D14C
:1003B0000A9B43B1009B5A1E022A07D9203B062BF9
:1003C00004D90720E7E70E2005B0F0BD03AB3246A5
:1003D0002946684605F054FF0028DCD1009B013B0C
:1003E000252BF0D801A252F823F000BFBB04020075
:1003F000B7040200B3040200C7030200C7030200EF
:10040000C7030200C7030200C7030200C7030200BC
:10041000C7030200C7030200C7030200C7030200AC
:10042000C7030200C7030200C7030200C70302009C
:10043000C7030200C7030200C7030200C70302008C
:10044000C7030200C7030200C7030200C70302007C
:10045000C7030200C7030200C7030200C70302006C
:10046000C7030200C7030200AF040200AB0402008E
:10047000A7040200A30402009F0402009B040200E0
:10048000850402000E4F0A9803AB32462946B8474E
:10049000002880D1039B23607DE70A4FF3E70A4FD2
:1004A000F1E70A4FEFE70A4FEDE70A4FEBE70A4F94
:1004B000E9E70A4FE7E70A4FE5E70A4FE3E700BF3E
:1004C000613A0200913A0200E937020091370200D6
:1004D00049370200B136020039360200B96B02001A
:1004E000B9690200296902002DE9F04184B000B326
:1004F000D1B10678682E17D101260396CAB1C3B1CF
:100500001E68B6B190461F4603AA434606460D46EE
:1005100005F0D8FE044640B9D8F800305A1E022A29
:100520000CD9203B062B09D90724204604B0BDE88E
:10053000F0810E24204604B0BDE8F0810023009332
:1005400003AA3B462946304606F080FB04460028B5
:10055000EBD13B68002B59D0D8F80020013A252A6E
:10056000E7D801A151F822F0330602003706020055
:100570002F06020033050200330502003305020096
:100580003305020033050200330502003305020083
:100590003305020033050200330502003305020073
:1005A0003305020033050200330502003305020063
:1005B0003305020033050200330502003305020053
:1005C0003305020033050200330502003305020043
:1005D0003305020033050200330502003305020033
:1005E000330502002B060200270602002306020044
:1005F0001F0602001B060200170602000106020089
:100600000F4F03AA30462946B847B0B9039B9D4215
:1006100018BF092489E70B4FF3E70B4FF1E70B4FA6
:10062000EFE70B4FEDE70B4FEBE70B4FE9E70B4F16
:10063000E7E70B4FE5E70B4FE3E7044675E700BF3D
:10064000793A0200C93A020011380200B9370200B3
:100650006D370200FD36020071360200E16B0200C8
:1006600071690200456A020013460A460146682085
:1006700005F0EEBD18B3F0B50C4685B019B106789B
:10068000622E054602D0072005B0F0BD04AF1E461D
:100690001346012247F8042D3A4605F041FE002892
:1006A000F2D1009033463A462846214606F0CEFA6B
:1006B0000028E9D1039B9C4218BF0920E4E70E20E3
:1006C000704700BFF0B587B0039001B3FAB1176867
:1006D00000201D4614464FF0620C05903A4605ABCB
:1006E0000DF113000E468DF813C005F02DFE08B174
:1006F00007B0F0BD05AB3A46314603A805F0C0FD92
:100700000028F5D1039B2BB1059B2360F0E70E2059
:1007100007B0F0BD054B00933A4605AB314628467D
:1007200006F076FA0028EFD0E2E700BF4963020046
:1007300038B370B50C4684B0E9B10678672E1AD18B
:1007400001260396D2B1CBB11E68BEB11D46134639
:1007500003AA064605F0E4FD70B90B4B009303AA0B
:100760002B463046214606F071FA28B9039BA34276
:1007700018BF092000E0072004B070BD0E2004B0AF
:1007800070BD0E20704700BFDD6A020013460A46A6
:100790000146672005F05CBD10B3F0B50C4685B08E
:1007A00019B10678642E054602D0072005B0F0BDC9
:1007B00004AE012746F8047D0092324605F018FE8B
:1007C0000028F3D10090324628460A9B214606F0C5
:1007D0003DFA0028EAD1039BA34218BF0920E5E7B0
:1007E0000E207047F0B587B0039001B3FAB11768D7
:1007F00000201D4614464FF0640C05903A4605ABA8
:100800000DF113000E468DF813C005F09DFD08B1E3
:1008100007B0F0BD05AB3A46314603A805F030FD00
:100820000028F5D1039B2BB1059B2360F0E70E2038
:1008300007B0F0BD054B00933A4605AB314628465C
:1008400006F0E6F90028EFD0E2E700BF7567020086
:10085000002839D070B50C4684B000292ED0067817
:10086000652E05462AD10126039652B34BB3089E46
:100870003EB316682EB31E681EB3089E366806B3D4
:100880001E461346114A009203AA06F0DFF9B0B9DA
:1008900000220092334603AA2146284606F0D6F9E4
:1008A00068B9009003AA2846089B214606F0CEF9B5
:1008B00028B9039B9C4218BF092000E0072004B020
:1008C00070BD0E2004B070BD0E207047AD670200F1
:1008D000F0B587B003908DF80B3009B302B31768F9
:1008E000002065240590154605AB3A460DF113002E
:1008F0008DF813400E4605F027FD044610B1204642
:1009000007B0F0BD05AB3A46314603A805F0B8FC88
:1009100004460028F3D1039B33B1059B2B60EEE71F
:100920000E24204607B0F0BD05AB3A4631460DF126
:100930000B0005F009FD04460028E0D10C9B002BBC
:10094000EBD0184605AB00939DF80B103B463246A2
:1009500005F0A4FE0028E0D00446D0E750B370B5FF
:100960000C4684B001B30678632E1DD10126039690
:10097000EAB1E3B11668D6B11E68C6B11D4613468A
:100980000D4A009203AA064606F060F968B9009085
:100990002B4603AA3046214606F058F928B9039B96
:1009A0009C4218BF092000E0072004B070BD0E2053
:1009B00004B070BD0E2070470D680200F0B587B01E
:1009C000039001B3FAB1176800201D4614464FF09A
:1009D000630C05903A4605AB0DF113000E468DF8F9
:1009E00013C005F0B1FC08B107B0F0BD05AB3A4645
:1009F000314603A805F044FC0028F5D1039B2BB138
:100A0000059B2360F0E70E2007B0F0BD054B009377
:100A10003A4605AB3146284606F0FAF80028EFD0F2
:100A2000E2E700BF49630200F8B130B50C4685B07B
:100A3000A9B10378662B4FF0000510D10123039371
:100A400082B1136873B11346009503AA06F0FEF84D
:100A500030B9039B9C4218BF092005B030BD072068
:100A600005B030BD0E2005B030BD0E20704700BF70
:100A7000F0B585B0019049B342B3176800201D4618
:100A800014464FF0660C03903A4603AB0DF10B0091
:100A90000E468DF80BC005F057FC08B105B0F0BD4F
:100AA00003AB3A46314601A805F0EAFB0028F5D130
:100AB000019B43B955B103AB3A463146284606F08F
:100AC0002BF80028EAD1039B2360E7E70E2005B04E
:100AD000F0BD00BFB0B199B110B50378682B82B0FA
:100AE00008D10123019342B1134601AA05F0EAFBA4
:100AF00002B010BD072002B010BD0E2002B010BD24
:100B0000072070470E20704728B322B3F0B583B09A
:100B100002AD002345F8043D1446531C2A460E46F8
:100B2000074605F023FC08B103B0F0BD23462A4672
:100B30003146384605F01AFC0028F5D1631D2A46D7
:100B40003846314605F012FC0028EDD1019B9E424B
:100B500018BF0920E8E70E20704700BF10B584B029
:100B6000019071B16AB1144604AB002243F8042D20
:100B700001A8226805F084FB08B9039B236004B038
:100B800010BD0E2004B010BD002A43D0002B41D070
:100B900000283FD010B40488013C6F2C00F2E080A4
:100BA000DFE804F0DAD6D2CEDEDEDEDEDEDEDEDE4A
:100BB000DEDEDECAC6C2BEBAB6B2AEAAA6A29E9A91
:100BC00096928E8ADEDEDEDEDEDEDEDEDEDEDEDE7D
:100BD000DEDEDE86827E7A76726E6A66625E5ADE5D
:100BE000DEDEDEDEDEDEDEDEDEDEDEDEDEDEDEDE25
:100BF000DEDEDE56524E4A46423EDEDEDEDEDEDE21
:100C0000DEDEDEDEDEDEDEDEDEDEDEDEDEDEDEDE04
:100C1000DEDEDE3A0E2070475DF8044B05F0E4BAE4
:100C20005DF8044B04F084BE5DF8044B04F010BF83
:100C30005DF8044B04F01CBE5DF8044B04F0E4BD09
:100C40005DF8044B04F040BE5DF8044B04F07CBD3D
:100C50005DF8044B04F0A0BE5DF8044B03F0BCBC8F
:100C60005DF8044B03F044BD5DF8044B03F09CBBFE
:100C70005DF8044B03F0F6BC5DF8044B03F008BBD1
:100C80005DF8044B03F01CBC5DF8044B03F0BABAEA
:100C90005DF8044B03F02ABA5DF8044B03F03EBB49
:100CA0005DF8044B03F068BA5DF8044B03F04EBCEA
:100CB0005DF8044B03F0BEBB5DF8044B01F0BEBC15
:100CC0005DF8044B01F0DEBA5DF8044B01F05CBD49
:100CD0005DF8044B01F0DEB95DF8044B01F07ABC1D
:100CE0005DF8044B01F084BD5DF8044B01F0FEBAE1
:100CF0005DF8044B01F036BA5DF8044B01F0DEBB41
:100D00005DF8044B01F0FAB95DF8044B01F0A2BBA9
:100D10005DF8044B01F018BC5DF8044B01F0CCBC4D
:100D20005DF8044B01F0FCBC5DF8044B01F076BAB1
:100D30005DF8044B01F042BB5DF8044B01F00ABBC7
:100D40005DF8044B00F0C8B85DF8044B00F00EB835
:100D50005DF8044B00F08CB85DF8044B00F054B81B
:100D6000002206201A605DF8044B7047E0B1DAB14A
:100D7000D3B10188032901D007207047F0B585B0B1
:100D80001F68ADF80A10154604461E464FF0000CC9
:100D90003A4603AB29460DF10A00CDF80CC005F028
:100DA000A9FA18B105B0F0BD0E20704703AB3A4662
:100DB0002946201D05F09EFA0028F3D103AB3A46E0
:100DC000294604F1080005F0BFFA0028EAD103AB78
:100DD0003A46294604F1100005F08CFA0028E1D1CA
:100DE000D4F80CC0009003AB3A462946604605F0A3
:100DF0000FFF0028D6D1A08805F0DEFF0028D1D152
:100E0000039B3360CEE700BFE0B1DAB1D3B1018814
:100E1000012901D007207047F0B583B01F68ADF8F5
:100E20000210154604461E464FF0000C3A4601AB30
:100E300029460DF10200CDF804C005F05BFA18B1A7
:100E400003B0F0BD0E20704701AB3A462946201D85
:100E500005F050FA0028F3D101AB3A46294604F1D7
:100E6000080005F071FA0028EAD1019B3360E7E73A
:100E7000E0B1DAB1D3B10188022901D0072070476F
:100E8000F0B583B01F68ADF80210154604461E4643
:100E90004FF0000C3A4601AB29460DF10200CDF8A7
:100EA00004C005F027FA18B103B0F0BD0E2070475A
:100EB00001AB3A462946201D05F01CFA0028F3D163
:100EC00001AB3A46294604F1080005F03DFA002836
:100ED000EAD1019B3360E7E7E0B1DAB1D3B1018831
:100EE000042901D007207047F0B583B01F68ADF822
:100EF0000210154604461E464FF0000C3A4601AB60
:100F000029460DF10200CDF804C005F0F3F918B13F
:100F100003B0F0BD0E20704701AB3A462946201DB4
:100F200005F0E8F90028F3D101AB3A46294604F16F
:100F3000080005F015FE0028EAD1019B3360E7E7C1
:100F400038B370B50C4684B0E9B10678722E054608
:100F500019D101260396CBB1099EBEB11E4600965B
:100F6000134603AA05F044FA70B9099B009303AA3B
:100F70002846089B214605F03BFA28B9039BA3426B
:100F800018BF092000E0072004B070BD0E2004B097
:100F900070BD0E20704700BF13460A4601467220FE
:100FA00005F056B9F8B110B50C4684B0A9B1037874
:100FB000732B12D10123039392B1136883B15B6841
:100FC00073B11346094A009203AA05F03FFE28B9FF
:100FD000039BA34218BF092000E0072004B010BD06
:100FE0000E2004B010BD0E20704700BFBD390200B6
:100FF00013460A460146732005F02AB913460A46ED
:101000000146742005F024B9F8B130B50C4685B01E
:10101000A9B10378792B4FF0000510D10123039378
:1010200082B1136873B11346009503AA05F00EFE52
:1010300030B9039B9C4218BF092005B030BD072082
:1010400005B030BD0E2005B030BD0E20704700BF8A
:10105000F0B587B0039001B3FAB1176800201D46C0
:1010600014464FF0790C05903A4605AB0DF113008C
:101070000E468DF813C005F067F908B107B0F0BD52
:1010800005AB3A46314603A805F0FAF80028F5D139
:10109000039B2BB1059B2360F0E70E2007B0F0BD4A
:1010A000054B00933A4605AB3146284605F0B0FDA6
:1010B0000028EFD0E2E700BFF5620200D0B110B522
:1010C0000C4682B081B10378782B0DD101230193B6
:1010D0006AB1134601AA05F023F930B9019BA34276
:1010E00018BF092002B010BD072002B010BD0E20AD
:1010F00002B010BD0E20704713460A460146782004
:1011000005F0A6B8002833D070B50C4684B049B3BA
:101110000678802E054625D1012603962AB323B3EF
:101120001E46134603AA05F0FBF8E0B9334603AAAE
:101130002146284605F01AF9A8B93378012B19D0B1
:1011400002D3022B0ED11020CDE9000003AA2846BD
:10115000089B214605F076FA28B9039B9C4218BFEC
:10116000092000E0072004B070BD0E2004B070BD5F
:101170000E2070470620E7E713460A460146802006
:1011800005F066B838B370B50C4684B0E9B106789E
:101190007E2E1AD101260396D2B1CBB11E68BEB104
:1011A0001D46134603AA064605F0BAF870B90B4B64
:1011B000009303AA2B463046214605F047FD28B987
:1011C000039BA34218BF092000E0072004B070BDB4
:1011D0000E2004B070BD0E20704700BF89300200A1
:1011E00013460A4601467E2005F032B838B370B582
:1011F0000C4684B0E9B10678752E1AD10126039603
:10120000D2B1CBB11E68BEB11D46134603AA064635
:1012100005F086F870B90B4B009303AA2B463046B5
:10122000214605F013FD28B9039BA34218BF0920EE
:1012300000E0072004B070BD0E2004B070BD0E2089
:10124000704700BF1933020013460A460146752055
:1012500004F0FEBF18B370B50C4684B0C9B106786F
:10126000872E054615D101260396AAB11E461346C0
:1012700003AA05F055F868B90090334603AA28463A
:10128000214605F0E3FC28B9039BA34218BF0920BF
:1012900000E0072004B070BD0E2004B070BD0E2029
:1012A000704700BFF0B587B003900AB303B31F685F
:1012B000144600201D460E464FF0870C05903A4616
:1012C00005AB21460DF113008DF813C005F03CF875
:1012D00008B107B0F0BD05AB3A46214603A804F0BB
:1012E000CFFF0028F5D1039B2BB1059B2B60F0E7C6
:1012F0000E2007B0F0BD054B00933A4605AB2146E2
:10130000304605F085FC0028EFD0E2E7F12E020020
:10131000002839D070B50C4684B000292ED006784C
:101320008C2E05462AD10126039652B3166846B381
:101330003BB31E682EB3089E1EB336680EB31E461E
:101340001346124A009203AA05F080FCB8B9104B6C
:10135000009303AA33462146284605F077FC70B96E
:101360000C4B009303AA2846089B214605F06EFC0F
:1013700028B9039BA34218BF092000E0072004B04E
:1013800070BD0E2004B070BD0E20704745290200CC
:10139000C93302001933020013460A4601468C2065
:1013A00004F056BF13460A4601468D2004F050BF94
:1013B00020B3F0B50C4685B0D1B107787D2F054636
:1013C00016D101270397B3B116460D4A009203AA1E
:1013D00005F03CFC68B90090334603AA2846214634
:1013E00005F034FC28B9039BA34218BF092000E094
:1013F000072005B0F0BD0E2005B0F0BD0E207047EF
:10140000216302002DE9F04387B003900E9E2BB3B9
:1014100026B3D6F800901D4600207D240590904606
:101420000F464A4605AB29460DF113008DF81340CF
:1014300004F08AFF044618B1204607B0BDE8F083E7
:1014400005AB4A46294603A804F01AFF04460028C3
:10145000F2D1039B3BB1059B3360EDE70E242046A0
:1014600007B0BDE8F0830D4B00934A4605AB294613
:10147000404605F0CDFB04460028DDD1B8F1000F51
:10148000E9D005ABB8F8001000932A464B46384621
:1014900005F004F90028DED00446CDE7F56202002D
:1014A00048B370B50C4684B0F9B106787C2E054679
:1014B0001BD101260396DAB1D3B1089EC6B11E46F0
:1014C00013460E4A009203AA05F0C0FB70B9089BB0
:1014D000009303AA33462846214604F0E5FF28B9C5
:1014E000039BA34218BF092000E0072004B070BD91
:1014F0000E2004B070BD0E20704700BF692E0200A0
:1015000013460A4601467C2004F0A2BE18B370B50B
:101510000C4682B0C9B10678762E054615D1012653
:101520000196AAB1A3B11E46134601AA04F0F8FE23
:1015300060B9334601AA2846214604F017FF28B9AE
:10154000019BA34218BF092000E0072002B070BD34
:101550000E2002B070BD0E20704700BF13460A4631
:101560000146762004F074BE002834D070B50C46D5
:1015700084B051B30678852E054626D10126039600
:1015800032B3089E26B31BB336680EB31E68FEB195
:101590001E46134603AA04F0C3FEB8B90F4B0093CE
:1015A00003AA33462146284605F050FB70B90C4B80
:1015B000009303AA2846089B214605F047FB28B95B
:1015C000039B9C4218BF092000E0072004B070BDB7
:1015D0000E2004B070BD0E20704700BF893302009A
:1015E000052D020013460A460146852004F030BE50
:1015F00018B370B50C4682B0C9B10678822E054684
:1016000015D101260196AAB1A3B11E46134601AA1F
:1016100004F086FE60B9334601AA2846214604F04C
:10162000A5FE28B9019BA34218BF092000E00720AE
:1016300002B070BD0E2002B070BD0E20704700BF1A
:1016400013460A460146822004F002BE28B370B554
:101650000C4684B0D9B10678812E054617D10126F3
:101660000396BAB1B3B11E46134603AA04F058FE5E
:1016700070B90B4B009303AA33462846214605F068
:10168000E5FA28B9039BA34218BF092000E0072010
:1016900004B070BD0E2004B070BD0E20704700BFB6
:1016A0009D38020013460A460146812004F0D0BD51
:1016B00078B370B50C4684B029B30678832E0546FE
:1016C00021D1012603960AB3089EFEB1F3B11E464E
:1016D000134603AA04F024FEB0B90F4B009303AAEB
:1016E00033462146284605F0B1FA68B9009003AAAE
:1016F0002846089B214605F0A9FA28B9039BA34276
:1017000018BF092000E0072004B070BD0E2004B00F
:1017100070BD0E20704700BFB9290200F0B587B038
:1017200003900AB303B31F68144600201D460E46FB
:101730004FF0830C05903A4605AB21460DF113009E
:101740008DF813C004F000FE08B107B0F0BD05AB82
:101750003A46214603A804F093FD0028F5D1039BE7
:101760002BB1059B2B60F0E70E2007B0F0BD054BB9
:1017700000933A4605AB2146304605F049FA002869
:10178000EFD0E2E7BD38020078B3F0B50C4685B083
:1017900029B30678842E054621D1012603960AB383
:1017A00003B30A9EF6B11E46134603AA04F0B8FD21
:1017B000B0B90F4F0097334603AA2146284605F0DB
:1017C00045FA68B9009703AA28460A9B214605F006
:1017D0003DFA28B9039BA34218BF092000E0072067
:1017E00005B0F0BD0E2005B0F0BD0E20704700BF63
:1017F0003539020013460A460146842004F028BD0C
:1018000008B330B50C4685B0B9B103787B2B4FF0E7
:10181000000512D10123039392B1136883B101290A
:1018200008D91346009503AA05F010FA30B9039BB6
:101830009C4203D0092005B030BD072005B030BD63
:101840000E2005B030BD0E20704700BFF0B587B048
:10185000039001B3FAB1176800201D4614464FF0FB
:101860007B0C05903A4605AB0DF113000E468DF842
:1018700013C004F069FD08B107B0F0BD05AB3A46EE
:10188000314603A804F0FCFC0028F5D1039B2BB1E2
:10189000059B2360F0E70E2007B0F0BD054B0093D9
:1018A0003A4605AB3146284605F0B2F90028EFD09C
:1018B000E2E700BFC1320200E0B110B50C4684B0CF
:1018C00091B103787A2B0FD1012303937AB1134698
:1018D000094A009203AA05F0B9F930B9039BA34263
:1018E00018BF092004B010BD072004B010BD0E20A1
:1018F00004B010BD0E2070471933020013460A468B
:1019000001467A2004F0A4BC30B370B50C4684B014
:10191000E1B106788E2E054618D101260396C2B194
:10192000BBB11E68AEB11E46134603AA04F0F8FC14
:1019300068B90090334603AA2846214605F086F987
:1019400028B9039B9C4218BF092000E0072004B07F
:1019500070BD0E2004B070BD0E207047F0B585B08C
:1019600001908DF80330F1B1EAB1166800201546F8
:101970008E270390324603AB0DF10B000C468DF819
:101980000B7004F0E1FC08B105B0F0BD03AB3246CA
:10199000214601A804F074FC0028F5D1019B2BB16D
:1019A000039B2B60F0E70E2005B0F0BD03AB324681
:1019B00021460DF1030004F0C7FC0028F0D0E3E756
:1019C00060B370B50C4682B011B30678882E054618
:1019D0001ED101260196F2B1EBB1069EDEB11E4684
:1019E000134601AA04F09CFC98B9334601AA21468B
:1019F000284604F0BBFC60B901AA2846069B214694
:101A000004F0B4FC28B9019BA34218BF092000E0F0
:101A1000072002B070BD0E2002B070BD0E207047CE
:101A200013460A460146882004F012BCD0B110B516
:101A30000C4682B081B10378892B0DD1012301932B
:101A40006AB1134601AA04F06BFC30B9019BA342B2
:101A500018BF092002B010BD072002B010BD0E2033
:101A600002B010BD0E20704713460A460146892079
:101A700004F0EEBBF0B110B50C4684B0A1B1037810
:101A80008A2B11D1012303938AB113687BB11346CA
:101A9000094A009203AA05F0D9F830B9039BA34282
:101AA00018BF092004B010BD072004B010BD0E20DF
:101AB00004B010BD0E207047C933020013460A4619
:101AC00001468A2004F0C4BB13460A4601468B2017
:101AD00004F0BEBB00284BD0002947D070B5047875
:101AE000862C84B03CD101240394002A3BD0002BE7
:101AF00039D0089C002C36D0099C002C33D01C68AF
:101B0000002C30D0089C24686CB3099C246854B322
:101B10001D46134603AA04460E4604F001FC00BB12
:101B2000144B009303AA2B463146204605F08EF84D
:101B3000B8B9114B009303AA089B3146204605F023
:101B400085F870B90D4B009303AA2046099B3146D6
:101B500005F07CF828B9039B9E4218BF092000E0DD
:101B6000072004B070BD0E2004B070BD0720704780
:101B70000E207047052D0200252902009929020038
:101B800013460A460146862004F062BB002840D076
:101B900070B50C4684B0002935D006787F2E0546F6
:101BA00031D101260396002A30D0002B2ED0089E7A
:101BB00066B3366856B3099E46B3366836B31E46DA
:101BC000134603AA04F0ACFBF0B9334603AA21463E
:101BD000284604F0CBFBB8B90F4B009303AA089B2F
:101BE0002146284605F032F870B90C4B009303AA41
:101BF0002846099B214605F029F828B9039BA342F2
:101C000018BF092000E0072004B070BD0E2004B00A
:101C100070BD0E20704700BF8930020021350200E0
:101C2000F0B587B0039001B3FAB1176800201D46E4
:101C300014464FF07F0C05903A4605AB0DF11300AA
:101C40000E468DF813C004F07FFB08B107B0F0BD5D
:101C500005AB3A46314603A804F012FB0028F5D143
:101C6000039B2BB1059B2360F0E70E2007B0F0BD6E
:101C7000054B00933A4605AB3146284604F0C8FFB1
:101C80000028EFD0E2E700BF41340200D0B110B528
:101C90000C4682B081B10378772B0DD101230193DB
:101CA0006AB1134601AA04F061FB30B9019BA3425B
:101CB00018BF092002B010BD072002B010BD0E20D1
:101CC00002B010BD0E20704713460A460146772029
:101CD00004F0BEBAD8B170B50C4684B021B1037817
:101CE0006D2B4FF0000502D0072004B070BD1346E5
:101CF00004AA012642F8046D009504F0A7FF00280D
:101D0000F3D1039B9C4218BF092004B070BD0E2084
:101D1000704700BFF0B585B0019049B342B3176872
:101D200000201D4614464FF06D0C03903A4603AB5D
:101D30000DF10B000E468DF80BC004F005FB08B149
:101D400005B0F0BD03AB3A46314601A804F098FA5D
:101D50000028F5D1019B43B955B103AB3A46314652
:101D6000284600F08DFD0028EAD1039B2360E7E7B9
:101D70000E2005B0F0BD00BFD0B130B50C4685B027
:101D800011B103786C2B02D0072005B030BD13468B
:101D900004AA012542F8045D064D009504F056FFA3
:101DA0000028F2D1039BA34218BF092005B030BD23
:101DB0000E2070474529020013460A4601466C2052
:101DC00004F046BAD0B130B50C4685B011B10378F5
:101DD000702B02D0072005B030BD134604AA0125A0
:101DE00042F8045D064D009504F030FF0028F2D162
:101DF000039BA34218BF092005B030BD0E207047D9
:101E00005D3B020013460A460146702004F020BAEA
:101E1000D0B130B50C4685B011B10378712B02D02A
:101E2000072005B030BD134604AA012542F8045D21
:101E3000064D009504F00AFF0028F2D1039B9C4256
:101E400018BF092005B030BD0E2070475D3B020071
:101E5000F0B587B0039001B3FAB1176800201D46B2
:101E600014464FF0710C05903A4605AB0DF1130086
:101E70000E468DF813C004F067FA08B107B0F0BD44
:101E800005AB3A46314603A804F0FAF90028F5D12B
:101E9000039B2BB1059B2360F0E70E2007B0F0BD3C
:101EA000054B00933A4605AB3146284604F0B0FE98
:101EB0000028EFD0E2E700BF013B02002DE9F04728
:101EC00084B058B329B307786E2F22D10127039726
:101ED00022B3176817B33F6807B3164603AA98469C
:101EE00007460D4604F042FA044698B90DF10B037B
:101EF00003AA2946384604F039FA044650B99DF839
:101F00000B30012B0FD03060039BAB4218BF09246C
:101F100000E00724204604B0BDE8F0870E242046E8
:101F200004B0BDE8F08798F800303668002BEBD09D
:101F3000DFF82CA04FF0000903E098F800304B4583
:101F4000E2D93346CDF800A003AA2946384604F06A
:101F50007DFE09F1010904360028EED00446D9E7D8
:101F60004529020013460A4601466E2004F070B966
:101F70002DE9F04784B0002843D000293CD00678F2
:101F80006F2E074638D101260396002A39D01668ED
:101F9000002E36D03668A6B39BB31E688EB3366863
:101FA0007EB3984616460C9B03AA0D4604F0DEF954
:101FB000044610BB0DF10B0303AA2946384604F072
:101FC000D5F90446C8B99DF80B30012B1ED03060FE
:101FD0000DF10B0303AA2946384604F0C7F904465D
:101FE00058B99DF80B30012B2CD0C8F80000039B8A
:101FF000AB4218BF092400E00724204604B0BDE826
:10200000F0870E24204604B0BDE8F0870C9B3668AC
:102010001B78002BDCD0DFF868A0814603E00C9B26
:102020001B784B45D4D93346CDF800A003AA2946E6
:10203000384604F00BFE09F1010904460436002875
:10204000EDD0DAE70C9BD8F800601B78002BCED0DF
:10205000DFF83090804603E00C9B1B784345C6D9DF
:102060003346CDF8009003AA2946384604F0EEFD29
:1020700008F1010804360028EED00446BDE700BF91
:102080006D2B02002529020013460A4601466F20E7
:1020900004F0DEB8E0B1DAB1D3B101881D2901D076
:1020A00007207047F0B583B01F68ADF802101546E1
:1020B00004461E464FF0000C3A4601AB29460DF18E
:1020C0000200CDF804C004F015F918B103B0F0BD5A
:1020D0000E20704701AB3A462946201D04F00AF94C
:1020E0000028F3D101AB3A46294604F1080000F07C
:1020F0009DFD0028EAD1019B3360E7E7E0B1DAB14A
:10210000D3B10188172901D007207047F0B583B0FB
:102110001F68ADF80210154604461E464FF0000C2D
:102120003A4601AB29460DF10200CDF804C004F097
:10213000E1F818B103B0F0BD0E20704701AB3A468C
:102140002946201D04F0D6F80028F3D101AB3A4609
:10215000294604F1080004F0F7F80028EAD1019BB1
:102160003360E7E72DE9F04184B0002839D0002A38
:1021700037D0002B35D00188192904D007252846EF
:1021800004B0BDE8F081D3F80080ADF80610164623
:10219000002504461F46424602AB31460DF10600BB
:1021A000029504F0A7F805460028E8D102AB4246A4
:1021B0003146201D04F09EF805460028DFD102AB11
:1021C0004246314604F1080000F0CAFD05460028E9
:1021D000D5D103A9A08804F099FD38B1029B3B60DA
:1021E000CDE70E25284604B0BDE8F0810A48314607
:1021F000039E4FF4967C02AB42460CFB060001F0B6
:102200001FF908B10546BAE7A08804F069FD002867
:10221000E4D00546B3E700BF407E0020E0B1DAB16C
:10222000D3B10188122901D007207047F0B583B0DF
:102230001F68ADF80210154604461E464FF0000C0C
:102240003A4601AB29460DF10200CDF804C004F076
:1022500051F818B103B0F0BD0E20704701AB3A46FB
:102260002946201D04F046F80028F3D101AB3A4678
:10227000294604F1080000F0CBFF0028EAD1019BB9
:102280003360E7E7E0B1DAB1D3B101881F2901D0AB
:1022900007207047F0B583B01F68ADF802101546EF
:1022A00004461E464FF0000C3A4601AB29460DF19C
:1022B0000200CDF804C004F01DF818B103B0F0BD61
:1022C0000E20704701AB3A462946201D04F012F853
:1022D0000028F3D101AB3A46294604F1080000F08A
:1022E000C3FF0028EAD1019B3360E7E7E0B1DAB130
:1022F000D3B101881A2901D007207047F0B583B007
:102300001F68ADF80210154604461E464FF0000C3B
:102310003A4601AB29460DF10200CDF804C003F0A6
:10232000E9FF18B103B0F0BD0E20704701AB3A468B
:102330002946201D03F0DEFF0028F3D101AB3A4609
:10234000294604F1080000F0ABFD0028EAD1019B0A
:102350003360E7E7E0B1DAB1D3B10188102901D0E9
:1023600007207047F0B583B01F68ADF8021015461E
:1023700004461E464FF0000C3A4601AB29460DF1CB
:102380000200CDF804C003F0B5FF18B103B0F0BDF2
:102390000E20704701AB3A462946201D03F0AAFFE4
:1023A0000028F3D101AB3A46294604F1080000F0B9
:1023B00013FE0028EAD1019B3360E7E72DE9F041E5
:1023C00084B0002839D0002A37D0002B35D00188BE
:1023D000112904D00726304604B0BDE8F081D3F8B7
:1023E0000080ADF806101546002604461F464246FA
:1023F00002AB29460DF10600029603F07BFF06466C
:102400000028E8D102AB42462946201D03F072FFA6
:1024100006460028DFD102AB4246294604F10800F7
:1024200000F0A6FF06460028D5D103A9A08804F035
:102430006DFC38B1029B3B60CDE70E26304604B000
:10244000BDE8F081A08804F04BFC0028F2D00646DD
:10245000C1E700BFE0B1DAB1D3B10188162901D0DC
:1024600007207047F0B583B01F68ADF8021015461D
:1024700004461E464FF0000C3A4601AB29460DF1CA
:102480000200CDF804C003F035FF18B103B0F0BD71
:102490000E20704701AB3A462946201D03F02AFF63
:1024A0000028F3D101AB3A46294604F1080003F0B5
:1024B0004BFF0028EAD1019B3360E7E7E0B1DAB1D6
:1024C000D3B10188182901D007207047F0B585B035
:1024D0001F68ADF80A10154604461E464FF0000C62
:1024E0003A4603AB29460DF10A00CDF80CC003F0C3
:1024F00001FF18B105B0F0BD0E20704794F80CC074
:1025000003ABCCF3000C3A462946201D8DF809C0D8
:1025100003F0F0FE0028EDD10A4BA06800933A4684
:1025200003AB294604F074FB0028E3D103AB3A4621
:1025300029460DF1090003F007FF0028DAD1039BBB
:102540003360D7E7FD280200E0B1DAB1D3B10188EA
:10255000152901D007207047F0B585B01F68ADF888
:102560000A10154604461E464FF0000C3A4603ABCF
:1025700029460DF10A00CDF80CC003F0BBFE18B1DE
:1025800005B0F0BD0E20704794F80EC003ABCCF33D
:10259000000C3A462946201D8DF809C003F0AAFE1A
:1025A0000028EDD103AB009304F108003B462A4616
:1025B000062104F073F80028E2D103AB3A4629461D
:1025C0000DF1090003F0C0FE0028D9D1039B336050
:1025D000D6E700BFE0B1DAB1D3B101881C2901D040
:1025E00007207047F0B583B01F68ADF8021015469C
:1025F00004461E464FF0000C3A4601AB29460DF149
:102600000200CDF804C003F075FE18B103B0F0BDB0
:102610000E20704701AB3A462946201D03F06AFEA2
:102620000028F3D101AB3A46294604F1080003F033
:102630008BFE0028EAD1019B3360E7E7E0B1DAB115
:10264000D3B10188202901D007207047F0B583B0AD
:102650001F68ADF80210154604461E464FF0000CE8
:102660003A4601AB29460DF10200CDF804C003F053
:1026700041FE18B103B0F0BD0E20704701AB3A46E1
:102680002946201D03F036FE0028F3D101AB3A465F
:10269000294604F1090000F0F3F80028EAD101AB63
:1026A0003A46294604F1080003F04EFE0028E1D125
:1026B000019B3360DEE700BFE0B1DAB1D3B101883E
:1026C000142901D007207047F0B583B01F68ADF81A
:1026D0000210154604461E464FF0000C3A4601AB68
:1026E00029460DF10200CDF804C003F003FE18B135
:1026F00003B0F0BD0E20704701AB3A462946201DBD
:1027000003F0F8FD0028F3D101AB3A46294604F165
:10271000080000F013FC0028EAD1019B3360E7E7D2
:10272000E0B1DAB1D3B10188132901D00720704795
:10273000F0B583B01F68ADF80210154604461E467A
:102740004FF0000C3A4601AB29460DF10200CDF8DE
:1027500004C003F0CFFD18B103B0F0BD0E207047E8
:1027600001AB3A462946201D03F0C4FD0028F3D1F1
:1027700001AB3A46294604F1080000F0F3FC0028BA
:10278000EAD1019B3360E7E7E0B1DAB1D3B1018868
:102790001E2901D007207047F0B583B01F68ADF83F
:1027A0000210154604461E464FF0000C3A4601AB97
:1027B00029460DF10200CDF804C003F09BFD18B1CD
:1027C00003B0F0BD0E20704701AB3A462946201DEC
:1027D00003F090FD0028F3D101AB3A46294604F1FD
:1027E000080000F011FF0028EAD1019B3360E7E701
:1027F000E0B1DAB1D3B101881B2901D007207047BD
:10280000F0B583B01F68ADF80210154604461E46A9
:102810004FF0000C3A4601AB29460DF10200CDF80D
:1028200004C003F067FD18B103B0F0BD0E2070477F
:1028300001AB3A462946201D03F05CFD0028F3D188
:1028400001AB3A46294604F1080003F07DFD00285B
:10285000EAD1019B3360E7E761B15BB110B582B0AB
:1028600050B11C46009413460A46102103F016FF8F
:1028700002B010BD0E2070470E2002B010BD00BF88
:1028800031B32DE9F0411E4684B09BB190B104787C
:10289000054604F0FE0C04A8C4F300044CEA04044A
:1028A00000F8014D90460F4603F04EFD30B104B0E4
:1028B000BDE8F0810E2004B0BDE8F08100964346EB
:1028C0003A46681C062103F0E9FE04B0BDE8F08139
:1028D0000E20704761B15BB110B582B050B11C469B
:1028E000009413460A46102103F0D8FE02B010BD32
:1028F0000E2070470E2002B010BD00BF61B15BB169
:1029000010B582B050B11C46009413460A464021CF
:1029100003F0C4FE02B010BD0E2070470E2002B0BE
:1029200010BD00BF60B130B583B032B12BB11024FF
:10293000009403F0CBFE03B030BD0E2003B030BDD9
:102940000E20704730B3F0B5144685B052B14BB18C
:102950001D460DF10F0307460E4603F007FD20B19B
:1029600005B0F0BD0E2005B0F0BD06230093224651
:10297000314638466B1C03F0A9FE0028F0D19DF8C3
:102980000F202B7862F30003520862F347032B7089
:1029900005B0F0BD0E20704760B130B583B032B1E4
:1029A0002BB11024009403F091FE03B030BD0E2033
:1029B00003B030BD0E20704760B130B583B032B186
:1029C0002BB14024009403F081FE03B030BD0E20F3
:1029D00003B030BD0E207047A8B32DE9F041144676
:1029E00084B062B35BB31D460DF10F0307460E467C
:1029F000B5F80A8003F0BAFCF0B99DF80F302A78D8
:102A000063F303021B0963F307122A700DF10F032E
:102A100022463146384603F0A9FC68B96B789DF828
:102A20000F2062F301036B70224605F10803314663
:102A3000384603F075FC40B104B0BDE8F0810E20CB
:102A400004B0BDE8F0810E20704705F10A0322466C
:102A50003146384603F064FC0028EDD12B89019300
:102A6000CDF800802246314638462B1D03F0EAFDA2
:102A7000E2E700BF81B17BB1F0B5064685B078B31F
:102A80000C461D461746009313460A46102103F0D4
:102A900005FE18B105B0F0BD0E207047337C04A8C8
:102AA00003F0FE02C3F30003134300F8013D3A466E
:102AB0002B46214603F048FC0028EBD12B463A4632
:102AC000214606F1120003F015FC0028E2D1009522
:102AD0003B46224606F11400082103F0DFFDD9E74A
:102AE0000E2005B0F0BD00BF00283DD0F0B5144663
:102AF00085B062B11D4653B14FF0100CCDF800C047
:102B00000F46064603F0E2FD20B105B0F0BD0E20F1
:102B100005B0F0BD0DF10F0322463946304603F0F3
:102B200025FC0028F1D19DF80F202B7C510862F381
:102B3000000361F34103920862F387032B7422467A
:102B400005F112033946304603F0EAFB0028DCD1D8
:102B50004FF0080C05F11403224639463046CDF8F3
:102B600000C003F0B3FDD0E70E20704770B3F0B59E
:102B7000144685B03AB31E462BB34FF0100CCDF877
:102B800000C00D46074603F0A1FDD0B90DF10F03BB
:102B900022462946384603F0E9FB90B90623009304
:102BA00022462946384606F1110303F08FFD40B94D
:102BB0009DF80F20337C62F30003520862F3470351
:102BC000337405B0F0BD0E2005B0F0BD0E20704787
:102BD00039B333B3F0B5064685B020B30C461D4675
:102BE0001746009313460A46102103F057FDB0B96B
:102BF000337C04A803F0FE02C3F30003134300F880
:102C0000013D3A462B46214603F09EFB38B900951C
:102C10003B46224606F11100062103F03FFD05B0B8
:102C2000F0BD0E2070470E2005B0F0BD002967D022
:102C30002DE9F0471E4684B0F3B1E8B10578C47BB6
:102C40000DF1100A814605F0FE00C5F300050543AD
:102C50000AF8015DC4F3000C04F0060545EA0C0512
:102C6000504690460F468DF80E50E40803F06CFB7A
:102C700030B104B0BDE8F0870E2004B0BDE8F087A5
:102C8000009643463A46062109F1010003F006FD8D
:102C90000028EED199F8073003F0FE05C3F30003D6
:102CA0001D4350463346424639468DF80F5003F0D7
:102CB0004BFB0028DDD1009643463A46062109F138
:102CC000080003F0EBFC0028D3D1334642463946D6
:102CD00009F10E0003F038FB0028CAD13346424602
:102CE00039460DF10E0003F02FFB0028C1D10096EC
:102CF00043463A46214609F1100003F055FBB8E778
:102D00000E20704750B3F0B5144685B062B11D4631
:102D100053B14FF0100CCDF800C00E46074603F03B
:102D2000D5FC20B105B0F0BD0E2005B0F0BD2246A7
:102D3000314638460DF10F0303F018FB0028F1D19E
:102D40009DF80F202B7C510862F3000361F34103CF
:102D5000920862F387032B7405B0F0BD0E20704714
:102D6000002967D02DE9F0411E4682B093B1054697
:102D700080B1447804F0040CC4F301044CEA040468
:102D800090460F468DF8064003F0DEFA30B102B0EF
:102D9000BDE8F0810E2002B0BDE8F0813346424626
:102DA00039460DF1060003F0CFFA0028EFD1AB78D9
:102DB00002ACC3F3000203F00E03134304F8013D19
:102DC000424633462046394603F0BEFA0028DED19B
:102DD000EB78C3F3000C03F00E0343EA0C0C4246FD
:102DE0003346394620468DF807C003F0ADFA002877
:102DF000CDD12B79C3F3000C03F00E0343EA0C0C86
:102E000042463346394620468DF807C003F09CFA07
:102E10000028BCD16B79C3F3000C03F00E054246C9
:102E200033463946204645EA0C048DF8074003F046
:102E30008BFAACE70E20704799B130B583B06BB117
:102E400060B1007800F0F005C0F3030402A82C4341
:102E500000F8014D03F078FA03B030BD0E2003B046
:102E600030BD0E20704700BFB8B110B582B08AB136
:102E700083B11C460DF1070303F078FA40B99DF8C1
:102E80000720237862F30303120962F30713237008
:102E900002B010BD0E2002B010BD0E20704700BF62
:102EA00019B32DE9F0411E4682B09BB190B1047870
:102EB000054604F0F00C02A8C4F303044CEA040431
:102EC00000F8014D90460F4603F03EFA30B102B0D3
:102ED000BDE8F0810E2002B0BDE8F08133464246E5
:102EE0003946681C03F030FAF1E70E20704700BF46
:102EF00011B32DE9F0411E4682B0CBB1C0B10478C8
:102F0000054604F0F00C02A8C4F303044CEA0404E0
:102F100000F8014D90460F4603F016FA28B93346E3
:102F200042463946681C03F00FFA02B0BDE8F08152
:102F30000E2002B0BDE8F0810E207047002949D074
:102F40002DE9F0411D4684B0E3B1D8B104460078C4
:102F5000A67C00F0FE0EC0F3000C04A84EEA0C0C98
:102F600000F801CD06F0060CC6F300064CEA060692
:102F700090460F468DF80E6003F0E6F930B104B0CC
:102F8000BDE8F0810E2004B0BDE8F0810095434615
:102F90003A460621601C03F081FB0028EFD12B4646
:102FA0004246394604F1080003F0A4F90028E6D1AE
:102FB000009504F10A0043463A46082103F06EFBEF
:102FC0000028DCD12B46424639460DF10E0003F0B5
:102FD000BBF9D4E70E207047002952D02DE9F0410B
:102FE0001E4684B0002B48D0002846D00478054601
:102FF00004F0FE0C04A8C4F300044CEA040400F836
:10300000014D90460F4603F09FF910B104B0BDE8A2
:10301000F081009643463A460621681C03F03EFBC9
:103020000028F3D1334642463946E81D03F08CF9B7
:103030000028EBD133464246394605F1080003F03B
:1030400059F90028E2D133464246394605F10A00D3
:1030500003F050F90028D9D133464246394605F1EC
:103060000C0003F047F90028D0D1334642463946D8
:1030700005F10E0003F03EF9C8E70E2004B0BDE8EC
:10308000F0810E20704700BF002869D0F0B51446CB
:1030900083B052B14BB11D460DF1060307460E46F3
:1030A00003F064F920B103B0F0BD0E2003B0F0BD11
:1030B0006B1C22463146384603F058F90028F2D1FD
:1030C000AB1C22463146384603F050F90028EAD1BD
:1030D0000DF1070322463146384603F047F9002830
:1030E000E1D19DF8073095F803C05A0863F3000C4E
:1030F00062F3410C9A0862F3820CDB0863F3C30CA1
:1031000022460DF107033146384685F803C003F027
:103110002DF90028C7D19DF806102B789DF807409F
:103120004A0861F3000362F341038A08CE0862F3A0
:1031300082032A7966F3C3030E0964F3000266F37F
:103140000613660866F34102A60866F38202C909FF
:10315000E40861F3C71364F3C3022B702A71A2E77A
:103160000E207047002951D02DE9F0411D4682B054
:103170009BB190B104788046C4F3000C02A804F01F
:10318000FE0444EA0C0400F8024D17460E4603F014
:10319000DBF830B102B0BDE8F0810E2002B0BDE82E
:1031A000F0812B463A46314608F1010003F0CCF895
:1031B0000028EFD12B463A46314608F1020003F0D1
:1031C000C3F80028E6D198F8033002ACC3F300023C
:1031D00003F00E03134304F8013D3A462B46204604
:1031E000314603F0B1F80028D4D198F80430C3F385
:1031F000000E03F00E0C3A462B46314620464CEAB0
:103200000E048DF8074003F09FF8C3E70E207047C7
:1032100039B32DE9F0411C4643B1054630B117469C
:103220000E4603F067F820B1BDE8F0810E20BDE83E
:10323000F08123463A463146A81C03F05BF800288B
:10324000F2D123463A463146281D03F053F80028B0
:10325000EAD123463A463146A81DBDE8F04103F0C5
:1032600049B80E20704700BF39B32DE9F0411C4624
:1032700043B1054630B117460E4603F03BF820B186
:10328000BDE8F0810E20BDE8F08123463A46314684
:10329000A81C03F02FF80028F2D123463A46314605
:1032A000281D03F027F80028EAD123463A46314684
:1032B000A81DBDE8F04103F01DB80E20704700BF07
:1032C00039B32DE9F0411C4643B1054630B11746EC
:1032D0000E4603F00FF820B1BDE8F0810E20BDE8E6
:1032E000F08123463A463146A81C03F003F8002833
:1032F000F2D123463A463146281D02F0FBFF002852
:10330000EAD123463A463146A81DBDE8F04102F015
:10331000F1BF0E20704700BF38B32DE9F0411446CD
:1033200042B11D4633B10F46064602F0F9FF20B107
:10333000BDE8F0810E20BDE8F081AB1C2246394685
:10334000304602F0EDFF0028F2D12B1D224639460F
:10335000304602F0E5FF0028EAD1AB1D224639468F
:103360003046BDE8F04102F0DBBF0E20704700BFE1
:1033700041B130B41BB110B130BC02F0E5BF0E203A
:1033800030BC70470E207047D8B1F0B5144683B0FA
:1033900042B11D4633B10E46074602F0C1FF20B1CF
:1033A00003B0F0BD0E2003B0F0BD4FF0080CAB1C15
:1033B000224631463846CDF800C003F087F903B005
:1033C000F0BD0E20704700BF002836D0F0B514467F
:1033D00083B052B14BB11F460DF107030E460546AF
:1033E00002F0C4FF20B103B0F0BD0E2003B0F0BD69
:1033F000BB1C22463146284602F092FF0028F2D13B
:103400003B1D22463146284602F08AFF0028EAD1B9
:10341000224631462846BB1D02F082FF0028E2D139
:103420009DF807203B78510862F3000361F34103E4
:10343000920862F382033B70D5E70E20704700BF0D
:10344000002962D02DE9F04F1D4683B073B168B1F9
:10345000DFF8BC8004460068CDF8008017460E46B1
:1034600003F0D6FB30B103B0BDE8F08F0E2003B0FF
:10347000BDE8F08FDFF89C906068CDF800902B4697
:103480003A46314603F0C4FB0028ECD1DFF888A0AF
:10349000A068CDF800A02B463A46314603F0B8FBB1
:1034A0000028E0D1DFF874B0E068CDF800B02B461A
:1034B0003A46314603F0ACFB0028D4D12069CDF860
:1034C00000802B463A46314603F0A2FB0028CAD1C1
:1034D0006069CDF800902B463A46314603F098FBE0
:1034E0000028C0D1A069CDF800A02B463A4631464D
:1034F00003F08EFB0028B6D1E069CDF800B02B4672
:103500003A46314603F084FBADE70E20704700BF1A
:10351000752A0200D12B0200D5280200FD280200E6
:10352000002867D02DE9F04F144683B06AB11D46DC
:103530005BB1DFF8C480CDF800800F46064603F08B
:1035400085FB30B103B0BDE8F08F0E2003B0BDE8BD
:10355000F08FDFF8A890CDF800902B1D2246394659
:10356000304603F073FB0028ECD1DFF894A0CDF8CF
:1035700000A005F1080322463946304603F066FBF9
:103580000028DFD1DFF87CB0CDF800B005F10C03E6
:1035900022463946304603F059FB0028D2D1CDF8F7
:1035A000008005F1100322463946304603F04EFBF9
:1035B0000028C7D1CDF8009005F114032246394602
:1035C000304603F043FB0028BCD1CDF800A005F144
:1035D000180322463946304603F038FB0028B1D1A3
:1035E000CDF800B005F11C0322463946304603F001
:1035F0002DFBA7E70E207047E92A02006D2B020081
:1036000099290200B929020099B130B583B06BB194
:1036100060B10078C0F3000500F00E0402A82C434E
:1036200000F8014D02F090FE03B030BD0E2003B053
:1036300030BD0E20704700BFC1B1F0B51C4683B04D
:1036400043B1054630B117460E4602F053FE20B195
:1036500003B0F0BD0E2003B0F0BD00943B463246EF
:10366000A81C052103F01AF803B0F0BD0E20704726
:10367000D8B1F0B5144683B042B11D4633B10E4601
:10368000074602F04DFE20B103B0F0BD0E2003B09E
:10369000F0BD4FF0050CAB1C224631463846CDF844
:1036A00000C003F013F803B0F0BD0E20704700BF58
:1036B00001B3F0B51D4683B043B1044630B11646A0
:1036C0000F4602F017FE20B103B0F0BD0E2003B08C
:1036D000F0BD2B4632463946A01C02F00BFE0028F6
:1036E000F2D1054B6068009332462B46394603F011
:1036F0008FFAE9E70E207047F562020000B3F0B5DB
:10370000144683B042B11D4633B10E46074602F05F
:1037100007FE20B103B0F0BD0E2003B0F0BDAB1C1E
:1037200022463146384602F0FBFD0028F2D1054B17
:10373000009322462B1D3146384603F087FAE9E70D
:103740000E2070472163020069B163B158B110B512
:1037500082B01C460068009413460A46062102F017
:1037600053FF02B010BD0E20704700BF68B130B5E6
:1037700083B03AB133B10624CDE9004402F062FFD0
:1037800003B030BD0E2003B030BD0E20704700BF27
:1037900081B110B582B053B148B1047802A8C4F326
:1037A000000400F8014D02F0CFFD02B010BD0E2064
:1037B00002B010BD0E207047A0B110B582B072B13A
:1037C0006BB11C460DF1070302F0D0FD28B9237838
:1037D0009DF8072062F30003237002B010BD0E2095
:1037E00002B010BD0E20704781B110B582B053B148
:1037F00048B1047802A8C4F3000400F8014D02F0B7
:10380000A3FD02B010BD0E2002B010BD0E20704707
:10381000A0B110B582B072B16BB11C460DF10703B7
:1038200002F0A4FD28B923789DF8072062F3000375
:10383000237002B010BD0E2002B010BD0E207047E4
:1038400040B3F0B5144683B042B11D4633B10E46C5
:10385000074602F08BFD20B103B0F0BD0E2003B08F
:10386000F0BD6B1C22463146384602F07FFD002831
:10387000F2D1AB1C22463146384602F077FD0028D3
:10388000EAD1054B009322462B1D3146384603F002
:10389000DDF9E1E70E207047D929020060B130B5AB
:1038A00083B032B12BB12024009402F00FFF03B09B
:1038B00030BD0E2003B030BD0E207047002937D038
:1038C0002DE9F0411E4684B073B368B30478054611
:1038D00004F0FE0C04A8C4F300044CEA040400F84D
:1038E000014D90460F4602F02FFD10B104B0BDE827
:1038F000F081009643463A460621681C02F0CEFE4F
:103900000028F3D1009643463A461021E81D02F004
:10391000C5FE0028EAD1009643463A4605F1170055
:10392000102102F0BBFEE1E70E2004B0BDE8F081FB
:103930000E20704700283ED02DE9F041144684B097
:103940005AB153B11D460DF10F0307460E4602F062
:103950000DFD30B104B0BDE8F0810E2004B0BDE82B
:10396000F0810623009322466B1C3146384602F054
:10397000ADFE0028EED19DF80F302A78590863F388
:1039800000022B4661F347024FF0100803F8072BA3
:103990003146CDF800802246384602F097FE0028D6
:1039A000D8D1CDF8008005F11703224631463846BC
:1039B00002F08CFECEE70E20704700BF00284AD0F0
:1039C000F0B5144685B042B11E4633B10D460746E8
:1039D00002F0CCFC20B105B0F0BD0E2005B0F0BD6A
:1039E0001E4B00932246331D2946384603F02EF91C
:1039F0000028F0D106F1080322462946384602F095
:103A0000B5FC0028E7D106F10A03224629463846CC
:103A100002F086FC0028DED106F10C03224629467E
:103A2000384602F07DFC0028D5D12246294638468A
:103A30000DF10F0302F09AFC0028CCD19DF80F2065
:103A4000B37B510862F3000361F34103920862F310
:103A50008203B373BFE70E20704700BF4529020001
:103A600041B130B41BB110B130BC02F06DBC0E20BE
:103A700030BC70470E20704740B130B41AB113B15A
:103A800030BC02F073BC0E2030BC70470E20704773
:103A9000B9B12DE9F0411C4643B1054630B1174696
:103AA0000E4602F027FC20B1BDE8F0810E20BDE8F3
:103AB000F08123463A463146A81CBDE8F04102F0A9
:103AC00019BC0E20704700BFB8B12DE9F041144673
:103AD00042B11D4633B10F46064602F021FC20B12B
:103AE000BDE8F0810E20BDE8F081AB1C22463946CE
:103AF0003046BDE8F04102F013BC0E20704700BF15
:103B000041B3F0B51D4683B043B1044630B116460B
:103B10000F4602F019FC20B103B0F0BD0E2003B037
:103B2000F0BD2B4632463946601C02F00DFC0028E1
:103B3000F2D12B4632463946A01C02F0DBFB0028AE
:103B4000EAD1054B6068009332462B46394603F0B4
:103B50005FF8E1E70E2070475928020040B3F0B546
:103B6000144683B042B11D4633B10E46074602F0FB
:103B7000FDFB20B103B0F0BD0E2003B0F0BD6B1C07
:103B800022463146384602F0F1FB0028F2D1AB1C48
:103B900022463146384602F0C3FB0028EAD1054BE5
:103BA000009322462B1D3146384603F04FF8E1E7DB
:103BB0000E2070472529020099B130B583B06BB152
:103BC00060B10078C0F3000500F07E0402A82C4329
:103BD00000F8014D02F0B8FB03B030BD0E2003B079
:103BE00030BD0E20704700BF30B310B582B002B3B5
:103BF000FBB11C460DF1070302F0B8FBB8B99DF804
:103C000007302278590863F3000261F341029908F2
:103C100061F38202D90861F3C302190961F3041246
:103C2000590961F345129B0963F38612227002B0B1
:103C300010BD0E2002B010BD0E207047B8B110B5F7
:103C400082B08AB183B11C460DF1070302F08EFBEE
:103C500040B99DF80720237862F30003520862F30D
:103C60004103237002B010BD0E2002B010BD0E2023
:103C7000704700BF40B130B41AB113B130BC02F08C
:103C80004FBB0E2030BC70470E20704738B370B564
:103C90000C4684B0E9B10678982E1AD10126039615
:103CA000D2B1CBB11E68BEB11D46134603AA06466B
:103CB00002F036FB70B90B4B009303AA2B4630463B
:103CC000214602F0C3FF28B9039B9C4218BF09207C
:103CD00000E0072004B070BD0E2004B070BD0E20BF
:103CE000704700BF7D48020013460A4601469820EF
:103CF00002F0AEBA002834D070B50C4684B051B38F
:103D00000678992E27D1012603963AB333B31E685D
:103D100026B3089E16B3366806B31D46134603AA9B
:103D2000064602F0FDFAB8B90F4B009303AA2B46E2
:103D30002146304602F08AFF70B90C4B009303AA6B
:103D40003046089B214602F081FF28B9039B9C4224
:103D500018BF092000E0072004B070BD0E2004B099
:103D600070BD0E20704700BFAD6702007D480200A5
:103D700013460A460146992002F06ABA48B370B564
:103D80000C4684B0F9B106789B2E05461BD101265E
:103D90000396DAB1D3B11E68C6B1089EB6B11E460D
:103DA000134603AA02F0BCFA70B9089B009303AA59
:103DB00033462846214602F0AFFB28B9039B9C42BC
:103DC00018BF092000E0072004B070BD0E2004B029
:103DD00070BD0E20704700BF13460A4601469B2067
:103DE00002F036BA20B3F0B50C4685B019B10678AA
:103DF000962E054602D0072005B0F0BD04AF1E4642
:103E00001346012247F8042D3A4602F089FA0028A9
:103E1000F2D1084B00933A4633462846214602F039
:103E200015FF0028E8D1039B9C4218BF0920E3E757
:103E30000E2070477D48020013460A460146962030
:103E400002F006BA20B3F0B50C4685B019B1067879
:103E5000972E054602D0072005B0F0BD04AF1E46E0
:103E60001346012247F8042D3A4602F059FA002879
:103E7000F2D1084B00933A4633462846214602F0D9
:103E8000E5FE0028E8D1039B9C4218BF0920E3E728
:103E90000E2070477D48020013460A4601469720CF
:103EA00002F0D6B910B3F0B50C4683B019B106785C
:103EB0009D2E054602D0072003B0F0BD02AF1E467E
:103EC0001346012247F8042D3A4602F029FA002849
:103ED000F2D133463A462846214602F021FA00281C
:103EE000EAD1019BA34218BF0920E5E70E207047E5
:103EF00013460A4601469D2002F0AAB960B3F0B508
:103F00000C4685B019B10678942E054602D00720DC
:103F100005B0F0BD04AF1E461346012247F8042D3C
:103F20003A4602F0FDF90028F2D133463A462146DE
:103F3000284602F0F5F90028EAD1084B00933A46EA
:103F400028460A9B214602F081FE0028E0D1039B0F
:103F50009C4218BF0920DBE70E207047AD670200C6
:103F600013460A460146942002F072B950B3F0B5E8
:103F70000C4683B019B106789A2E054602D0072068
:103F800003B0F0BD02AF1E461346012247F8042DD0
:103F90003A4602F0C5F90028F2D133463A462146A6
:103FA000284602F0BDF90028EAD13A462846089B87
:103FB000214602F0B5F90028E2D1019B9C4218BFCE
:103FC0000920DDE70E20704713460A4601469A2075
:103FD00002F03EB920B3F0B50C4685B019B10678B1
:103FE000952E054602D0072005B0F0BD04AF1E4651
:103FF0001346012247F8042D3A4602F091F90028B1
:10400000F2D1084B00933A4633462846214602F047
:104010001DFE0028E8D1039B9C4218BF0920E3E75E
:104020000E2070477D48020013460A46014695203F
:1040300002F00EB920B3F0B50C4685B019B1067880
:104040009C2E054602D0072005B0F0BD04AF1E46E9
:104050001346012247F8042D3A4602F061F9002880
:10406000F2D1084B00933A4633462846214602F0E7
:10407000EDFD0028E8D1039B9C4218BF0920E3E72F
:104080000E2070473549020013460A4601469C201F
:1040900002F0DEB810B3F0B50C4683B019B1067863
:1040A0009E2E054602D0072003B0F0BD02AF1E468B
:1040B0001346012247F8042D3A4602F031F9002850
:1040C000F2D133463A462846214602F029F9002823
:1040D000EAD1019B9C4218BF0920E5E70E207047FA
:1040E00013460A4601469E2002F0B2B8E0B1DAB1AA
:1040F000D3B10188342901D007207047F0B583B0CF
:104100001F68ADF80210154604461E464FF0000C1D
:104110003A4601AB29460DF10200CDF804C002F089
:10412000E9F818B103B0F0BD0E20704701AB3A4674
:104130002946201D02F0DEF80028F3D101AB3A46F3
:104140002946A01D02F0D6F80028EBD101AB3A4673
:10415000294604F1080002F0CDF80028E2D101ABB5
:104160003A46294604F10A0000F01AFC0028D9D189
:10417000019B3360D6E700BFE0B1DAB1D3B101886B
:10418000322901D007207047F0B583B01F68ADF821
:104190000210154604461E464FF0000C3A4601AB8D
:1041A00029460DF10200CDF804C002F0A3F818B1C1
:1041B00003B0F0BD0E20704701AB3A462946201DE2
:1041C00002F098F80028F3D101AB3A462946A01D29
:1041D00002F090F80028EBD101AB3A46294604F1F1
:1041E000080002F087F80028E2D101AB3A462946E0
:1041F00004F10A0000F018FC0028D9D1019B3360BB
:10420000D6E700BFE0B1DAB1D3B10188352901D0DA
:1042100007207047F0B583B01F68ADF8021015464F
:1042200004461E464FF0000C3A4601AB29460DF1FC
:104230000200CDF804C002F05DF818B103B0F0BD83
:104240000E20704701AB3A462946201D02F052F875
:104250000028F3D101AB3A462946A01D02F04AF8E6
:104260000028EBD101AB3A46294604F1080002F0E0
:1042700041F80028E2D101AB3A46294604F10A0090
:1042800000F0B4FA0028D9D1019B3360D6E700BF13
:10429000E0B1DAB1D3B10188372901D007207047E6
:1042A000F0B583B01F68ADF80210154604461E46EF
:1042B0004FF0000C3A4601AB29460DF10200CDF853
:1042C00004C002F017F818B103B0F0BD0E2070471B
:1042D00001AB3A462946201D02F00CF80028F3D124
:1042E00001AB3A462946A01D02F004F80028EBD1A4
:1042F00001AB3A46294604F1080001F0FBFF002813
:10430000E2D101AB3A46294604F10A0000F098FADE
:104310000028D9D1019B3360D6E700BFE0B1DAB104
:10432000D3B10188332901D007207047F0B583B09D
:104330001F68ADF80210154604461E464FF0000CEB
:104340003A4601AB29460DF10200CDF804C001F058
:10435000D1FF18B103B0F0BD0E20704701AB3A4653
:104360002946201D01F0C6FF0028F3D101AB3A46D3
:104370002946A01D01F0BEFF0028EBD101AB3A4653
:10438000294604F1080001F0B5FF0028E2D101AB95
:104390003A46294604F10A0000F0A6FB0028D9D1CC
:1043A000019B3360D6E700BFE0B1DAB1D3B1018839
:1043B000392901D007207047F0B583B01F68ADF8E8
:1043C0000210154604461E464FF0000C3A4601AB5B
:1043D00029460DF10200CDF804C001F08BFF18B1A1
:1043E00003B0F0BD0E20704701AB3A462946201DB0
:1043F00001F080FF0028F3D101AB3A462946A01D09
:1044000001F078FF0028EBD101AB3A46294604F1D0
:10441000080001F06FFF0028E2D101AB3A462946BF
:1044200004F10A0000F092FB0028D9D1019B33600F
:10443000D6E700BFE0B1DAB1D3B10188302901D0AD
:1044400007207047F0B583B01F68ADF8021015461D
:1044500004461E464FF0000C3A4601AB29460DF1CA
:104460000200CDF804C001F045FF18B103B0F0BD63
:104470000E20704701AB3A462946201D01F03AFF55
:104480000028F3D101AB3A462946A01D01F032FFC6
:104490000028EBD101AB3A46294604F1080001F0AF
:1044A00029FF0028E2D101AB3A46294604F10A006F
:1044B00000F078FB0028D9D1019B3360D6E700BF1C
:1044C000E0B1DAB1D3B10188362901D007207047B5
:1044D000F0B583B01F68ADF80210154604461E46BD
:1044E0004FF0000C3A4601AB29460DF10200CDF821
:1044F00004C001F0FFFE18B103B0F0BD0E207047FC
:1045000001AB3A462946201D01F0F4FE0028F3D104
:1045100001AB3A462946A01D01F0ECFE0028EBD184
:1045200001AB3A46294604F1080001F0E3FE0028F9
:10453000E2D101AB3A46294604F10A0000F06EFBD5
:104540000028D9D1019B3360D6E700BFE0B1DAB1D2
:10455000D3B10188312901D007207047F0B583B06D
:104560001F68ADF80210154604461E464FF0000CB9
:104570003A4601AB29460DF10200CDF804C001F026
:10458000B9FE18B103B0F0BD0E20704701AB3A463A
:104590002946201D01F0AEFE0028F3D101AB3A46BA
:1045A0002946A01D01F0A6FE0028EBD101AB3A463A
:1045B000294604F1080001F09DFE0028E2D101AB7C
:1045C0003A46294604F10A0000F074F90028D9D1CE
:1045D000019B3360D6E700BFE0B1DAB1D3B1018807
:1045E0003B2901D007207047F0B583B01F68ADF8B4
:1045F0000210154604461E464FF0000C3A4601AB29
:1046000029460DF10200CDF804C001F073FE18B187
:1046100003B0F0BD0E20704701AB3A462946201D7D
:1046200001F068FE0028F3D101AB3A462946A01DEF
:1046300001F060FE0028EBD101AB3A46294604F1B7
:10464000080001F057FE0028E2D101AB3A462946A6
:1046500004F10A0000F00EFB0028D9D1019B336061
:10466000D6E700BFE0B1DAB1D3B10188382901D073
:1046700007207047F0B583B01F68ADF802101546EB
:1046800004461E464FF0000C3A4601AB29460DF198
:104690000200CDF804C001F02DFE18B103B0F0BD4A
:1046A0000E20704701AB3A462946201D01F022FE3C
:1046B0000028F3D101AB3A462946A01D01F01AFEAD
:1046C0000028EBD101AB3A46294604F1080001F07D
:1046D00011FE0028E2D101AB3A46294604F10A0056
:1046E00000F0D4FA0028D9D1019B3360D6E700BF8F
:1046F000E0B1DAB1D3B101883A2901D0072070477F
:10470000F0B583B01F68ADF80210154604461E468A
:104710004FF0000C3A4601AB29460DF10200CDF8EE
:1047200004C001F0E7FD18B103B0F0BD0E207047E2
:1047300001AB3A462946201D01F0DCFD0028F3D1EB
:1047400001AB3A462946A01D01F0D4FD0028EBD16B
:1047500001AB3A46294604F1080001F0CBFD0028E0
:10476000E2D101AB3A46294604F10A0000F0C2FA50
:104770000028D9D1019B3360D6E700BFB9B12DE93C
:10478000F0411C4643B1054630B117460E4601F0D4
:10479000B1FD20B1BDE8F0810E20BDE8F0812346D7
:1047A0003A463146A81CBDE8F04101F0E3BF0E20B7
:1047B000704700BFB9B12DE9F0411C4643B1054631
:1047C00030B117460E4601F095FD20B1BDE8F081ED
:1047D0000E20BDE8F08123463A463146A81CBDE8CC
:1047E000F04101F0FFBF0E20704700BF29B3F0B5C4
:1047F0001D4683B043B1044630B116460F4601F062
:1048000079FD20B103B0F0BD0E2003B0F0BD2B4602
:1048100032463946A01C01F06DFD0028F2D1204639
:10482000638830F8041B0095023311FB03F13A460C
:10483000334689B201F032FFE4E70E20704700BF33
:10484000C9B1F0B51D4683B043B1044630B1174637
:104850000E4601F04FFD20B103B0F0BD0E2003B0B5
:10486000F0BD2046009530F8021B3B46324601F071
:1048700015FF03B0F0BD0E20704700BFB8B12DE9A1
:10488000F041144642B11D4633B10F46064601F0D1
:1048900047FD20B1BDE8F0810E20BDE8F081AB1CE2
:1048A000224639463046BDE8F04101F039BD0E20C0
:1048B000704700BF00293BD02DE9F8431E4693B353
:1048C000074680B39046894601F014FD88B93B88BD
:1048D000BC1C054653B3334642464946204601F0C8
:1048E00009FD30B9334642464946A01C01F042FF5B
:1048F00008B1BDE8F883334642464946A01D01F0A1
:10490000F9FC0028F5D104F1080033464246494637
:1049100001F0F0FC01350A340028EAD13B88AB42B3
:1049200004D9002CD7D10E20BDE8F8830020E0E7A1
:104930000E20704788B3F0B5144683B042B11D46CF
:1049400033B10E46074601F011FD20B103B0F0BDB2
:104950000E2003B0F0BD6B1C22463146384601F0F4
:1049600005FD0028F2D1AB1C22463146384601F045
:10497000D7FC0028EAD12B1D22463146384601F0EB
:10498000CFFC0028E2D1AB1D0093224631463846C9
:1049900005F1080301F088FDD8E70E20704700BF3D
:1049A0002DE9F84F61B11D4653B1044640B1904620
:1049B000894601F09FFC074630B13846BDE8F88FC4
:1049C0000E273846BDE8F88F2B4642464946A01CC4
:1049D00001F0BAFC07460028EFD1A378104811492E
:1049E0002288012B0CBF82468A46002AE5D03E462B
:1049F00004F1040B03E02388B342DED9A378012B32
:104A00000CBF06EB460006EBC6000BEB40002B4646
:104A100042464946D04701360028ECD00746CCE74D
:104A20007D470200B547020000295BD02DE9F04F19
:104A30001C4683B003B30546F0B116460F4601F09D
:104A400059FCB0B92B88002B48D0804605F10209EB
:104A500005F1080B234632463946484601F08AFEE6
:104A600038B923463246394609F10400FFF7A4F865
:104A700030B103B0BDE8F08F0E2003B0BDE8F08F79
:104A800008EB880A4FEA4A0A05EB0A02234692F825
:104A900007C03946CCF3000C32460DF107008DF803
:104AA00007C001F051FC0028E3D10BEB0A002346BC
:104AB0003246394601F01EFC0028DAD109F108001F
:104AC00023463246394601F015FC09F10A0908F17E
:104AD00001080028CDD12B884345BBD8002003B066
:104AE000BDE8F08F0E20704759B32DE9F8431C46FE
:104AF00023B3054610B31746884601F0FBFBD8B92F
:104B00002B8803B3064605F102090DE009F1020006
:104B100023463A46414601F02DFE013609F10609C9
:104B200050B92B88B3420ED923463A4641464846EF
:104B300001F0E0FB0028E9D0BDE8F8830E20BDE8D5
:104B4000F8830E2070470020BDE8F88339B3F0B534
:104B50001C4683B043B1054630B116460F4601F0FE
:104B6000C9FB20B103B0F0BD0E2003B0F0BD234659
:104B700032463946A81C01F0E7FB0028F2D1234653
:104B800032463946281D01F0B5FB0028EAD1A98834
:104B9000009433463A46A81D01F080FDE2E70E205E
:104BA000704700BFC1B32DE9F84F1E468BB30546D1
:104BB00078B39046894601F09DFBB8B92B882BB39A
:104BC000044605F1020A05F1060BE7000AEB0700AF
:104BD00033464246494601F0CDFD38B93346424698
:104BE00049460BEB070001F085FB08B1BDE8F88FE3
:104BF00007F10800284433464246494601F07AFB53
:104C000001340028F2D12B88A342DED80020BDE871
:104C1000F88F0E20BDE8F88F0E20704739B3F0B53D
:104C20001C4683B043B1054630B116460F4601F02D
:104C300061FB20B103B0F0BD0E2003B0F0BD2346F0
:104C400032463946A81C01F055FB0028F2D1234614
:104C500032463946281D01F04DFB0028EAD1A988CB
:104C6000009433463A46A81D01F018FDE2E70E20F5
:104C7000704700BF41B130B41BB110B130BC01F07E
:104C800063BB0E2030BC70470E20704781B3F0B577
:104C90001C4683B043B1054630B116460F4601F0BD
:104CA00029FB20B103B0F0BD0E2003B0F0BD2346B8
:104CB00032463946A81C01F047FB0028F2D12346B2
:104CC00032463946281D01F015FB0028EAD123465B
:104CD00032463946A81D01F00DFB0028E2D1E988D3
:104CE000009433463A4605F1080001F0D7FCD9E7B5
:104CF0000E20704741B130B41BB110B130BC01F08F
:104D0000F9BA0E2030BC70470E20704760B3F0B582
:104D10000C4685B019B10678AC2E054602D00720A6
:104D200005B0F0BD04AF1E461346012247F8042D1E
:104D30003A4601F0F5FA0028F2D1009033463A469F
:104D40002146284601F082FF0028E9D100903A462A
:104D500028460A9B214601F079FF0028E0D1039BF9
:104D6000A34218BF0920DBE70E207047F0B587B0DB
:104D7000039001B3FAB1176800201D4614464FF0A6
:104D8000AC0C05903A4605AB0DF113000E468DF8BC
:104D900013C001F0D9FA08B107B0F0BD05AB3A462F
:104DA000314603A801F06CFA0028F5D1039B2BB122
:104DB000059B2360F0E70E2007B0F0BD0A4B00937F
:104DC000284605AB3A46314601F022FF0028E3D1E0
:104DD000064B00933A4605AB31460C9801F018FF9C
:104DE0000028E5D0D8E700BF75670200B95A020075
:104DF000002837D0F0B50C4685B019B10678A22E40
:104E0000054602D0072005B0F0BD04AF1E4613468C
:104E1000012247F8042D3A4601F082FA0028F2D127
:104E2000114B00933A4633462146284601F00EFFC7
:104E30000028E8D10D4B00933A460A9B21462846AC
:104E400001F004FF0028DED100903A4628460B9B73
:104E5000214601F0FBFE0028D5D1039BA34218BFD9
:104E60000920D0E70E207047ED5B0200B55C020020
:104E7000F0B587B0039001B3FAB1176800201D4662
:104E800014464FF0A20C05903A4605AB0DF1130005
:104E90000E468DF813C001F057FA08B107B0F0BD07
:104EA00005AB3A46314603A801F0EAF90028F5D1EE
:104EB000039B2BB1059B2360F0E70E2007B0F0BDEC
:104EC000054B00933A4605AB3146284601F0A0FE5B
:104ED0000028EFD0E2E700BF3D5D020068B3F0B507
:104EE0000C4685B019B10678A32E054602D00720DE
:104EF00005B0F0BD04AF1E461346012247F8042D4D
:104F00003A4601F00DFA0028F2D10D4B00933A46D3
:104F100033462146284601F099FE0028E8D100904A
:104F20003A4628460A9B214601F090FE0028DFD130
:104F3000039BA34218BF0920DAE70E20704700BF89
:104F4000B55C0200F0B587B0039001B3FAB1176801
:104F500000201D4614464FF0A30C05903A4605ABC1
:104F60000DF113000E468DF813C001F0EDF908B1F4
:104F700007B0F0BD05AB3A46314603A801F080F911
:104F80000028F5D1039B2BB1059B2360F0E70E2091
:104F900007B0F0BD054B00933A4605AB31462846B5
:104FA00001F036FE0028EFD0E2E700BFF562020014
:104FB00020B3F0B50C4685B019B10678A62E05468B
:104FC00002D0072005B0F0BD04AF1E4613460122F3
:104FD00047F8042D3A4601F0A3F90028F2D1084B16
:104FE00000933A4633462846214601F02FFE00281A
:104FF000E8D1039BA34218BF0920E3E70E207047C6
:10500000955D0200F0B587B0039001B3FAB117685F
:1050100000201D4614464FF0A60C05903A4605ABFD
:105020000DF113000E468DF813C001F08DF908B193
:1050300007B0F0BD05AB3A46314603A801F020F9B0
:105040000028F5D1039B2BB1059B2360F0E70E20D0
:1050500007B0F0BD054B00933A4605AB31462846F4
:1050600001F0D6FD0028EFD0E2E700BFF5620200B4
:1050700058B3F0B50C4685B019B10678A12E054697
:1050800002D0072005B0F0BD04AF1E461346012232
:1050900047F8042D3A4601F043F90028F2D133468F
:1050A0003A462146284601F03BF90028EAD1009013
:1050B0003A4628460A9B214601F0C8FD0028E1D166
:1050C000039B9C4218BF0920DCE70E20704700BFFD
:1050D000F0B587B0039001B3FAB1176800201D4600
:1050E00014464FF0A10C05903A4605AB0DF11300A4
:1050F0000E468DF813C001F027F908B107B0F0BDD6
:1051000005AB3A46314603A801F0BAF80028F5D1BC
:10511000039B2BB1059B2360F0E70E2007B0F0BD89
:10512000054B00933A4605AB3146284601F070FD29
:105130000028EFD0E2E700BFF5620200D8B170B5F9
:105140000C4684B021B10378AB2B4FF0000502D0A0
:10515000072004B070BD134604AA012642F8046D6E
:10516000009501F073FD0028F3D1039BA34218BF03
:10517000092004B070BD0E20704700BFF0B587B0A5
:10518000039001B3FAB1176800201D4614464FF092
:10519000AB0C05903A4605AB0DF113000E468DF8A9
:1051A00013C001F0D1F808B107B0F0BD05AB3A4625
:1051B000314603A801F064F80028F5D1039B2BB118
:1051C000059B2360F0E70E2007B0F0BD054B009370
:1051D0003A4605AB3146284601F01AFD0028EFD0CB
:1051E000E2E700BFF562020020B3F0B50C4685B0DF
:1051F00019B10678A82E054602D0072005B0F0BDEB
:1052000004AF1E461346012247F8042D3A4601F02A
:1052100087F80028F2D1084B00933A4633462846D7
:10522000214601F013FD0028E8D1039BA34218BFDB
:105230000920E3E70E2070471D5F020013460A466F
:105240000146A82001F004B868B3F0B50C4685B05B
:1052500019B10678A02E054602D0072005B0F0BD92
:1052600004AF1E461346012247F8042D3A4601F0CA
:105270007DF80028F2D10D4B00933A463346214683
:10528000284601F0E3FC0028E8D100903A46284681
:105290000A9B214601F0DAFC0028DFD1039BA342E0
:1052A00018BF0920DAE70E20704700BFAD67020083
:1052B000F0B587B0039001B3FAB1176800201D461E
:1052C00014464FF0A00C05903A4605AB0DF11300C3
:1052D0000E468DF813C001F037F808B107B0F0BDE5
:1052E00005AB3A46314603A800F0CAFF0028F5D1C5
:1052F000039B2BB1059B2360F0E70E2007B0F0BDA8
:10530000054B00933A4605AB3146284601F080FC38
:105310000028EFD0E2E700BFF562020050B3F0B51D
:105320000C4683B019B10678A72E054602D0072097
:1053300003B0F0BD02AF1E461346012247F8042D0C
:105340003A4600F0EDFF0028F2D133463A462146B6
:10535000284600F0E5FF0028EAD13A462846089B97
:10536000214600F0DDFF0028E2D1019BA34218BFD7
:105370000920DDE70E20704713460A460146A720A4
:1053800000F066BF002835D0F0B50C4685B019B1E5
:105390000678AA2E054602D0072005B0F0BD04AF5E
:1053A0001E461346012247F8042D3A4600F0B8FF86
:1053B0000028F2D1104B00933A460A9B214628461A
:1053C00001F044FC0028E8D1009033463A462146DB
:1053D000284601F03BFC0028DFD13A4628460B9BCB
:1053E000214600F06FFF0028D7D1039BA34218BFCE
:1053F0000920D2E70E207047216302002DE9F04119
:1054000086B0039021B31AB3D2F800800020AA24FA
:1054100005901E46154605AB42460DF113008DF86A
:1054200013400F4600F090FF044618B1204606B026
:10543000BDE8F08105AB4246394603A800F020FFE5
:1054400004460028F2D1039B3BB1059B2B60EDE79E
:105450000E24204606B0BDE8F0810D4B0093424675
:1054600005AB39460C9801F0D3FB04460028DDD18A
:105470000C9B002BE9D0198805AB00933A464346B4
:10548000304601F0C1F80028DFD00446CEE700BF67
:10549000F562020060B3F0B50C4685B019B106782C
:1054A000A92E054602D0072005B0F0BD04AF1E4668
:1054B0001346012247F8042D3A4600F031FF002838
:1054C000F2D10A9B00933A4633462146284600F023
:1054D000EBFF0028E8D13A4628460B9B214600F016
:1054E000F1FE0028E0D1039BA34218BF0920DBE7AF
:1054F0000E20704713460A460146A92000F0A8BEB8
:105500002DE9F04184B0002836D011B10678A52EDF
:1055100004D00724204604B0BDE8F0810DF1100846
:105520001F461346012248F8042D424606460D4602
:1055300000F0F6FE04460028ECD13B4642462946E0
:10554000304600F0EDFE04460028E3D100900A9BAF
:1055500042462946304601F079FB04460028D9D15D
:105560000A9B1B680BB3023342462946304600F0C3
:10557000D7FE30B10446CDE70E24204604B0BDE886
:10558000F0810A9B42461B682946304600F0C8FE5F
:105590000028EFD10A9B1B68009442463046043332
:1055A000294601F053FB0028E4D1039B9D4218BF1C
:1055B0000924AFE7F0B587B0039001B3FAB11768DB
:1055C00000201D4614464FF0A50C05903A4605AB49
:1055D0000DF113000E468DF813C000F0B5FE08B1B2
:1055E00007B0F0BD05AB3A46314603A800F048FECF
:1055F0000028F5D1039B2BB1059B2360F0E70E201B
:1056000007B0F0BD054B00933A4605AB314628463E
:1056100001F0FEFA0028EFD0E2E700BF01600200CF
:1056200060B3F0B50C4685B019B10678A42E0546D6
:1056300002D0072005B0F0BD04AF1E46134601227C
:1056400047F8042D3A4600F06BFE0028F2D13346AD
:105650003A462146284600F063FE0028EAD1084B6E
:1056600000933A4628460A9B214601F0EFFA0028AB
:10567000E0D1039B9C4218BF0920DBE70E20704756
:105680003D600200F0B587B0039001B3FAB117682E
:1056900000201D4614464FF0A40C05903A4605AB79
:1056A0000DF113000E468DF813C000F04DFE08B149
:1056B00007B0F0BD05AB3A46314603A800F0E0FD67
:1056C0000028F5D1039B2BB1059B2360F0E70E204A
:1056D00007B0F0BD054B00933A4605AB314628466E
:1056E00001F096FA0028EFD0E2E700BF0160020067
:1056F00010B3F0B50C4683B019B10678AD2E05464F
:1057000002D0072003B0F0BD02AF1E4613460122AF
:1057100047F8042D3A4600F003FE0028F2D1334644
:105720003A462846214600F0FBFD0028EAD1019BBD
:105730009C4218BF0920E5E70E20704713460A4631
:105740000146AD2000F084BD2DE9F04186B000286F
:1057500036D0002A34D0002B32D00188512904D011
:105760000725284606B0BDE8F081D3F80080ADF8E3
:105770000E101646002504461F46424604AB31462D
:105780000DF10E00049500F0B5FD05460028E8D1A6
:1057900004AB42463146201D00F0ACFD0546002812
:1057A000DFD1424604AB3146A01D00F07BFB05462D
:1057B0000028D6D1A379022B07D0049B3B60D0E709
:1057C0000E25284606B0BDE8F081A37B03F0FD035B
:1057D000042BF2D1A08805A901F028FB0528ECD004
:1057E000084A05983B6804A900914C2101FB002060
:1057F00032460189406800F02FFE0028DDD00546C2
:10580000AFE700BF94800020E0B1DAB1D3B10188E6
:10581000532901D007207047F0B583B01F68ADF859
:105820000210154604461E464FF0000C3A4601ABE6
:1058300029460DF10200CDF804C000F05BFD18B15F
:1058400003B0F0BD0E20704701AB3A462946201D3B
:1058500000F050FD0028F3D101AB3A462946A01DC7
:1058600000F016FC0028EBD1019B3360E8E700BF95
:10587000E0B1DAB1D3B10188532901D007207047D4
:10588000F0B583B01F68ADF80210154604461E46F9
:105890004FF0000C3A4601AB29460DF10200CDF85D
:1058A00004C000F027FD18B103B0F0BD0E20704712
:1058B00001AB3A462946201D00F01CFD0028F3D11B
:1058C000019B3360F0E700BFE0B1DAB1D3B10188EA
:1058D000522901D007207047F0B583B01F68ADF89A
:1058E0000210154604461E464FF0000C3A4601AB26
:1058F00029460DF10200CDF804C000F0FBFC18B100
:1059000003B0F0BD0E20704701AB3A462946201D7A
:1059100000F0F0FC0028F3D101AB3A462946A01D67
:1059200000F0C2FB0028EBD1019B3360E8E700BF29
:10593000E0B1DAB1D3B10188562901D00720704710
:10594000F0B583B01F68ADF80210154604461E4638
:105950004FF0000C3A4601AB29460DF10200CDF89C
:1059600004C000F0C7FC18B103B0F0BD0E207047B2
:1059700001AB3A462946201D00F0BCFC0028F3D1BB
:1059800001AB3A462946A01D00F09AFB0028EBD156
:10599000019B3360E8E700BF2DE9F04186B00028A5
:1059A00038D0002A36D0002B34D00188502904D0BA
:1059B0000725284606B0BDE8F081D3F80080ADF891
:1059C0000E101646002504461F46424604AB3146DB
:1059D0000DF10E00049500F08DFC05460028E8D17D
:1059E00004AB42463146201D00F084FC05460028E9
:1059F000DFD104AB42463146A01D00F00BFA05464C
:105A00000028D6D1237B012B09D0062B07D0049B7D
:105A10003B60CEE70E25284606B0BDE8F081A088A1
:105A200005A901F003FA0528F1D0084B059A04A94D
:105A300000914C2101FB02324346118950683246E5
:105A400000F00AFD0028E2D00546B2E7948000206D
:105A5000E0B1DAB1D3B10188552901D007207047F0
:105A6000F0B583B01F68ADF80210154604461E4617
:105A70004FF0000C3A4601AB29460DF10200CDF87B
:105A800004C000F037FC18B103B0F0BD0E20704721
:105A900001AB3A462946201D00F02CFC0028F3D12A
:105AA00001AB3A462946A01D00F0E6FA0028EBD1EA
:105AB000019B3360E8E700BF71B3F0B51C4683B0CB
:105AC00043B1054630B116460F46FDF7B5F920B192
:105AD00003B0F0BD0E2003B0F0BD23463246394678
:105AE000681CFDF7A9F90028F2D1AB7802A8C3F32E
:105AF000000203F01E03134300F8013D3246234623
:105B0000394600F021FC0028E2D1AB7803F006030F
:105B1000022B18BF0720DBE70E20704780B3F0B5DB
:105B2000144683B042B11F4633B10E460546FDF719
:105B30009BF920B103B0F0BD0E2003B0F0BD7B1C7B
:105B4000224631462846FDF78FF90028F2D1224639
:105B5000314628460DF1070300F008FC0028E9D182
:105B60009DF80720BB78510862F3000361F34203FC
:105B7000D10861F3C303120962F30413BB70D9E7C0
:105B80000E20704778B32DE9F041144642B11D460E
:105B900033B10F46064600F0E9FB20B1BDE8F081C5
:105BA0000E20BDE8F0816B1C22463946304600F0DD
:105BB000DDFB0028F2D1AB1C22463946304600F00E
:105BC000AFFB0028EAD12B1D22463946304600F0B3
:105BD000CDFB0028E2D1AB1D224639463046BDE858
:105BE000F04100F09DBB0E20704700BF00285BD045
:105BF0002DE9F041144682B04AB11E463BB10D4634
:105C00000746FDF7F1FF30B102B0BDE8F0810E208C
:105C100002B0BDE8F081731C224629463846FEF7E3
:105C20000DF80028F0D106F108032246294638462F
:105C300000F076FB0028E7D106F10A030093224624
:105C4000331D2946384600F02FFC0028DCD1174BC5
:105C50000093224606F10C032946384600F0F6FF71
:105C60000028D1D1DFF84880CDF8008006F110037C
:105C700022462946384600F0E9FF0028C4D1CDF875
:105C8000008006F1140322462946384600F0DEFF64
:105C90000028B9D1CDF8008006F118032246294624
:105CA000384600F0D3FFAFE70E207047855B020057
:105CB0001D5B020000283AD0F0B5144683B062B1F3
:105CC0001E4653B1DFF870C0CDF800C00D46074640
:105CD00000F0BCFF20B103B0F0BD0E2003B0F0BD5A
:105CE000144B00932246331D2946384600F0AEFF80
:105CF0000028F0D106F10A0322462946384600F072
:105D00000FFB0028E7D106F10C032246294638464E
:105D100000F006FB0028DED106F1080300932246BE
:105D20002946384606F1100300F0BEFBD3E70E20EB
:105D3000704700BF1D5B0200AD67020039B32DE95B
:105D4000F0411C4643B1054630B117460E4600F0FF
:105D5000D1FA20B1BDE8F0810E20BDE8F0812346E4
:105D60003A463146A81C00F0C5FA0028F2D1234675
:105D70003A463146281D00F0BDFA0028EAD12346F4
:105D80003A463146A81DBDE8F04100F0B3BA0E20F6
:105D9000704700BF002838D0F0B5144683B042B138
:105DA0001E4633B10D46074600F0BAFA20B103B0E3
:105DB000F0BD0E2003B0F0BDB31C22462946384684
:105DC00000F0D4FA0028F2D1331D22462946384685
:105DD00000F0A6FA0028EAD10D4B0093224606F106
:105DE00008032946384600F031FF0028DFD1B368A8
:105DF000002BDCD01B882246CDE90033294606F172
:105E00000C03384600F01EFCD1E70E20704700BF9F
:105E100021630200002942D0F0B51C4683B043B193
:105E2000054630B116460F4600F064FA20B103B0C3
:105E3000F0BD0E2003B0F0BD234632463946A81C03
:105E400000F098FC0028F2D1234632463946A81DBE
:105E500000F07AFA0028EAD1234632463946E81D96
:105E600000F072FA0028E2D123463246394605F1A5
:105E7000080000F03FFA0028D9D1234632463946BF
:105E800005F10A0000F036FA0028D0D169890094A3
:105E900033463A4605F10C0000F000FCC7E70E203F
:105EA000704700BFC1B32DE9F0411D46B3B10446B0
:105EB000A0B116460F4600F047FA68B92378012BC7
:105EC0000FD0022B07D12B4632463946A01CBDE825
:105ED000F041FFF79FBF0720BDE8F0810E20BDE82D
:105EE000F08104F1020840462B463246394600F064
:105EF00001FA0028F0D1201D2B463246394600F029
:105F000039FC0028E8D12B463246394604F1080016
:105F1000BDE8F04100F0EEB90E207047002847D0F0
:105F20002DE9F041144684B07AB11D466BB10E469E
:105F3000074600F01BFA28B92B78012B09D0022B59
:105F400007D0072004B0BDE8F0810E2004B0BDE802
:105F5000F08105F10408434622463146384600F0F8
:105F6000DFF90028EED10DF10F0322463146384605
:105F700000F0FCF90028E5D105F10803224631467E
:105F8000384600F0CDF90028DCD105F10A03009372
:105F900022463146384605F10C0300F085FA002808
:105FA000D0D1AB799DF80F2062F30003AB71C9E744
:105FB0000E20704708B3F0B583B05AB153B11C46F8
:105FC0000DF107030F460646154600F0CFF920B144
:105FD00003B0F0BD0E2003B0F0BD2A46394630466E
:105FE000231D00F06FF90028F2D123789DF80720D7
:105FF00062F30003237003B0F0BD0E20704700BFB2
:10600000C9B1F0B583B053B148B104460230164669
:106010000F461D4600F06EF920B103B0F0BD0E2012
:1060200003B0F0BD21886068009533463A4600F021
:1060300013FA03B0F0BD0E20704700BFC8B1F0B531
:1060400083B052B14BB11C4602330F46064615468B
:1060500000F066F920B103B0F0BD0E2003B0F0BD32
:106060000094231D2A463946304600F01DFA03B03D
:10607000F0BD0E20704700BF41B130B41BB110B16C
:1060800030BC00F037B90E2030BC70470E2070478E
:1060900041B130B41BB110B130BC00F02BB90E20AF
:1060A00030BC70470E20704741B130B41BB110B105
:1060B00030BC00F049B90E2030BC70470E2070474C
:1060C00041B130B41BB110B130BC00F03DB90E206D
:1060D00030BC70470E207047CAB1C0B110B503295B
:1060E00082B011D10378B02B02D0072002B010BDCE
:1060F000134602AA012442F8044D00F011F90028C9
:10610000F4D1019B032BF1D0092002B010BD0E2069
:10611000704700BF13460A460146B02000F098B809
:10612000CAB1C0B110B5032982B011D10378B12B27
:1061300002D0072002B010BD134602AA012442F883
:10614000044D00F0EDF80028F4D1019B032BF1D0B1
:10615000092002B010BD0E20704700BF13460A464A
:106160000146B12000F074B8C0B1BAB1B3B1F0B516
:106170001E6885B07EB10A9C6CB104AE1C46134605
:10618000012246F8042D32460F46054600F0C8F8B5
:1061900030B105B0F0BD0E2005B0F0BD0E20704747
:1061A0000D4B0093324623463946284600F04EFDFB
:1061B0000028EED1039B226801334AB10A9A1D449C
:1061C00015602268128813449F4218BF0920E0E737
:1061D0000A9A1060F8E700BF2D68020013460A46CD
:1061E0000146B22000F034B8E0B1DAB1D3B1018891
:1061F000702901D007207047F0B583B01F68ADF853
:106200000210154604461E464FF0000C3A4601ABFC
:1062100029460DF10200CDF804C000F06BF818B16A
:1062200003B0F0BD0E20704701AB3A462946201D51
:1062300000F060F80028F3D101AB3A462946A01DD2
:1062400000F010FB0028EBD1019B3360E8E700BFB2
:10625000A2B19BB130B41C68042C0CD90D0A0C0CF3
:1062600010705170080E05219570D470107130BCFB
:10627000002019607047092030BC70470E2070471D
:10628000D1B1C8B1C3B130B41C68121B032A15D9EF
:1062900002680020150A62F3070065F30F20150C51
:1062A00065F31740120E62F31F6008511A6804323A
:1062B00000201A6030BC70470E207047092030BCA7
:1062C000704700BF78B172B16BB110B41468091B8C
:1062D00003290AD90159196013685DF8044B043386
:1062E0000020136070470E20704709205DF8044BB2
:1062F000704700BF10B41C68121B012A0BD902881A
:106300000A552144120A4A701A685DF8044B023299
:1063100000201A60704709205DF8044B704700BFE9
:1063200030B41468091B01290BD90519015D68787F
:1063300041EA00211980136802330020136030BC49
:106340007047092030BC704710B41C68944208D0D4
:1063500002780A551A685DF8044B013200201A6071
:10636000704709205DF8044B704700BF10B41468F3
:106370008C4208D0015D197013685DF8044B01333D
:1063800000201360704709205DF8044B704700BF80
:1063900030B41468651C8D4204D8015D197013680F
:1063A0000133136030BC704770B5049C2568AB4264
:1063B0001CD051552568061C05F1010518BF0126A2
:1063C000AB42256012D0565526680136266060B172
:1063D0009B1B99420AD80D46014690192A4605F0A2
:1063E0000AFE216829442160002070BD092070BD8B
:1063F000F8B51468069DA14295F800C025D0045D4B
:106400002C701468661C1660B1422F781DD0A51C34
:10641000A94203D2DBB100201860F8BD845D15608D
:10642000012CF7D1ABB11B689BB1BC450DD3491B07
:106430008F420AD8144641193A46184605F0DBFD4A
:1064400023681F4427600020F8BD0920F8BD1846C6
:10645000F8BD0E20F8BD00BF70B5049C25685E1B1A
:10646000012E1FD9561951550D0A75702568061C45
:1064700005F1020518BF0126AB42256012D0565522
:1064800026680136266060B19B1B99420AD80D46EA
:10649000014690192A4605F0AEFD21682944216085
:1064A000002070BD092070BDF8B51468069E0D1B54
:1064B000012D1DD90519045D6D78B6F800C044EAB8
:1064C000052434801568AF1CB942176010D003351D
:1064D000A94203D273B100201860F8BDC45D3688AC
:1064E0001560012CF6D1ABB11B689BB1664503D991
:1064F0000920F8BD1846F8BD491B8E42F8D814464D
:1065000041193246184605F076FD23681E44266080
:106510000020F8BD0E20F8BD2DE9F041069EBEB169
:10652000B3B11C68A4B114680D1B022D3CD9A51C85
:10653000A94210D300EB040C075D9CF801C0156064
:10654000348847EA0C27BC4237D20C20BDE8F081E2
:106550000E20BDE8F0810027651CA94227D3045D09
:10656000156024B3EFB107F1FF3C1FFA8CFC0CF16E
:10657000010C4FEA4C0C002405F1020E714500EBB2
:1065800005080BD310F805E098F801801D684EEA65
:10659000082E25F804E01568023515600234A4457C
:1065A000EAD137800020D4E70920BDE8F08100223D
:1065B000378010461A60BDE8F0812C46CCE700BF5A
:1065C00070B4039CCAB1C3B1BCB126681D68AD1BD1
:1065D000042D15D9751C2560905525685019515505
:1065E0000D0A0A0C090E45708270C17022680432CF
:1065F000226000201A6070BC70470E2070BC70478B
:10660000092070BC704700BF70B5049C2568061C4B
:1066100018BF0126AB4212D05655256801352560BA
:1066200060B15B1B99420AD80E46014650193246AA
:1066300005F0E1FC216831442160002070BD092093
:1066400070BD00BFF8B51468BDF81870BDF81C60C7
:106650008C421DD0651CA94203D2DBB1002018601A
:10666000F8BD045D1560012CF7D1ABB11B689BB17F
:10667000BE420DD8491B8E420AD8144641193246F3
:10668000184605F0B8FC23681E4426600020F8BDBB
:106690000920F8BD1846F8BD0E20F8BD70B5049C61
:1066A00090B18AB184B126689B1B99420AD80D46E5
:1066B000014690192A4605F09EFC21682944216074
:1066C000002070BD092070BD0E2070BD70B5BDF8F2
:1066D000105083B11668891B8D420AD8144681195F
:1066E0002A46184605F087FC23681D4425600020D3
:1066F00070BD092070BD0E2070BD00BFB8B32DE97C
:10670000F041144642B11D4633B10F460646FFF72D
:106710002DFE20B1BDE8F0810E20BDE8F0816B1C9C
:10672000224639463046FFF721FE0028F2D1AB1C45
:10673000224639463046FFF719FE0028EAD1EB1C05
:10674000224639463046FFF711FE0028E2D12B1DC4
:10675000224639463046FFF709FE0028DAD16B1D84
:10676000224639463046BDE8F041FFF7FFBD0E2016
:10677000704700BFB9B12DE9F0411C4643B1054651
:1067800030B117460E46FFF7B5FD20B1BDE8F081E8
:106790000E20BDE8F08123463A463146A81CBDE8EC
:1067A000F041FFF7D1BD0E20704700BFB8B12DE911
:1067B000F041144642B11D4633B10F460646FFF77D
:1067C000AFFD20B1BDE8F0810E20BDE8F081AB1C2B
:1067D000224639463046BDE8F041FFF7C7BD0E20DE
:1067E000704700BF61B15BB110B582B050B11C46BB
:1067F000009413460A461021FFF750FF02B010BD67
:106800000E2070470E2002B010BD00BF60B130B541
:1068100083B032B12BB110240094FFF757FF03B0BF
:1068200030BD0E2003B030BD0E207047B8B12DE949
:10683000F041144642B11D4633B10F460646FFF7FC
:106840006FFD20B1BDE8F0810E20BDE8F081AB1CEA
:10685000224639463046BDE8F041FFF761BD0E20C3
:10686000704700BF09B3F0B51D4683B0D3B10446ED
:10687000C0B117460E46FFF73DFD08B103B0F0BDAD
:106880002B463A463146A01CFFF734FD0028F5D1CF
:106890002046009530F8041B3B463246FFF7FEFECB
:1068A00003B0F0BD0E2003B0F0BD0E20704700BF56
:1068B000002835D0F0B5144683B072B31D4663B3DB
:1068C0000E460746FFF72CFD08B103B0F0BD154B8F
:1068D000009322462B1D3146384600F0B7F90028B8
:1068E000F3D105F10803224631463846FCF7A8FFEC
:1068F0000028EAD105F11003224631463846FDF75B
:10690000B9F90028E1D105F1140322463146384691
:1069100003B0BDE8F040FFF74DBB0E2003B0F0BD63
:106920000E207047FD66020001B32DE9F0411D46BF
:1069300043B1044630B117460E46FFF705FD20B1BE
:10694000BDE8F0810E20BDE8F081A01C2B463A4640
:1069500031460134FFF7F8FC0028F1D12B463A46C6
:1069600031462046BDE8F041FFF7EEBC0E207047EF
:1069700000B32DE9F041154642B11C4633B10F4634
:106980000646FFF7F3FC20B1BDE8F0810E20BDE81C
:10699000F081A31C2A46394630460134FFF7E6FC55
:1069A0000028F1D123462A4639463046BDE8F04159
:1069B000FFF7DCBC0E20704799B32DE9F0431E466B
:1069C00083B053B348B304780DF10809054604F0C9
:1069D000FE00C4F30004044309F8014D4846904604
:1069E0000F46FFF7B1FCA8B96B7803F0FE04C3F3C0
:1069F00000031C4348463346424639468DF807405B
:106A0000FFF7A2FC30B9334642463946A81CFFF7CF
:106A10009BFC40B103B0BDE8F0830E2003B0BDE89D
:106A2000F0830E207047334642463946E81CFFF794
:106A30008BFC0028EED1334642463946281DFFF72D
:106A400083FCE7E7C0B3F0B5144683B08AB383B3E1
:106A50001D460DF107030F460646FFF787FC30BBC6
:106A60009DF807302A78590863F3000261F3410268
:106A70009B0863F387022A700DF10703224639460B
:106A80003046FFF773FC90B99DF807206B785108EA
:106A900062F3000361F34103920862F387036B70B2
:106AA0002246AB1C39463046FFF760FC30B103B0DC
:106AB000F0BD0E2003B0F0BD0E207047EB1C224647
:106AC00039463046FFF752FC0028F0D12B1D2246F4
:106AD00039463046FFF74AFCE9E700BFC8B1F0B5D8
:106AE00083B052B14BB11C4604330F4606461546DF
:106AF000FFF716FC20B103B0F0BD0E2003B0F0BDCF
:106B0000009023462A463946304600F09FF803B0ED
:106B1000F0BD0E20704700BFF9B12DE9F0411C46D1
:106B200043B1054630B117460E46FFF70DFC20B1C4
:106B3000BDE8F0810E20BDE8F08123463A4631469B
:106B4000A81CFFF7D7FB0028F2D123463A4631466E
:106B5000281DBDE8F041FFF7CDBB0E20704700BFF8
:106B600039B32DE9F0411C4643B1054630B1174613
:106B70000E46FFF7BFFB20B1BDE8F0810E20BDE857
:106B8000F08123463A463146A81CFFF7B3FB0028A4
:106B9000F2D123463A463146281DFFF7ABFB0028C9
:106BA000EAD123463A463146A81DBDE8F041FFF739
:106BB000A1BB0E20704700BF81B110B582B053B1A8
:106BC00048B1047802A8C4F3000400F8014DFFF7AF
:106BD000BBFB02B010BD0E2002B010BD0E207047EE
:106BE000A0B110B582B072B16BB11C460DF10703B4
:106BF000FFF7BCFB28B923789DF8072062F3000358
:106C0000237002B010BD0E2002B010BD0E207047E0
:106C1000F0B51E68059F06F1010C944514D80028B4
:106C200014BF4FF0010C4FF0000C01F806C01E68B5
:106C300006F101068E461E6005D01FB1BC46BDE8B8
:106C4000F04060473846F0BD0920F0BD2DE9F04125
:106C500014688C4282B01ED01F460DF10703804697
:106C600016460D46FFF794FB9DF80700012805D056
:106C7000B8B9D7B1386002B0BDE8F0817FB13B68E8
:106C80006BB1089A9AB11446294632464046A0474D
:106C900002B0BDE8F081092002B0BDE8F0810E200D
:106CA000E9E70B2002B0BDE8F0813846E3E7104683
:106CB000E1E700BF094B9A7832B193F82E2112B167
:106CC00004231846704701224FF4967101FB0233EA
:106CD0000121997000230260184670473C7E002015
:106CE000094B1A88824207D0B3F82C21824208BF90
:106CF000012202D00520704700224FF4967101FB5B
:106D000002330020987070473C7E00200B4B1A889D
:106D1000824205D0B3F82C21824208D0052070476A
:106D20009A78012AF6D100230B600020704793F86F
:106D30002E31012BF8D00520704700BF3C7E00208B
:106D40001C4B9A78C2B193F84E2032B393F89A2034
:106D50002AB393F8E62022B393F832211AB393F8BA
:106D60007E2112B393F8CA212AB193F81622F2B108
:106D700004231846704706224C2101FB02F110B48F
:106D800001F10C041944234401244B608C7000234E
:106D900002605DF8044B184670470122ECE70222BE
:106DA000EAE70322E8E70422E6E70522E4E7072210
:106DB000E2E700BF948000201B4B1A88824227D054
:106DC000B3F84C20824225D0B3F89820824223D0D9
:106DD000B3F8E420824221D0B3F8302182421FD0A0
:106DE000B3F87C2182421DD0B3F8C821824207D07B
:106DF000B3F81422824208BF072202D00520704750
:106E000006224C2101FB0233002098705860704725
:106E10000022F6E70122F4E70222F2E70322F0E77C
:106E20000422EEE70522ECE7948000202B4B1A8821
:106E300082421DD0B3F84C20824220D0B3F8982073
:106E4000824224D0B3F8E420824226D0B3F8302125
:106E5000824228D0B3F87C2182422AD0B3F8C821DC
:106E600082422CD0B3F8142282422ED005207047E3
:106E70009A78012ADED100220A600020704793F838
:106E80004E20012AF8D0B3F898208242DAD193F844
:106E90009A20012AD6D10222EEE793F8E620012AB1
:106EA000D4D10322E8E793F83221012AD2D1042277
:106EB000E2E793F87E21012AD0D10522DCE793F89E
:106EC000CA21012ACED10622D6E793F81632012B29
:106ED00008BF0722D0D00520704700BF9480002053
:106EE000B0B1AAB1A3B1F0B40C4E0778002401E010
:106EF0004C2C0FD016F83450BD424FEAC40C04F1AC
:106F00000104F5D16644746824B1A446F0BC60471E
:106F10000E2070470620F0BC704700BF48C002003A
:106F200060DF704762DF704763DF704764DF704780
:106F300065DF704766DF704767DF704768DF70475F
:106F400069DF704790B18AB183B130B583B01D4617
:106F500002AB14460DF1010243F8042D89B20DF184
:106F60000202F9F787FB18B103B030BD0E2070475D
:106F70000199BDF80200FFF7D5FF2A462146019B83
:106F8000F9F7A0FB03B030BD98B192B18BB170B5E9
:106F900088B01D4608AB14460DF1070243F8142DC6
:106FA00004AE89B202AA0296F9F7D8FC18B108B06B
:106FB00070BD0E207047DDE90201FFF7B5FF2A46DC
:106FC0002146039BF9F7FAFC08B070BDB8B1B2B125
:106FD000ABB170B58AB01D4605AB1446009306AA46
:106FE00010230DEB03068DF80B30039203AB0DF16C
:106FF0000B020596F9F7D0FB18B10AB070BD0E2050
:107000007047059A03999DF80B00FFF78FFF2A46FA
:107010002146059BF9F7E6FB0AB070BD10B30AB331
:1070200003B3F0B58DB01F460CAB1646102203F823
:10703000212D0C4606A905460DF1200C0846042218
:10704000079100210493CDF814C0F8F76BFA05AB53
:107050000093A1B2284604AB07AAF9F7F9FB18B1CF
:107060000DB0F0BD0E207047DDE904120798FFF760
:107070005FFF059A00929DF80F303A463146F9F7C6
:1070800027FC0DB0F0BD00BF78B172B16BB130B567
:1070900085B0144604AA1D4602AB42F80C3D89B2E5
:1070A000F9F7C2FC18B105B030BD0E207047019849
:1070B000FFF740FF2A462146019BF9F7D9FC05B0AE
:1070C00030BD00BF08B302B3FBB130B58BB01D4675
:1070D0000AAB144608AA43F8142D89B204AAF9F79A
:1070E00011F980B90498212811D0222801D106ABCA
:1070F00008930599FFF724FFDDE904322146009249
:107100002A46F9F733F90BB030BD0E2070470DF168
:107110000E030993EDE700BF70B36AB363B32DE9C3
:10712000F04188B00DF120081E464FF0FF3348F8BB
:10713000183D8CB21546214642460746F9F7CAFC6F
:10714000B8B9029B06AA212B039217D0222B01D19A
:1071500004AB069342462146384603ABF9F7C4F91F
:1071600038B9DDE90201FFF7E9FE32462946F9F7B1
:107170007BFA08B0BDE8F0810E2070470DF10603E0
:107180000793E7E7D0B1CAB1C3B1F0B5CFB01D46A0
:10719000104B029309AE04AF1446029A019206AB5B
:1071A00003960A9710AEF82703AA0C93ADF8227045
:1071B0000796F9F781F818B14FB0F0BD0E2070476F
:1071C00001A90398FFF7ACFE2A462146F9F794F887
:1071D0004FB0F0BD4C5D002058B352B34BB3F0B587
:1071E00087B01D4606AB144604AA43F8102D0DF1D6
:1071F0000602F9F79DFAD0B90299E1B103A8FFF7A9
:107200009FFDA0B903990D4ABDF80600029E4C23CC
:1072100003FB01F3D718D052191D1144B3883B81E9
:107220000291FFF789FE2A462146F9F7AFFA07B027
:10723000F0BD0E207047BDF80600F2E794800020F4
:107240006CDF70476DDF70476EDF70476FDF704730
:1072500070DF704771DF704772DF704773DF704710
:1072600074DF704775DF704776DF704777DF7047F0
:1072700078DF704779DF70477ADF70477BDF7047D0
:107280007CDF70477DDF70477EDF70477FDF7047B0
:1072900080DF704781DF704782DF704783DF704790
:1072A00084DF704785DF704786DF704787DF704770
:1072B00088DF704789DF70478EDF70478ADF70474D
:1072C0008BDF70478CDF70478DDF7047A0B19AB1BC
:1072D00093B170B58CB01D4605AB1446009308AA57
:1072E00006AB0AAE0393049204AB03AA0596FAF721
:1072F0000FF818B10CB070BD0E207047DDE9041214
:107300000398FFF7DFFF2A462146FAF745F80CB04D
:1073100070BD00BF50B14AB143B108B51146FFF787
:10732000D3FF1A46BDE80840FAF73CB80E20704774
:1073300070B16AB163B130B585B0144604AA1D4678
:1073400002AB42F80C3DFAF795FB18B105B030BD21
:107350000E2070470198FFF7B1FF2A462146FAF741
:10736000ADFB05B030BD00BFD8B1D2B1CBB170B567
:1073700096B01D46144605AB0DF10F02CDE9003263
:107380001F2206AB0EAE04938DF80E208DF80F2051
:107390000DF10E0304AA0596F9F7D2FD18B116B047
:1073A00070BD0E2070479DF80F30059A9DF80E10A5
:1073B0000498FFF751FF2A462146F9F7EDFD16B074
:1073C00070BD00BF80B17AB173B130B589B01446D9
:1073D00008AA1D4604AB42F81C3D02AB0593F9F721
:1073E000E1FD18B109B030BD0E2070470198FFF7DC
:1073F00035FF2A462146F9F7FBFD09B030BD00BF35
:1074000050B14AB143B108B51146FFF729FF1A46FA
:10741000BDE80840F9F7F2BD0E20704780B17AB19F
:1074200073B130B585B01D4604AB144602AA43F8CB
:107430000C2D0DF10202F9F7D9FE18B105B030BDDF
:107440000E2070470199BDF80200FFF70BFF2A4696
:107450002146F9F7F9FE05B030BD00BF70B16AB141
:1074600063B130B583B01D4614460DF105030DF12F
:107470000602FAF74BF818B103B030BD0E20704782
:107480009DF80510BDF80600FFF7EEFE2A462146DE
:10749000FAF764F803B030BD60B15AB153B130B5FA
:1074A00083B014460DF107021D46FAF7EFFB18B141
:1074B00003B030BD0E2070479DF90700FFF7D6FEE0
:1074C0002A462146FAF700FC03B030BD60B15AB13C
:1074D00053B130B583B014460DF106021D46F9F7DD
:1074E000EDFD18B103B030BD0E207047BDF80600A9
:1074F000FFF7BEFE2A462146F9F7FEFD03B030BD78
:1075000080B17AB173B130B583B0144602AA1D467A
:107510000DF1020342F8043D89B2F9F775FD18B187
:1075200003B030BD0E2070470198FFF7A3FE2A4636
:107530002146019BF9F78CFD03B030BD70B16AB1F3
:1075400063B130B585B0144604AA1D4602AB42F8BB
:107550000C3DFAF7B1F918B105B030BD0E207047F7
:107560000198FFF789FE2A462146FAF7C7F905B0C8
:1075700030BD00BF78B172B16BB130B585B0144683
:1075800004AA1D4602AB42F80C3D89B2FAF738F95D
:1075900018B105B030BD0E2070470198FFF76EFEA0
:1075A0002A462146019BFAF751F905B030BD00BFCC
:1075B00090B18AB183B170B5C4B01D4644AB1446D6
:1075C0000DF10E0243F8FC2D06AE04AA0496F9F75D
:1075D000EFFE18B144B070BD0E207047DDE9040124
:1075E000FFF750FEDDE9041200952346F9F70AFF84
:1075F00044B070BDB0B1AAB1A3B1F0B5C5B003AF8E
:107600001D460DF10E06F82314460497ADF80E3012
:1076100006AF04AA009605AB0597F9F741FF18B12C
:1076200045B0F0BD0E2070473288DDE90401FFF758
:1076300027FE2A462146F9F763FF45B0F0BD00BF9B
:1076400080B17AB173B130B585B01D4604AB144634
:1076500002AA43F80C2D0DF10202F9F793FD18B1BF
:1076600005B030BD0E2070470199BDF80200FFF74C
:107670000BFE2A462146F9F7B3FD05B030BD00BF29
:1076800098B192B18BB12DE9F04389B005461F4600
:10769000164606AB002203A88946CDE90323FFF76F
:1076A00009FB20B109B0BDE8F0830E207047039BB1
:1076B000DFF8A0804FF4967404FB03F408EB040396
:1076C00004F1040C04F12402424428460CEB0805A2
:1076D0005A60059504F1570204F1400545444244BF
:1076E0009D60DA6004F1670504F1A8024544424454
:1076F0001D615A6104F1C40504F1DB0245444244B2
:107700009D61DA6104F1EB0505AA0192454404AAE2
:10771000009249461A461D620DF10B03FAF736FA3C
:107720000028BFD1059B38F8040053B1049A9DF896
:107730000B10FFF7ABFD3A463146059BFAF770FA9E
:10774000B0E7FFF7CDFA0028ACD138F80400059B6C
:10775000ECE700BF3C7E002098B192B18BB170B5D0
:1077600088B01D4603AB1446009304AE89B20DF1F8
:1077700009030DF10A020396F9F7C4FC18B108B029
:1077800070BD0E207047039A9DF80910BDF80A00DD
:10779000FFF77EFD2A462146F9F7EEFC08B070BDE2
:1077A000C0B1BAB1B3B170B594B01D46144605ABC3
:1077B00006AACDE900320FAB07AA0BAE04930592DF
:1077C00089B204AB0DF10E020696FAF783F918B1EF
:1077D00014B070BD0E207047DDE905230499BDF893
:1077E0000E00FFF761FD2A462146FAF7C9F914B0E9
:1077F00070BD00BF78B172B16BB130B583B01D46BA
:1078000002AB144643F804DD0DF10202F9F722FD44
:1078100018B103B030BD0E2070470199BDF80200C9
:10782000FFF744FD2B4622460199F9F73BFD03B0D3
:1078300030BD00BF80B17AB173B130B585B01D469F
:107840000DF10D03144600930DF10E0203ABFAF790
:10785000B7F818B105B030BD0E2070479DF80D2067
:107860009DF80C10BDF80E00FFF722FD2A462146B8
:10787000FAF7D6F805B030BD60B15AB153B130B5A2
:1078800083B014460DF106021D46FAF7CFF818B181
:1078900003B030BD0E207047BDF80600FFF70AFDAB
:1078A0002A462146FAF7E0F803B030BD50B14AB19C
:1078B00043B108B51146FFF703FD1A46BDE808407D
:1078C000FAF702B90E207047A0B19AB193B170B522
:1078D0008EB01D46144605AB06AA009309AE04926D
:1078E00089B204AB0DF10E020596F9F73DFE18B111
:1078F0000EB070BD0E207047DDE90412BDF80E0019
:10790000FFF7D0FC2A462146F9F76CFE0EB070BD99
:1079100090B18AB183B130B583B01D4602AB144635
:107920000DF1010243F8042D89B20DF10202F9F7BD
:10793000EBFF18B103B030BD0E2070470199BDF8C0
:107940000200FFF7B9FC2A4621469DF90130FAF7FB
:1079500005F803B030BD00BF70B16AB163B130B596
:1079600083B01D4614460DF105030DF10602F9F72B
:107970003FFE18B103B030BD0E2070479DF80510D2
:10798000BDF80600FFF788FC2A462146F9F758FEA5
:1079900003B030BD80B17AB173B130B58BB01D4644
:1079A0000AAB144602AA43F8242D0DF10202F9F79E
:1079B0004DFE18B10BB030BD0E2070470199BDF8D7
:1079C0000200FFF767FC2A462146F9F76BFE0BB071
:1079D00030BD00BF98B192B18BB170B59AB01D4661
:1079E000144605AB06AA009310AE049204AB0DF149
:1079F0000E020596F9F7C8FE18B11AB070BD0E2038
:107A00007047DDE90412BDF80E00FFF749FC2A4675
:107A10002146F9F7EFFE1AB070BD00BFA0B19AB1D0
:107A200093B170B5A0B01D4620AB144610AA43F820
:107A30006C2D04AA009206AE0DF10E020496F9F721
:107A400037FE18B120B070BD0E207047DDE904216B
:107A5000BDF80E00FFF722FC2B4622460499F9F7E9
:107A60005DFE20B070BD00BF70B16AB163B130B5CA
:107A700085B0144604AA1D4602AB42F80C3DFAF745
:107A80007BF918B105B030BD0E2070470198FFF7A3
:107A9000D7FB2A462146FAF78FF905B030BD00BF63
:107AA00078B172B16BB130B585B0144604AA1D46E9
:107AB00002AB42F80C3D89B2FAF70CF918B105B0E7
:107AC00030BD0E2070470198FFF7BCFB2A462146C7
:107AD000019BFAF71FF905B030BD00BF78B172B154
:107AE0006BB130B589B0144602AA1D46019204ABB1
:107AF00001AA0393FAF766F918B109B030BD0E2058
:107B000070470198FFF7A4FB2A462146FAF77AF955
:107B100009B030BD80B17AB173B130B589B01446C7
:107B200002AA1D46019204AB89B201AA0393FAF797
:107B30006FF918B109B030BD0E2070470198FFF7FA
:107B400089FB2A462146019BFAF782F909B030BD2C
:107B5000002831D0002A2FD073B370B598B01D46DD
:107B600014460AAB0DF12F020DF136060293039273
:107B70000DF13D0311AA049605930DF14B060DF18D
:107B8000520306920DF159020796089302AE09922C
:107B90000DF1030301AA0196FAF790F908B118B0A4
:107BA00070BD9DF803100198FFF74EFB2A46214651
:107BB000FAF7D8F918B070BD0E20704700284BD0E6
:107BC000002A49D0002B47D02DE9F041E4B01F46F0
:107BD00036AB06930DF1EF0307930DF5837308930E
:107BE0000DF21D1309934DAB0A930DF24B130B933A
:107BF0000DF5B1730C930DF279130D9316AB0E9333
:107C00001AAB0F931EAB109322AB119326AB1293BA
:107C10002AAB13932EAB0DF10F08149332AB16461B
:107C200006AD0EAC1593CDF8008004AA05AB049503
:107C30000594FAF79DF910B164B0BDE8F08198F8A9
:107C40000020DDE90401FFF701FB3A463146FAF76F
:107C50001BFA64B0BDE8F0810E20704794DF7047D6
:107C600095DF704796DF704797DF704799DF704761
:107C70009ADF70479BDF70479CDF70479DDF70473E
:107C800098DF70479EDF704790B18AB183B170B5BD
:107C900086B01D4605AB1446009304AE89B20DF1C3
:107CA0000E0303AA0596FCF729F918B106B070BDBA
:107CB0000E207047059ABDF80E10BDF80C00FFF7B6
:107CC000CDFF2A462146FCF74BF906B070BD00BF38
:107CD00088B182B17BB130B585B01D4604AB144686
:107CE00002AA43F8042D89B20DF10602FCF772F9DD
:107CF00018B105B030BD0E2070470399BDF80600DD
:107D0000FFF7AEFF2A462146FCF78EF905B030BDDD
:107D100088B182B17BB130B585B01D4604AB144645
:107D200002AA43F8042D89B20DF10602FCF75AF8B5
:107D300018B105B030BD0E2070470399BDF806009C
:107D4000FFF790FF2A462146FCF776F805B030BDD4
:107D500088B182B17BB130B585B01D4604AB144605
:107D600002AA43F8042D89B20DF10602FCF76AF865
:107D700018B105B030BD0E2070470399BDF806005C
:107D8000FFF772FF2A462146FCF786F805B030BDA2
:107D9000B8B1B2B1ABB170B588B0144608AA1D46EF
:107DA000002342F8103D07AB009306AE059289B25E
:107DB00005AB0DF10E020796FBF79CFF18B108B05A
:107DC00070BD0E207047079A0599BDF80E00FFF7A9
:107DD0004DFF2A462146FBF7CBFF08B070BD00BF20
:107DE00088B182B17BB130B585B01D460DF10E036F
:107DF0001446009389B203AB0DF10A02FCF7B6F802
:107E000018B105B030BD0E207047BDF80E20BDF88A
:107E10000C10BDF80A00FFF72BFF2A462146FCF79D
:107E2000D3F805B030BD00BFA8B1A2B19BB170B509
:107E30008AB01D4614460DF10A0304AA00930B26CE
:107E4000039289B203AB02AAADF80A60FBF796FF72
:107E500018B10AB070BD0E207047BDF80A20039912
:107E6000BDF80800FFF706FF2A462146FBF7B4FFDE
:107E70000AB070BDC8B1C2B1BBB170B5C2B01546D1
:107E8000F4221E46ADF80E2005AB002202AC04938E
:107E90000292ADF80C2089B201AB0DF102020194FF
:107EA000FCF7C8F818B142B070BD0E2070470199B8
:107EB000BDF80200FFF7E0FE32462946FCF7E4F881
:107EC00042B070BD68B162B15BB130B583B01D46E0
:107ED00014460DF1060301AAFBF7E4FF18B103B045
:107EE00030BD0E207047BDF80610BDF80400FFF746
:107EF000C5FE2A462146FBF7FBFF03B030BD00BF9D
:107F0000A0B19AB193B130B585B0144604AA1D460C
:107F1000002342F8083D04AB89B243F8042D0DF16B
:107F20000602FBF7B3FE18B105B030BD0E20704756
:107F30000399BDF80600FFF7A3FE2A462146FBF78A
:107F4000D3FE05B030BD00BF70B16AB163B130B5CA
:107F500083B01D46144689B20DF1060301AAFCF751
:107F600099F818B103B030BD0E207047BDF8061067
:107F7000BDF80400FFF786FE2A462146FCF7B0F85C
:107F800003B030BDA0DF7047A1DF7047A2DF7047AC
:107F9000A3DF7047A4DF7047A5DF7047A6DF7047F7
:107FA000A7DF7047A8DF7047A9DF7047AADF7047D7
:107FB000ABDF7047ACDF7047ADDF7047B8B1B2B12F
:107FC000ABB170B586B0144606AA1D46002342F830
:107FD0000C3D05AB00930DF10A06049204AB0DF1C4
:107FE00009020596FDF730F918B106B070BD0E20F4
:107FF0007047DDE904129DF80900FFF7C3FF2A4628
:108000002146059BFDF754F906B070BD002835D018
:10801000002A33D0002B31D02DE9F043ADF2744D5E
:108020001F461CAB16930CAB189304AB199305AB0E
:108030001A9306AB16461B9309AA4FF4007315ACAE
:108040000DF128090DF12C08ADF85E30ADF848307F
:10805000109207AB9CAA10AD0894119314920EAC29
:10806000CDE9009808AB0DF10E020A950B94FCF7D0
:10807000BFFE28B10DF2744DBDE8F0830E207047AD
:10808000D9F800200899D8F80030BDF80E00FFF7A5
:108090007DFFD8F800303A463146FCF7E9FE0DF294
:1080A000744DBDE8F08300BF98B192B18BB170B54B
:1080B00086B01D4605AB144600930DF1120689B239
:1080C00004AB0DF10E020596FCF7D2FF18B106B015
:1080D00070BD0E207047059ABDF81010BDF80E0057
:1080E000FFF752FF2A462146059BFCF7F1FF06B039
:1080F00070BD00BFF8B1F2B1EBB1F0B5ADF50D7DDB
:10810000154604AA079203AA08920CAA07AC06AF68
:108110000B924FF400721E460594ADF824200DF129
:108120000A0405AB009702AA0694FCF7D7FE20B11B
:108130000DF50D7DF0BD0E20704705993A68BDF82C
:108140000800FFF725FF3B6832462946FCF7FAFE98
:108150000DF50D7DF0BD00BFC8B1C2B1BBB1F0B52A
:10816000ADF5077D1D4614464FF4007306AA03AF14
:1081700004AE0493059289B200970DF10A0302AA96
:108180000396FDF74DFA20B10DF5077DF0BD0E20E9
:108190007047BDF80A103A68BDF80800FFF7FAFE0C
:1081A0003B682A462146FDF76DFA0DF5077DF0BDC7
:1081B000B0B1AAB1A3B1F0B5ADF5077D144603AED9
:1081C00004AA1D4606AF039289B200960DF10A0378
:1081D00002AA0597FDF794F920B10DF5077DF0BDD2
:1081E0000E207047BDF80A103268BDF80800FFF78E
:1081F000D3FE33682A462146FDF7DCF90DF5077DED
:10820000F0BD00BFC8B1C2B1BBB170B5ADF5067D60
:1082100014464FF400721D46ADF802200DF1020322
:1082200006AA02AE0493059201AB6A460196FCF7DA
:10823000BFFE20B10DF5067D70BD0E207047BDF864
:1082400000000199FFF7AAFE019B03B19B682A4633
:108250002146FCF7D7FE0DF5067D70BD80B17AB1E1
:1082600073B130B585B01D460DF10E031446009371
:108270000DF10A0203ABFDF751F818B105B030BD9E
:108280000E207047BDF80E20BDF80C10BDF80A0096
:10829000FFF786FE2A462146FDF76EF805B030BD91
:1082A000B8B1B2B1ABB170B5ADF5067D06AE14464E
:1082B00002AA1D460192059601AB4FF400760DF11E
:1082C0000202ADF81260FCF78FFF20B10DF5067DBC
:1082D00070BD0E2070470199BDF80200FFF762FEE5
:1082E0002A462146FCF7AAFF0DF5067D70BD00BFAA
:1082F000C8B1C2B1BBB1F0B5ADF5077D14460DF103
:108300000E0606AA05AF1D464FF4007C049204AB8E
:10831000CDE9006703AAADF80EC0FDF7BBF820B1A8
:108320000DF5077DF0BD0E2070473B68328804993B
:10833000BDF80C00FFF738FE2A462146FDF7DAF8B3
:108340000DF5077DF0BD00BFF0B1EAB1E3B12DE955
:10835000F041ADF5067D144606AA04AE0DF11408F1
:1083600003924FF400721D460DF10A07ADF80A2082
:1083700003ABCDE9006802AA0497FDF703F828B122
:108380000DF5067DBDE8F0810E207047D8F800306D
:1083900032680399BDF80800FFF708FE32680092C2
:1083A000039B2A462146FDF729F80DF5067DBDE819
:1083B000F08100BFA0B19AB193B170B588B01D46ED
:1083C00008AB144606AA43F8042D05AA009204AE91
:1083D0000DF10E020596FCF799FC18B108B070BDBE
:1083E0000E207047059A0799BDF80E00FFF7E2FDD1
:1083F000059A0092079B2A462146FCF7B7FC08B075
:1084000070BD00BF78B172B16BB130B583B01446A6
:1084100002AA1D460DF1020342F8043DFCF78EFE50
:1084200018B103B030BD0E2070470198FFF7C0FDB2
:108430002A462146019BFCF7A1FE03B030BD00BFD8
:1084400070B16AB163B130B583B01D46144689B2CC
:108450000DF1060301AAFDF74BF918B103B030BDC9
:108460000E207047BDF80610BDF80400FFF7A4FD0C
:108470002A462146FDF762F903B030BDB0DF7047F0
:10848000B1DF7047B2DF704760B15AB153B130B558
:1084900083B014460DF106021D46FDF71DFE18B10E
:1084A00003B030BD0E207047BDF80600FFF7E6FFB1
:1084B0002A462146FDF72EFE03B030BD60B15AB109
:1084C00053B130B583B014460DF106021D46FDF7D9
:1084D00027FE18B103B030BD0E207047BDF806006E
:1084E000FFF7CEFF2A462146FDF738FE03B030BD28
:1084F00098B192B18BB170B586B01D46144605ABEC
:1085000003AA00930026049204AB0DF10A0205961B
:10851000FDF72AFE18B106B070BD0E207047DDE9E8
:108520000412BDF80A00FFF7ADFF2A462146FDF709
:1085300055FE06B070BD00BF32DF704743DF7047A5
:1085400049DF704738B132B12BB108B589B200F0BC
:108550002DF910B108BD0E207047BDE80840FFF7A7
:10856000EBBF00BF68B162B15BB130B583B01446F8
:1085700002AA1D4642F804DD00F026F918B103B046
:1085800030BD0E2070470198FFF7DAFF2A462146DA
:10859000019B00F039F903B030BD00BF70B16AB182
:1085A00063B130B58FB014460EAA1D4602AB42F837
:1085B000343D00F0A5F818B10FB030BD0E20704763
:1085C0000198FFF7BBFF2A462146019B00F0B8F84F
:1085D0000FB030BD2DE9F04F8DB06B4683E803003E
:1085E0009DF805600A2E73D8404D414F0FCD04AC65
:1085F0000FC495E80F0057F826509DF800700597B6
:1086000084E80F009DF801303A480A95049302F07F
:10861000D9FA04A90022374802F0ECF910B10DB0E4
:10862000BDE8F08F3348DFF8D4A002F01BFD324BD9
:1086300053F82630CAF8003002F006FF80460028C2
:108640004FD1DFF8B0900446074602F097FF0122B1
:1086500083460DF10E01484602F0E2FB0646002873
:108660003FD19DF80EC0BFB3DAF80050454444EA4C
:108670000C045D4504F00303C4F38502C4F3052133
:10868000C4F38F3003D24FEA0C24D846DDE7032B26
:1086900008BF4FF0FF3302F0F3FF04A803F084F9A2
:1086A00007460028D1D0049B0DF10F011B0A0122BF
:1086B00048468DF80F3002F009FB049B8DF80F300F
:1086C00001220DF10F014846374602F0FFFABCE7E0
:1086D00007200DB0BDE8F08F4FEA0C24D8460127E3
:1086E000B3E703200DB0BDE8F08F00BFA8C20200C1
:1086F000C8C20200285D0020F4C20200305D0020E4
:10870000D0B130B50C4685B011B10378432B02D0FF
:10871000072005B030BD134604AA012542F8045DC8
:10872000064D0095FEF792FA0028F2D1039BA34272
:1087300018BF092005B030BD0E20704775880200B3
:10874000F0B587B0039001B3FAB1176800201D4659
:1087500014464FF0430C05903A4605AB0DF113005B
:108760000E468DF813C0FDF7EFFD08B107B0F0BD60
:1087700005AB3A46314603A8FDF782FD0028F5D146
:10878000039B2BB1059B2360F0E70E2007B0F0BDE3
:10879000054B00933A4605AB31462846FEF738FABA
:1087A0000028EFD0E2E700BFC188020050B139B124
:1087B0000378322B04D1012914BF0920002070470F
:1087C000072070470E207047D8B170B50C4684B0B2
:1087D00021B10378492B4FF0000502D0072004B0E7
:1087E00070BD134604AA012642F8046D0095FEF7F9
:1087F0002DFA0028F3D1039BA34218BF092004B02F
:1088000070BD0E20704700BFF0B587B0039001B374
:10881000FAB1176800201D4614464FF0490C059028
:108820003A4605AB0DF113000E468DF813C0FDF767
:108830008BFD08B107B0F0BD05AB3A46314603A841
:10884000FDF71EFD0028F5D1039B2BB1059B23608E
:10885000F0E70E2007B0F0BD054B00933A4605AB9C
:1088600031462846FEF7D4F90028EFD0E2E700BFF2
:108870008162020010B32DE9F041144682B06AB162
:108880001D465BB14FF01008CDF800800E4607463C
:10889000FDF71CFF30B102B0BDE8F0810E2002B040
:1088A000BDE8F081CDF8008005EB08032246314693
:1088B0003846FDF70BFF02B0BDE8F0810E2070478F
:1088C00069B163B158B110B582B01C46009413462B
:1088D00020300A461021FDF7E1FE02B010BD0E2047
:1088E000704700BFF0B587B080B359B30023CDE91E
:1088F00003330778059305460E4604A903A800F044
:1089000019FB04280446F8D0C0B9039B01221A7051
:10891000DDE90323284631465D1E013204AB049590
:10892000FEF7DEFA0628054614D038B9DDE9030360
:10893000013399B2049300F017FB00B103242046E1
:1089400007B0F0BD0924204607B0F0BD0E24204634
:1089500007B0F0BD0748F6F7EFFD039A05AE04AB8C
:108960002946384601320096FDF72AFE0028DDD060
:10897000E4E700BFFECADDBA11DF7047002832D03D
:1089800070B582B002AC002344F8043D06460D46A3
:1089900000932146684600F0CDFA0428F9D008B1CA
:1089A00002B070BD009B114A04211970019B294639
:1089B000013B30460193F8F7A7F888B900992246A1
:1089C0000131F8F7CBF858B9019B094A00980133F7
:1089D000012499B20193147000F0C6FA0028DFD088
:1089E000032002B070BD0E20704700BFB05D0020B4
:1089F000B65D002008B5074B1B7803B908BDFFF72B
:108A0000BBFF00F04BFA044B93E80300BDE80840BD
:108A1000FFF7E0BDB65D0020B05D002010B582B06C
:108A200002AB002203F8012D04461846F7F7E4FADA
:108A30000A4B9C4205D19DF80700F7F703FB02B0F3
:108A400010BDBFF34F8F0649064BCA6802F4E062BF
:108A50001343CB60BFF34F8F00BFFDE7FECADDBA03
:108A600000ED00E00400FA0530B5054683B00028AB
:108A70003BD002AC002344F8043D009321466846F5
:108A800000F058FA0428F9D0E8B9009B02221A70C5
:108A9000DDE90021234628464C1E013200210194C5
:108AA000F8F772F8062814D080B9DDE90003013325
:108AB00099B2019300F058FA08B1F6F73DFDF6F7C8
:108AC0000DFE03B030BDF6F737FDDEE7F6F734FDF7
:108AD000EBE7009800F07AFA20B90648F6F72CFD8B
:108AE00003B030BDF6F728FDF7E70E20F6F724FDBA
:108AF000BFE700BFFECADDBA00B585B004AB03E92D
:108B000007009DF80430042B07D8DFE803F00910B4
:108B1000152103000F20F6F70FFD05B05DF804FBEB
:108B2000F6F7F4FDFFF766FF05B05DF804FBF6F716
:108B3000D5FD05B05DF804FB08220DEB02010748E6
:108B400003F059FA064B01221A7005B05DF804FBD8
:108B50000448F6F7F1FC05B05DF804FBB85D0020B1
:108B6000C05D0020FECADDBA044B187800B970471A
:108B7000002203481A7000F01BB800BFC05D00203F
:108B8000B85D002008B54188084A043189B2F6F77B
:108B900027FD38B9F6F70AFD00B108BDBDE8084069
:108BA00003F0D6B9F6F7C8FCF4E700BF698A020003
:108BB00018B310B504460068A18803780139032B67
:108BC00089B200F1010013D0052B0ED03BB10C4847
:108BD000F6F7B2FC206800F075F920B910BDFFF778
:108BE00081FE0028F6D0032010BD00F00BF8F1E75D
:108BF000FFF7C4FE0028EDD0F5E70E20704700BF58
:108C0000FECADDBABFF34F8F0549064BCA6802F4AE
:108C1000E0621343CB60BFF34F8F00BFFDE700BF9F
:108C200000ED00E00400FA05F0B589B001AB05AC39
:108C300083E807000C2220460021F6F773FC9DF81C
:108C4000043005228DF81420062B09D8DFE803F044
:108C50000426406555620D00784B1A78032A7AD0B5
:108C60000020F6F769FC09B0F0BD744A029B117848
:108C700007930220042303298DF814308DF818007F
:108C800000F090806E4D2E78022E00F0A3806D4B88
:108C900094E807001B68984709B0F0BDBDF80820AC
:108CA000674D0121B2F5FA7F2B788DF8141042D868
:108CB0008B425BD1634B94E807001B68984762487E
:108CC00001F0A2F808B1F6F737FC02232B70CAE7CF
:108CD0005B4B1A78022AC3D10298BDF80C10594D8B
:108CE0008DF814200690ADF81C1094E807002C684D
:108CF00004251D70A04709B0F0BD04210022514B8E
:108D00008DF814108DF8182094E807001B68984718
:108D100009B0F0BD04210122F1E7494D2B78032B66
:108D20004AD1484E8DF8143094E8070033689847CC
:108D300001232B7097E7012B23D1424B94E80700C6
:108D40001B689847002001F05FF808B1F6F7F4FBC4
:108D500003232B7087E700223A4D8DF8142094E806
:108D600007002C6801251D70A0477CE7042B7FF4C9
:108D700077AF344B94E807001B68984705232B70A6
:108D800071E7042B7FF46CAF2E4B94E807001B684F
:108D90009847002001F038F808B1F6F7CDFB06231C
:108DA0002B7060E70399137049B3284B99422BD07D
:108DB0001020F6F7C1FB6AE7062B7FF451AF0322C0
:108DC000204B8DF814201B6894E807009847042373
:108DD0002B7048E7039F2B7001F000F86FB11A4B1E
:108DE0009F420ED12B78042B11D0062B14D0052BCB
:108DF00017D000F0F3FE0820DBE700F0EFFE0E20B6
:108E0000D7E700F0EBFED3E7012313703FE7012320
:108E10002B7000F0E3FE3AE703232B7000F0DEFE38
:108E200035E7384600F0F0FF18B92E7000F0D6FE96
:108E30002DE700F0D3FE0320BBE700BFB4610020A4
:108E4000BC5F0020C45D0020C85D0020C05F002022
:108E5000F8B50E4C2378A3B90D4E35788DB990B185
:108E60000C4F03463B600C4801232370337001F024
:108E700053F828B1072818BF0320257035703D60CE
:108E8000F8BD0820F8BD0E20F8BD00BFBC5F002073
:108E9000B4610020C45D0020298C020008B500F0F8
:108EA0009DFF05480549064A002303700B701360B7
:108EB000BDE8084001F098B8BC5F0020B461002014
:108EC000C45D002038B5044600F088FFC4B1174BDC
:108ED0009C4204D0102400F081FE204638BD144D81
:108EE0002B78042B11D0062B06D0052B14D0082488
:108EF00000F074FE204638BD03232B700024EAE7FF
:108F00000E2400F06BFE204638BD012300242B7098
:108F100000F064FE204638BD204600F075FF044690
:108F200010B902232B70D6E70324D4E7C85D0020D4
:108F3000BC5F002080B179B1094A137853B1012B8D
:108F40000CD1084B036002204FF4FA7310700B80B1
:108F500000207047082070470E207047042070479B
:108F6000B4610020C05F0020A8B181B1154B9842C8
:108F700001D010207047B1F5FA7F0AD870B5124EB3
:108F80003378022B82B008D0082002B070BD0720D1
:108F900070470C2070470E20704704460D4600F0C5
:108FA0001DFF2946204600F075FF38B1112818BF73
:108FB0000320019000F012FE0198E6E703233370CE
:108FC000F7E700BFC05F0020B461002080B1094B0B
:108FD000984201D010207047074B1A78022A01D01E
:108FE000042A03D101221A7000207047082070471C
:108FF0000E207047C05F0020B4610020F0B5244E01
:1090000024493388244A0C681278244D244F1B01CC
:1090100043F00E03E4001BB242F0C00204F4FF640C
:10902000D9B21443C3F3072351FA84F21A445242CB
:1090300089B0EA706970002204212846AB702C7058
:10904000F7F718F808AA318822F81A0D3868F7F7E8
:1090500011F8144B3968328804910446000A042739
:109060000226ADF81420587006AA04A902A81C70A4
:10907000ADF8064002950693ADF80C70ADF81C6093
:1090800001F074FB10B10020F6F756FA09B0F0BDFC
:1090900024640020C8610020CC61002020640020EE
:1090A000C46100201C64002070B5204A204B128847
:1090B00047F601600021824286B0197010D047F651
:1090C000025082420CD04FF60340824226D047F62F
:1090D00004308242174D22D00846F1220F2104E0CD
:1090E000144D2F212A800220D122002459700426F9
:1090F000DA70ADF80C0004AA02A968469C700093CF
:1091000002950494ADF81440ADF8046001F02EFB14
:1091100010B12046F6F710FA06B070BD054D2A8052
:109120001121A970C1223F210320DEE7365D002016
:1091300014640020186400202DE9F041784E794C29
:10914000794F90B0002501A88DF80450F6F754FF30
:109150002A460CA93046F7F711F858B99DF80400D3
:10916000F6F770FF2378042B45D8DFE803F0545856
:109170000D8D48006D4B9DF8040001221A70F6F722
:1091800061FF10B0BDE8F0819DF83030002BD9D1DF
:109190009DF83430012BD5D1654B186850B1654B23
:1091A000654D1A882968063A043102F024FF2868C0
:1091B00001F02CFB614A624813680190013303F00F
:1091C00007034FEAC30C1360CCF100030025C37002
:1091D000042380F800C045704FF0030C85702A46C8
:1091E00029460DEB030084F800C0ADF8083001F00B
:1091F000BDFA0028A6D00020F6F79EF9A2E79DF858
:109200003030012B03D19DF83430012B5BD00E9808
:1092100001F0FCFA96E73B78032B93D1EBE79DF83E
:109220003030012B8ED19DF83420022A8AD10E993C
:10923000DFF808810A7898F8000002F007028242FD
:1092400044D03D4B04251868257001F0DFFAD8F8AA
:109250000030DFF8ECC0ADF80850DB00DBB20025D1
:1092600059428CF803102A46294601A88CF8003090
:10927000CDF804C08CF801508CF8025001F076FA59
:1092800000283FF45FAFB6E79DF83030012B7FF444
:1092900059AF9DF83430012B03D0022B7FF452AF2D
:1092A000B5E7234A274B12681B687AB32149079216
:1092B0000A880221063AADF820208DF8181013B163
:1092C00006AA07CA9847012323703BE7BDF83C2054
:1092D000184DDFF874C018482A80062A8CF8003030
:1092E000016003D80020F6F727F92A88154B1D687E
:1092F000063A0123ADF828208DF824301DB109ABC2
:1093000093E80700A847022323701BE703228DF888
:109310000C20002BD7D003AA07CA9847D3E700BF79
:1093200020C30200B8610020B6610020395D002032
:10933000BC610020EC620020C0610020C8610020F8
:10934000F4620020F0620020B5610020F0B5904E7C
:10935000904C914F8FB000250DF103008DF8035014
:10936000F6F74AFE2A460AA93046F6F707FF58B92B
:109370009DF80300F6F766FE2378052B1CD8DFE87E
:1093800003F0181F3643770C844B9DF8030001222D
:109390001A70F6F757FE0FB0F0BD9DF82830012B7C
:1093A000D9D19DF82C30002B00F0D980022BD2D1DE
:1093B00028E03B78032BCED10020F6F7BDF8CAE7B2
:1093C0009DF82830002B70D19DF82C30002BC2D195
:1093D000FFF714FE724B734A4FF40031C3F80813C1
:1093E000012159600521022311602370B3E79DF824
:1093F0002830012BAFD19DF82C20002A00F0968058
:10940000022AA8D10C982DE09DF82830012BA2D17A
:109410009DF82C20002A00F08980022A9BD10C980C
:10942000027843788578C17813442B440B4413F0B9
:10943000FF0F17D15C4B1B680133C2F3C20203F06C
:1094400007039A4204D0013303F007039A4209D17B
:10945000534B4FF400310122C3F808135A600C98A3
:109460000523237001F0D2F900283FF474AFA3E77D
:109470009DF82830012B1ED0022B7FF46CAF494A97
:109480001368013B1360002B7CD1484A484B156898
:109490001B68039306238DF804301DB101AB93E8DC
:1094A0000700A8470123237055E7012B7FF453AF32
:1094B0009DF82C307AE79DF82C30022B7FF44BAFCF
:1094C0000C98017843788578C2780B442B44134478
:1094D00013F0FF0FC6D1DFF8D0C0DCF80030013345
:1094E000C1F3C20103F00702914204D0013202F03D
:1094F00007029142B6D12A4A2C494FF40030C2F8F3
:109500000803012050600D682949002203F0070379
:10951000CCF800300A608DF810201DB104AB93E840
:109520000700A84701230C9823709BE71C494FF4C0
:10953000003541F64660C1F80853C1F84405D1F83A
:1095400044054FF0040C3E30C1F84405CB60C1F82F
:1095500044210B60C1F8045384F800C0FBE61249B3
:1095600012480A6805688DF81C30013202F00702C3
:109570000A600F4A1360002D94D007AB93E80700F0
:10958000A8478FE7FFF73AFD03232370E3E600BF08
:1095900034C30200BA610020B66100203A5D0020A9
:1095A00000A0004028640020CC610020F062002070
:1095B000C4610020F0B5047887B054B9874B8DF8AA
:1095C0000C401B780122032B8DF808205CD007B0DB
:1095D000F0BD012C78D0022CF9D1436800898DF8B8
:1095E0000C4001220493ADF814008DF80820002BE4
:1095F00000F0AF80002800F0B6800328049C40F201
:10960000D380637803F00F05052D00F01782002D3D
:1096100000F085800E2D00F0AB800F2D40F0C4804F
:109620009DF80820012A00F0EB80022ACFD106A87D
:10963000002500F8115DF6F7DFFC684B1C78012C63
:1096400000F08281022C1AD1654B4FF603421A803A
:10965000FFF72AFD634B4FF4003141F64662C3F831
:109660000813C3F84425D3F8442501203E32C3F83B
:109670004425D860C3F844511860C3F804139DF81A
:109680000700F6F7DFFCA2E7574B1B78002B9ED0B4
:1096900006A800F8114DF6F7AFFC02A95348F6F7FB
:1096A00007FD00285BD1524B9DF807001A78002A6D
:1096B000E7D0504A1278002AE3D000221A70F6F759
:1096C000C1FCFFF743FE82E7444B8DF808401B784E
:1096D0008DF80C40032B7FF47AAF434B1B78002BA3
:1096E0003FF475AF06A8002400F8114DF6F784FC8E
:1096F00002A94148F6F7DCFC00286BD13F4B9DF8EE
:1097000007001A78002ABCD03A4A1278002AB8D04A
:1097100000221A70F6F796FCFFF70EFD57E72F4B65
:109720001B78032B11D1304B1B7873B106A800F8BE
:10973000115DF6F761FC02A92C48F6F7B9FC002888
:10974000B1D02846F5F7F8FEADE7204601F05EF807
:109750003DE71846F5F7F0FEBDF814004AE720464D
:10976000F5F7EAFE9FE7F5F7E7FEBDF8140044E7DA
:10977000042819D02278570616D5160614D5A578D0
:10978000E17813442B440B4413F0FF020CD1851EE7
:1097900029462046F6F76EFC6219635D527843EA6B
:1097A000022398420AD0049C204601F02FF800289A
:1097B0003FF40DAF0020F5F7BFFE08E7074B1B781D
:1097C000032B03D1084B1B78002B8BD1049801F09D
:1097D0001DF8FCE62046F5F7AFFE8FE7B6610020E6
:1097E000365D002000A00040B761002034C30200B5
:1097F0003A5D0020345D002020C30200395D002066
:109800002278550676D4110674D4A578E1781344ED
:109810002B440B4413F0FF0F6CD1627925794FF67E
:10982000034345EA02259D426DD047F604339D422D
:1098300069D047F601639D4200F0A18047F60253CC
:109840009D4257D1062855D106AC002304F8113D9E
:109850002046F6F7D1FB804D2B78012B00F0D1800C
:109860009DF80700F6F7EEFB049800F0CFFF2B7889
:10987000032B7FF4ACAE794B1B78002B3FF4A7AEE3
:10988000204600268DF80760F6F7B6FB7448F6F719
:10989000F1FC744B1A783AB1734A127822B118B1BC
:1098A0002A78032A00F0C2809DF80700F6F7CAFB69
:1098B000204600248DF80740F6F79EFB6B48F6F72C
:1098C000D9FC6B4B1A78002A3FF4D9AE664A12785D
:1098D000002A3FF4D4AE00283FF4D1AE2A78032A00
:1098E0007FF4CDAE9DF807001C70F6F7ABFBFFF7D9
:1098F00023FC6CE606AC002304F8113D2046F6F785
:109900007BFB554DACE70728F4D1A379112BF1D19E
:1099100006AC002304F8113D2046F6F76DFB47F630
:1099200002539D4297D054D847F604339D424A4D86
:1099300096D12B78022B93D14E484F490123032215
:1099400003700B702A708BE74C4B47F601621A804C
:10995000FFF7AAFB4A4B4FF4003141F64662C3F8C9
:109960000813C3F84425D3F844253E32C3F84425F0
:10997000DC60C3F844511C60C3F804137FE606287A
:10998000B8D106AC002304F8113D2046F6F734FBAD
:10999000314D3A4A2B7847F60251032B118037D0CC
:1099A000FFF782FB364B4FF4003141F64662C3F8B5
:1099B0000813C3F84425D3F8442501203E3200267D
:1099C000C3F84425D860C3F844611860C3F8041391
:1099D00046E747F601639D42DAD04FF603439D42C6
:1099E0001D4D7FF43DAF2B78012B3FF439AF234B56
:1099F00047F604321A80FFF757FB184B01221A7002
:109A00002EE71E4A4FF60341022311802B7027E7F1
:109A1000184A1C4F1C4E184810490023137001228D
:109A20003B60336003700B702A70B9E79DF8070044
:109A30001E70F6F707FBFFF789FC39E7BFF34F8F7E
:109A40001249134BCA6802F4E0621343CB60BFF3C0
:109A50004F8F00BFFDE700BFB6610020B761002057
:109A600034C302003A5D0020345D002020C30200B0
:109A7000395D0020BA610020B8610020365D002009
:109A800000A00040C8610020CC61002000ED00E093
:109A90000400FA052DE9F043474CD4F84451012D58
:109AA00087B002D007B0BDE8F083D4F804339B033D
:109AB000F8D50026414BC4F84461E5601B7823B912
:109AC0003F4B1D7007B0BDE8F08306AFDFF808918B
:109AD00007F8116D022338468DF80C608DF80830B8
:109AE000F6F78AFA99F80080B8F1010F41D0B8F181
:109AF000020F18D1334B4FF603421A80FFF7D4FA06
:109B00004FF4003241F64663C4F80823C4F84435E4
:109B1000D4F844353E33C4F84435E560C4F84461B4
:109B20002560C4F804239DF80700F6F78BFA99F82E
:109B30000030032BB6D1244B1B78002BB2D0384613
:109B400000248DF80740F6F757FA02A91F48F6F7E8
:109B5000AFFA68BB1E4B9DF807001A782AB31D4A5E
:109B6000127812B300221A70F6F76CFAFFF7EEFBC8
:109B700098E7144B47F601621A80FFF795FA4FF405
:109B8000003241F64663C4F80823C4F84435D4F8DB
:109B900044353E33C4F84435C4F80C80C4F84461FD
:109BA000C4F80080C4F80423BDE7F6F74BFA79E760
:109BB0002046F5F7C1FCCDE700A00040385D00204D
:109BC000B9610020365D0020B761002034C3020077
:109BD0003A5D0020345D0020B66100202DE9F04799
:109BE00086B006AC002504F8105D2046F6F704FAAE
:109BF0006F4B704A1E780121117006B11D709DF8DF
:109C000008006D4D6D4FF6F71DFA4FF00008012367
:109C100020462B708DF80880F6F7EEF96848F6F7C5
:109C200029FB3B7833BB9DF80800F6F70BFA20467A
:109C30004FF000088DF80880F6F7DEF96148F6F776
:109C400019FB614B1A78F2B129789DF80820002998
:109C500077D0002875D05D4909780329104614D1C2
:109C600083F80080F6F7EEF9FFF766FA8EB906B0D2
:109C7000BDE8F0872A789DF80830002A65D118469B
:109C8000F6F7E0F9D3E79DF80800F6F7DBF9002EC8
:109C9000EDD006AE4FF0000806F8118DDFF82CA1CC
:109CA0008DF80C80022330468DF80830F6F7A4F9C1
:109CB0009AF80090B9F1010F55D0B9F1020F1AD1FD
:109CC000434B4FF603421A80FFF7EEF9414B4FF436
:109CD000003141F64662C3F80813C3F84425D3F8AF
:109CE000442501203E32C3F84425D860C3F844819E
:109CF0001860C3F804139DF80700F6F7A3F99AF863
:109D00000030032BB3D1344B1B78002BAFD030463F
:109D100000268DF80760F6F76FF921462848F6F718
:109D2000C7F900283FD13B789DF80700002B37D0BA
:109D30002B78ABB300233B70F6F784F9FFF706FBF3
:109D400095E71046F6F77EF990E7002897D01F4A6E
:109D50001278032A184693D187F80080F6F772F933
:109D6000FFF7F4FA63E71A4B47F601621A80FFF730
:109D70009BF9184B4FF4003141F64662C3F80813C3
:109D8000C3F84425D3F844253E32C3F84425C3F82C
:109D90000C90C3F84481C3F80090C3F80413AAE7F9
:109DA000F6F750F963E73046F5F7C6FBBBE700BFAF
:109DB000B9610020385D0020345D00203A5D00204C
:109DC00034C3020020C30200395D0020B6610020C8
:109DD000365D002000A00040B761002010B582B0C1
:109DE00002A8002400F8014DF6F706F9044A054BD5
:109DF0009DF8070014701C70F6F724F902B010BD2E
:109E0000385D0020345D00201D4A137863B310B51F
:109E100086B0034606A800241A4900F8114D1470B4
:109E200001220B608DF808408DF80C20F6F7E4F85D
:109E300002A91548F6F73CF9C0B9144B9DF8070084
:109E40001C7824B9F6F7FEF8204606B010BD104A7B
:109E50001478002CF6D000241C70F6F7F3F8FFF706
:109E60006BF9204606B010BD112070472046F5F76B
:109E700063FB064B9DF807001C78002CE7D1E1E757
:109E8000B5610020BC61002020C30200395D0020C4
:109E9000345D002040B139B110B51A4A146886B05B
:109EA00024B1112006B010BD0E207047034606A84D
:109EB0001360154B00F8114D19808DF808408DF88E
:109EC0000C40F6F799F802A91048F6F7F1F8A0B996
:109ED0000F4B9DF807001C7854B10E4A14783CB122
:109EE00000241C70F6F7AEF8FFF730FA2046D9E7E9
:109EF000F6F7A8F8204606B010BD2046F5F71CFB83
:109F0000E6E700BFC46100202464002034C30200DF
:109F10003A5D0020345D0020F8B5274B1B785BBB11
:109F2000264B1B7843BB002844D0254C254A0927E3
:109F30004FF0FF310126C4F81075C4F804354FF412
:109F40000037C4F80835E6604FF48063C4F808139E
:109F50004021C4F804730546C2F880311A4882F8DB
:109F60000A131360F6F770F91848F6F76DF91848F8
:109F700000F06CFC10B1F8BD0820F8BD154A164B76
:109F80001060164A186041F646631560C4F80873FD
:109F9000C4F84435D4F844351149124A3E33C4F864
:109FA0004435E660C4F844012660C4F804730E70BA
:109FB0001070F8BD0E20F8BDBA610020B861002015
:109FC00000A0004000E100E034C3020020C3020012
:109FD000B5950200C8610020CC610020F06200202D
:109FE000B6610020B761002010B5064B00241C604C
:109FF00000F052FC0449054A054B0C7014701C70AB
:10A0000010BD00BFF0620020BA610020B8610020DE
:10A01000B66100202DE9F041804D2C78002C4ED106
:10A020007F4E377807BB7F4C23681BB97E4A117877
:10A03000002971D07D490A689088834200F08D80A4
:10A040007B4910680A78C05C002A00F0C5800023B4
:10A05000C0280B7078D0DD20F5F7B2FF23680133FC
:10A0600023600020BDE8F081724B34701A68DAB1C9
:10A0700093E80300704A714D1C6085E8030092E884
:10A0800003009C806E4D6F4B664E146085E80300A4
:10A0900093E803006C4D948034601C609C8085E8DC
:10A0A0000300FFF7B7FF3C46684A6948694B1470E4
:10A0B00000221B68027098470020BDE8F0815D4ACD
:10A0C000116800232B7029B392E803005A4D5B4EB0
:10A0D000136086E8030095E803009380584E594AC0
:10A0E000504F2B6086E8030092E80300564EAB8089
:10A0F0003B601360938086E80300FFF78BFF534AB1
:10A100005348544B1470012202701B68984700207A
:10A11000BDE8F0810C46F2E74F490978002989D162
:10A120004E4F397800295CD0404A12689188002946
:10A1300086D1C020F5F744FF4349002301220B607C
:10A140003B7023603270B7E7DC20F5F739FF2368F6
:10A15000013323600020BDE8F081404F97F800C034
:10A16000BCF1000FE5D1DFF8C08098F80000C8B15D
:10A17000334BC4F800C01E68002E46D03078364AF3
:10A1800088F800C00125C0280B60157001D0DB28BD
:10A19000DBD127490123DB200B70F5F711FF0020ED
:10A1A000BDE8F0812C4D95F800C0BCF1000F3FF4E4
:10A1B00047AF254B2060D3F80080B8F1000F19D0CD
:10A1C0001F4A2870106098F800000B60C0284FF0FC
:10A1D00001033B70DBD1DCE7C028DBD0DB28D9D022
:10A1E000B3E7124B15491960C02001231370F5F72E
:10A1F000E7FE61E7C020F5F7E3FE114A85F800802D
:10A200000123C2F80080337056E7C020F5F7D8FE6E
:10A21000012388F800602B704EE700BF2C640020FB
:10A2200094660020806600202F6400208C66002049
:10A230007D66002044660020586600203C660020B1
:10A2400050660020346600202C6600207C660020CA
:10A250006866002074660020956600202E64002049
:10A2600000286AD02DE9F0410378032B26D0042B77
:10A2700006D0022B16D00320BDE8F041F5F75CB9FB
:10A28000944B1A780AB901221A70934C05792378F5
:10A29000002B53D1C02D03D1904901220B602270B5
:10A2A000BDE8F08143689A07FAD08D488D4A436033
:10A2B00003230370BDE8F041136818478A4D2C78DA
:10A2C000002C5AD1894E3778002F40F0D980884C25
:10A2D0002368CBB9874A1178B1B98749097899B908
:10A2E000864F3978002900F00982854A12689188E2
:10A2F00081B9C020F5F764FE8249002301220B607A
:10A300003B7023603270CBE77D490A6890888342B6
:10A3100000F012817C4910680A78C05C002A00F0C5
:10A3200085800023C0280B7000F02681DD20F5F722
:10A3300047FE236801332360B2E77047674E3268F7
:10A34000002A45D0714F3B681BB17149097800293B
:10A3500041D0704F3B686BB1DFF8B4816E4901208A
:10A36000B2F5FD7F88F800000B60C0F04E81C02D73
:10A3700000F024810023237092E7684A11680023CB
:10A380002B70002950D092E80300654D654E136094
:10A3900086E8030095E803009380634E634A544FB8
:10A3A0002B6086E8030092E80300564EAB803B60CA
:10A3B0001360938086E80300FFF72CFE5C4A484850
:10A3C0001470484B012202701B68BDE8F041184729
:10A3D000C02DB7D164E7002A40F0FE804E490B60E3
:10A3E000A5F1C0031D2B45D8DFE813F0A001440000
:10A3F000440044004400440044004400440044003D
:10A40000440044004400440044004400440044002C
:10A41000440044004400440044004400440044001C
:10A4200044002C003C0030000C46C7E7C02802D096
:10A43000DB2840F0A28001230B70DB20BDE8F04157
:10A44000F5F7BEBD3B4B01221A7029E7394B19784D
:10A4500011B100211970DB252F4B1968531C8D5445
:10A4600033601DE7334B19780029F5D000211970AE
:10A47000C025F1E72F4B1B78002B7FF411AFEBE7E2
:10A48000264B34701A68DAB193E80300244A254D4C
:10A490001C6085E8030092E803009C80224D234B5A
:10A4A000134E146085E8030093E80300154D948073
:10A4B00034601C609C8085E80300FFF7ABFD3C46E0
:10A4C0001B4A07481470074B002202701B68BDE846
:10A4D000F04118474C660020966600206466002014
:10A4E00068660020746600202C64002094660020BA
:10A4F000806600202F640020956600202E640020D6
:10A500008C6600202C6600207D660020906600206E
:10A510002D640020846600208866002044660020A8
:10A52000586600203C6600205066002034660020FB
:10A530007C660020606600207D4F97F800C0BCF16B
:10A54000000F7FF4D6AEDFF81C8298F80000D0B17F
:10A55000784BC4F800C01E68002E00F0C780307829
:10A56000754A88F800C00125C0280B60157001D01D
:10A57000DB2802D171495EE7DC20F5F721FD236875
:10A58000013323608CE66C4D95F800C0BCF1000FE0
:10A590003FF4C0AE6A4B2060D3F80080B8F1000FE2
:10A5A00000F0B680634A2870106098F800000B60D5
:10A5B000C0284FF001033B70DAD1DBE76148624904
:10A5C00043600223037002810B68984700232370C5
:10A5D0003B6088F8003063E6042A70D1C02D00F09B
:10A5E000A5805A4B1B68002B3FF4C4AEDFF878817E
:10A5F0005749404601F0FFFC3268564BB2F5FD7FEB
:10A60000C3F80080BFF4B6AEEAE6A5F1C0011D298B
:10A6100050D801A050F821F0BDA50200B5A6020057
:10A62000B5A60200B5A60200B5A60200B5A60200B6
:10A63000B5A60200B5A60200B5A60200B5A60200A6
:10A64000B5A60200B5A60200B5A60200B5A6020096
:10A65000B5A60200B5A60200B5A60200B5A6020086
:10A66000B5A60200B5A60200B5A60200B5A6020076
:10A67000B5A60200B5A60200B5A60200B5A6020066
:10A68000B5A6020045A40200A5A6020091A60200FC
:10A690003149087810B100200870DB25511C9D5409
:10A6A0003160FDE52C4908780028F7D000200870BB
:10A6B000C025F3E7284909780029EFD0F0E5B2F585
:10A6C000FD7FFFF48DAEC02D7FF454AE21490968A3
:10A6D000994228D01D4B002018601A481A4B41603F
:10A6E0000221028101701B68984743E6C020F5F7FC
:10A6F00067FC012388F800602B70D1E5174B1849DF
:10A70000196001231370C020BDE8F041F5F758BC73
:10A71000C020F5F755FC074A85F800800123C2F8F0
:10A7200000803370BCE500233B60D6E73B68CDE793
:10A730002E64002050660020956600207D66002073
:10A740002C66002068660020746600208466002065
:10A750007866002088660020606600208C660020F5
:10A760003C6600202F6400203064002070B582B069
:10A7700002AB002403F8014D044618460D46164668
:10A78000F5F73AFC84B31A4B1A78DAB994E8030067
:10A79000184A82E8030025B195E80300164A82E8CA
:10A7A000030026B196E80300144A82E80300012260
:10A7B0001A70FFF72FFC9DF80700F5F743FC002007
:10A7C00002B070BD26B196E803000D4B83E803008C
:10A7D00025B195E803000B4B83E8030094E80300E0
:10A7E000094B83E80300E6E70E2002B070BD00BF0E
:10A7F0007C6600203C660020506600202C6600200D
:10A8000034660020586600204466002098B10B4B47
:10A81000984204D00A4B984206D000207047094A5B
:10A8200013682BB108207047074A1368002BF9D131
:10A830001060184670470E20704700BF78660020F1
:10A8400030640020906600208466002098B170B5C6
:10A850000A4D296809B1082070BD04460723084A3B
:10A860000848094EF5F752FB0849094B094A0E60A2
:10A870001A602C6070BD0E20704700BF7466002007
:10A8800061A2020048C302007866002090660020A2
:10A890008466002030640020024B00221A60F5F725
:10A8A000A3BB00BF7466002010B51B4B1A6882B0B2
:10A8B000AAB100221A601B6800934FF08043012266
:10A8C000164C0099C3F80823A36862703BB1D3E922
:10A8D00000230020A2609847A368002BF7D1104BFB
:10A8E0001A68B2B100221A601B6801934FF08043CE
:10A8F00002220A4C0199C3F8082323690122A2709D
:10A900003BB1D3E900230120226198472369002B42
:10A91000F7D102B010BD00BF0001004098660020D2
:10A920000401004060B910B5064CA3683BB1D3E9FF
:10A9300000230020A2609847A368002BF7D110BD28
:10A94000704700BF9866002010B582B002A80023AF
:10A95000144C00F8013DF5F74FFB237853B1E36841
:10A960009DF8070001330122E360A270F5F76AFB4E
:10A9700002B010BD0C4A6360E3601068A36010F081
:10A98000010023610AD001F071FA20B94FF0804331
:10A990000122C3F8182501232370E0E7072100F006
:10A9A00005F8F0E79866002000E100E04901002882
:10A9B00010B4C9B2C3B215DB00F1604202F56142C6
:10A9C00082F800134009800000F1604000F561400A
:10A9D00003F01F0201239340C0F8803103605DF84B
:10A9E000044B7047024A03F00F0422441176E9E752
:10A9F000FCEC00E0F0B506796F4C7601A31987B046
:10AA0000DD7E002D40F089804D7F1D770B685D1C39
:10AA10000CD001254FF0A04705FA03F3C7F808351D
:10AA20000B6803F5E073032547F823504B685F1C60
:10AA300006D003F5E0734FF0A045002745F82370DA
:10AA4000037905688F6904EB43131B7FC5F82475F0
:10AA5000002B46D00F7D4B7D05683B43C5F86C3518
:10AA6000D1E900750368C3F80C75C3F814550B7D64
:10AA7000012B7FD0A31905465A600B69A351EAB197
:10AA80000379097F026804EB43131B7F002B4BD132
:10AA9000C2F81C31D2F81C012A6800900098C2F854
:10AAA0004431D2F844212B680192444A0198C3F8FA
:10AAB0000423286840F30730FFF778FF2B792A68D2
:10AAC00004EB43131B7F5BB30823C2F80035344407
:10AAD00000200123E376E0752076A075A07607B00C
:10AAE000F0BD91F814C04D7D076845EA0C05C7F824
:10AAF0006C55D1E900C70568C5F81475C5F80CC5D3
:10AB00000D7D012DB6D18D686F1C3DD005F5E0752A
:10AB10004FF0A04747F8253036E0082007B0F0BDD9
:10AB20000423C2F80035D2E70023C2F81031D2F86E
:10AB300010012A6802900298C2F82031D2F8200150
:10AB40002A6803900398C2F82431D2F824012A68B5
:10AB500004900498C2F84431D2F844212B6805923D
:10AB6000174A0598C3F80423286840F30730FFF715
:10AB70001DFFA3E78B685D1C06D003F5E0734FF063
:10AB8000A045002745F82370CB685D1C0DD001253A
:10AB90004FF0A04705FA03F3C7F80835CB6803F573
:10ABA000E073032547F82350CB6805688F68C5F824
:10ABB0000835C5F810755DE7AC660020800002001E
:10ABC00010030200F0B404793C4B016864011A19C7
:10ABD000127F002A6DD00022C1F800251A190179D0
:10ABE00055680268B5B103EB4111097F002963D1B3
:10ABF0003349C2F808130268324E120B51B24909A8
:10AC0000203102F01F02012505FA02F246F8212048
:10AC100001790268D2F80C75D2F8146503EB411182
:10AC20004FF0FF3C097FB1B3D2F80815D2F81055A8
:10AC3000C2F80CC5C2F814C50268C2F808C5C2F84B
:10AC400010C57A1C06D007F5E0774FF0A04202202D
:10AC500042F82700771C06D006F5E0764FF0A042B8
:10AC6000022042F82600681C06D005F5E0754FF07A
:10AC7000A042022042F825004A1C06D001F5E071EE
:10AC80004FF0A042022042F8210023440022DA764D
:10AC90005A60F0BC7047D2F80815D2F81055C2F8C7
:10ACA00014C5C2F80CC50268C2F808C5C2F810C5C0
:10ACB000C7E7C1F8002591E703499AE7AC66002091
:10ACC0008402020000E100E010030200F0B5037905
:10ACD000524C5B01E51887B02D7F25B101F060452E
:10ACE000B5F1005F58D123449E7D002E57D19A754F
:10ACF00099609E8205796D016219137F13BB01680B
:10AD0000C1F81C31D1F81C61016804960126049F2A
:10AD10008E600168D2F808C0C1F81C31D1F81C312E
:10AD20000593059B968A938A5768B6B201331CF83F
:10AD300006609BB29382C1F81C65002F32D00020C0
:10AD400007B0F0BD03689168C3F82061D3F82031E3
:10AD500001930368019FC3F85861D3F858610368F1
:10AD60000296967D029FC3F84415C3F848650368B0
:10AD7000012199605368002BE1D1036801E00029AB
:10AD800049D1D3F82021D3F85811002AF7D000294F
:10AD900014BF0F20002039E0102007B0F0BD1120B3
:10ADA00007B0F0BD967D938A9E4222D9016804E0E7
:10ADB000938A9BB2B3F5807F03D0D1F81C31002B6E
:10ADC000F6D0938A9BB2B3F5807FECD0C1F81C71AA
:10ADD000D1F81C310393039BB2F814E0938A1FFA55
:10ADE0008EFE01331CF80EE09BB29382C1F81CE585
:10ADF000D9E7938A9BB2B3F5807F0CD00268D2F872
:10AE00001C31002BFBD00123D36000202C440023F5
:10AE1000A37507B0F0BD0F20F8E700BFAC660020B7
:10AE2000F0B403798E4E5B01F41888B0257F6DB3C2
:10AE300001F06045B5F1005F44D16568002D45D053
:10AE400004684FF40475C4F80853F418E57D45BB55
:10AE500033440024DA75D9605C761C7603795B0193
:10AE6000F5182F7F002F38D1A97E0268002900F045
:10AE70008880F4186168002900F094804FF4017311
:10AE80000020C2F8043308B0F0BC70476568EDB12B
:10AE900004684FF40175C4F80853F418E57D002DDB
:10AEA000D6D0247E002C43D00379026806EB4313EE
:10AEB0001B7F002B00F0C0804FF40473C2F80433F2
:10AEC000112000E0102008B0F0BC7047E57D002D97
:10AED000BED0247E64B31120F5E703680025C3F8D3
:10AEE0001051D3F8107103680197019FC3F84451C2
:10AEF000D3F8445103680295029DC3F83415C3F892
:10AF00003825002C39D00268D2F8003243F02003F3
:10AF1000C2F80032037902685B01F1184968C1B1D7
:10AF20004FF404730020C2F8043308B0F0BC70473B
:10AF3000334419611A7603795B01F418247F002CDD
:10AF4000CBD1026895E7002C40F08180002840F0CA
:10AF50008280D2F81011D2F84441D2F8240100299D
:10AF6000F1D000284FF00002334414BF03201046F4
:10AF70009442DA7518BF0F20A5E7036801221A6012
:10AF8000C8E7C2F82411D2F8244102680394039C54
:10AF9000C2F80811D2F80811026804910121049C3A
:10AFA0001160CEE7C2F84411D2F844210592059A07
:10AFB0000268D2F82471D2F80851D2F8441145B988
:10AFC000002932D1002FF4D033440022DA75032057
:10AFD00079E7002FF8D151BBE57D9DB1C2F808118A
:10AFE000D2F8081106910699E568617ED2F8182515
:10AFF0006A54627EE17D0132D2B26276627E914213
:10B00000D6D808E0C2F80851D2F80811079107997C
:10B01000D2F81825627E334400219A7ED9758AB110
:10B020000368012208461A604DE7002FCCD1334453
:10B030000022DA750F2046E74FF40173C2F804339B
:10B04000112040E703680121104659603BE7334473
:10B050000F20D97537E733440320DC7533E700BF91
:10B06000AC660020114A037902EB4313197FE1B962
:10B070009B7ED3B910B4016883B0C1F82431D1F8F4
:10B08000244101680094009CC1F80831D1F80831CE
:10B09000016801930123019C0B60017902EB4112CD
:10B0A000937603B05DF8044B70477047AC660020A0
:10B0B000F0B5A94C237F8FB0002B73D1A74AD2F8EB
:10B0C0000413890546D4A54BD3F80423520704D5AD
:10B0D000D3F80821002A40F0D480A04BD3F81C21DB
:10B0E000BAB1A18AA27D8A4200F2B9800021C3F8D8
:10B0F0001C11D3F81C310593059B52B1A3688DF840
:10B100002810A1750B938DF83020D4E900130AA8FC
:10B110009847924BD3F84421D2B10022C3F844217E
:10B12000D3F84411A27E04910499002A40F094803F
:10B13000E37D6BB10023617EE268E37501238DF846
:10B1400030108DF828300B92D4E900130AA89847E4
:10B150000FB0F0BDD2F824110029B4D0C2F82431C8
:10B16000D2F82411A37E07914FF401710798C2F819
:10B1700008130BB901235360784A02238DF8283055
:10B18000D2F88034C2F88034E07DE2680D93002369
:10B190008DF83000E375237621680B9263680AA866
:10B1A00098479AE76D4BD3F82421002A00F0978046
:10B1B0000022C3F82421D3F82411029102218DF832
:10B1C00028100299D3F88014C3F880140D91D3F895
:10B1D0003C15E3688DF830100B93E27522762168F8
:10B1E00063680AA898475D4BD3F84421B2B10022A6
:10B1F000C3F84421D3F84401E17D0190019869B17D
:10B20000D3F83C35E1688DF8303001230B918DF88F
:10B210002830E275D4E900130AA898474F4BD3F8B9
:10B220002021002A94D00022C3F82021D3F8200145
:10B23000A17D0090009800298AD0D3F84C15A3680E
:10B240008DF830100B938DF82820A275D4E90013E7
:10B250000AA898470FB0F0BD01221A6068E70022E3
:10B26000C3F81C21D3F81C210692069AA18AA28A4F
:10B27000A06889B20132415C92B2A282C3F81C1567
:10B2800047E7E27D002A54D00022C3F80821D3F812
:10B2900008210892089AE168627ED3F818358B5429
:10B2A000637EE27D0133DBB26376637E93427FF49B
:10B2B00014AF237E2168002B52D0E268657E20699E
:10B2C000E3750B9200230122E060237663768DF80C
:10B2D00030508DF8282063680AA89847FDE6D3F817
:10B2E000101100293FF47FAFC3F81021D3F81011DB
:10B2F00003910399D3F83C15E07DC9B288427FF4ED
:10B3000072AF257EE768D4E90016DDB1D3F800C23C
:10B31000E5752CF020052276C3F80052012223693E
:10B320008DF83000E3600B978DF828200AA8B0470D
:10B3300059E7C3F80821D3F8081109910999D3F8FE
:10B340001835B2E701238DF83000E5750B978DF8BD
:10B3500028300AA8B04746E7AC660020002000402D
:10B36000A37E13B90A4B01225A60094AE068636858
:10B370004FF40175C2F80853627E8DF83020002525
:10B3800001220B90E5758DF828200AA89847A4E6BD
:10B39000002000403EDF704700B54FF0804301229F
:10B3A00083B09A671021234A4FF49A70F4F7D4F8C7
:10B3B00008B1F4F7C1F8204B20491A6802A800230D
:10B3C00040F8042D4FF49A7200F056FD08B1F4F7DE
:10B3D000B3F81B4800F09AFD08B1F4F7ADF819482E
:10B3E000FDF736FD58B9F4F7A7F900F0EFFD70B995
:10B3F000FDF7BAFBA8B9FFF7CDFF0028F3D0F4F7AB
:10B400009BF8F4F799F900F0E1FD0028F0D0F4F78B
:10B41000CDF80828ECD900F0B5FDFDF7A5FB002814
:10B42000E9D0F4F789F8FFF7B5FF0028DBD0F4F78F
:10B4300083F8E6E7CC66002060C30200C87B0020EA
:10B44000858B0200F98A0200F8B54FF08043002294
:10B450000121C3F800211A461960D2F80031002BEF
:10B46000FBD03A4B3A491B683A4D002201244FF475
:10B4700080305C600426DC60C3F80425C3F84021FA
:10B48000C3F84421C3F84821C3F84C21C3F804038E
:10B4900040F6C410C3F80042C3F81065C3F8400575
:10B4A0004FF48270C3F844050A601C6028680321C9
:10B4B00000F092FA002847D1274A284B0321C3F80D
:10B4C0000815C2F800021346C2F810011461D3F83F
:10B4D0001021002AFBD000222149C3F810215A6014
:10B4E0001A602C680A800321C3F80C45C3F81015B4
:10B4F000D3F82415DFF880C01A4F1B4E1B4D21F0E6
:10B50000FF01C3F82415D3F8241541F07101C3F8E5
:10B510002415012440F20311C3F81CC5C3F83045BB
:10B52000C3F82C25C3F834154FF48471C3F81415EF
:10B530000F49C3F818150F493A7034702A600B6927
:10B5400043F010030B61F8BD3046F8BD3C5D0020B0
:10B55000FC7C0020147E00200010004000F0014020
:10B56000107E0020027D0020127E0020047D00203D
:10B57000FF00030000ED00E000294176F8B5364AEF
:10B58000364D1369364C374F374E43F01003136175
:10B59000D4F80C3143B102230022C4F80C21C7F8BF
:10B5A00080313378042B23D02B68D3F840213AB173
:10B5B0000022C3F84021D4F80C31002BF4D0EAE784
:10B5C000D3F844110029E3D02849C3F8442191F964
:10B5D000001024484B090122603301F01F0102FAD8
:10B5E00001F140F82310224B186810441860F8BD90
:10B5F00001236360D4F80034012B06D040F201121D
:10B6000000211C48F3F78EFFCEE71A4B197801F0A2
:10B610000F010229F2D85A78B9B101290CBF0F20C5
:10B6200055206AB199788142E8D10233013A53FA40
:10B6300082F203E013F8011F8142DFD19A42F9D16F
:10B640000D4A138801331380D8E7981C0B4900F08A
:10B65000C3FC0028F4D0D1E700ED00E03C5D002001
:10B660000010004000E100E0127E00203B5D002061
:10B67000FC7C0020087D0020107E002064C30200B6
:10B680002DE9F04FBA4EDFF810833568DFF80C93E0
:10B69000DFF80CE3DFF80CC398F80040C9F800109D
:10B6A00002F03F0705F0C0053D434FF0000A0127B7
:10B6B00083B035608EF80070ACF800A0002C44D048
:10B6C000834698B103284BD0012C42D1581C01D09D
:10B6D000272972D8A7480027BBF1010F078000F087
:10B6E000BE80BBF1020F6CD000202BE0CDE9002121
:10B6F00000F068F9A048A14BC0F808750324C0F811
:10B7000010B5C0F814B5C0F80845C3F800B2C3F8C6
:10B7100010B11F61DDE900211D46D5F81031002B65
:10B72000FBD001239942934C4FF0000008BF9201D7
:10B73000C5F8100168602860208088F800300CBFD0
:10B740003260306003B0BDE8F08F052003B0BDE883
:10B75000F08F01230220ACF8003003B0BDE8F08F79
:10B76000012CF6D0834C23886FEA43436FEA53439E
:10B77000ACF8003000F026F97F4A804BC2F808751B
:10B78000C2F810A5C2F814A5C2F808B5C3F800A203
:10B790001A46C3F810A11F61D2F81031002BFBD05C
:10B7A000002301211846C2F8103153601360238032
:10B7B00088F8001003B0BDE8F08FACF800402046D8
:10B7C000C0E76F4F03F00F00012B7D70387000F061
:10B7D000BF80C0F0B780022B6DD0013366D1032A41
:10B7E00082D8DFE802F00C0C02324BB211F0300FBD
:10B7F000644A18BF63F03F0300201360A2E75F4D67
:10B8000000F0E0F840F25B625F4BC5F83825C5F800
:10B810003C35D9F800305B4A5B0002330024032634
:10B82000C5F80835C5F80475C5F80041C5F80062CB
:10B830001368C5F80C3500F0C7F80123C5F80032CD
:10B8400020462B6088F800607CE70A464F48504944
:10B8500000F0DAF800287FF447AF042072E7484C84
:10B8600040F2011239462046F3F75CFE00F0AAF8D8
:10B87000424B454A40F25B61C3F83815C3F83C259A
:10B88000D9F800205200023203250421C3F808250C
:10B890003846C3F80445C3F80071C3F80052C3F832
:10B8A0000C71C3F804B088F800104BE70123ACF822
:10B8B0000030042046E72A465521B81CF3F732FE33
:10B8C00000F080F82D4B304A40F25B61C3F8381528
:10B8D000C3F83C25D9F800202A4952000232C3F8A7
:10B8E000082500200322C3F80475C3F80001C3F83B
:10B8F00000220A68C3F80C2533680A33DB00B3F56D
:10B90000BC7F15D8214B1A6840F27123C2F840352C
:10B91000194B1A4802F5A07201240221C3F8102520
:10B92000C3F81405C3F80445002088F8001009E79F
:10B93000164AB3F57A7F126810D840F2E243C2F893
:10B940004035E5E72A461349B81C00F054FBB7E739
:10B950002A460F21B81CF3F7E5FDB1E7B3F5CB6F2D
:10B9600094BF40F2537340F6C413C2F84035CFE79A
:10B97000047D0020107E002000F0014000100040F7
:10B98000087D0020147E0020555555003C5D0020A8
:10B990003B5D002064C30200127E00200C7E00206C
:10B9A000027D0020007D0020044B054A1978128892
:10B9B0000260002208461A70704700BF027D002016
:10B9C000007D0020704700BF024B4FF40072C3F8A7
:10B9D000502670470010004070B120F02003D82B93
:10B9E0000AD020F01003EC2B06D020F00403F02B3B
:10B9F00002D00338012804D803298CBF042000207A
:10BA000070470420704700BF4AB1012A0DD0022AB6
:10BA100017D0032A0FD0042A19D0002070470F4BEB
:10BA2000036008230B70012070470D4B036009234E
:10BA300010460B7070470B4B03601A230B700120EC
:10BA40007047094B03600A230B7001207047074BB6
:10BA500003601B230B700120704700BF0080004073
:10BA60000090004000A0014000A0004000B0014054
:10BA70000649074A074B9B1A03DD043BC858D050C0
:10BA8000FBDC00F013F8F3F7DBFC000070C40200ED
:10BA9000C05C00204C5D0020FEE7FEE7FEE7FEE70D
:10BAA000FEE7FEE7FEE7FEE7FEE7FEE730B4A24B67
:10BAB0001B78062B1BD0A14AD2F8883043F47003C0
:10BAC000C2F88830BFF34F8FBFF36F8F4FF0102352
:10BAD000D3F80022002AC0F2FE80D3F80432002BF3
:10BAE000C0F2F980964B974A1A6030BC7047964B6B
:10BAF0001B681B07DFD1954B1B6803F0F003302B4D
:10BB000002D1934B934A1A60904B1B6803F0F002EA
:10BB1000302A49D003F0E003402B45D08B4B1B6803
:10BB200003F0F003302B00F0C780884B1B6803F054
:10BB3000F002302A26D003F0E003402B22D0834BC2
:10BB40001B6803F0F003302B56D0804B1B6803F0CA
:10BB5000F003302B39D07D4B1B6803F0F003502BE2
:10BB600058D07A4B1B6803F0F002302A03D003F060
:10BB7000E003402B9FD1784B784A1B6803F04F03BA
:10BB8000136098E76C4B1B784FF080420021062B26
:10BB9000C2F80C11C2F81011C2F838158BD16A4BDB
:10BBA0001B68180787D1CAE76D4B634A1B68127878
:10BBB0006C49C3F34233062A0B607FF47CAF624BBF
:10BBC0001B681D077FF477AFA8E75B4B664C1A78BC
:10BBD00066496748674B0525256001250D600024EF
:10BBE0003F21062A046019607FF465AF564B1B683D
:10BBF0001A077FF460AFAEE74F4B5F4A1B78032113
:10BC0000062B11607FF457AF4F4B1B6819077FF469
:10BC100052AF9AE74FF08052584BD2F80414C3F851
:10BC20002015D2F80814C3F82415D2F80C14C3F860
:10BC30002815D2F81014C3F82C15D2F81414C3F830
:10BC40003015D2F81814C3F83415D2F81C14C3F800
:10BC50004015D2F82014C3F84415D2F82414C3F8C0
:10BC60004815D2F82814C3F84C15D2F82C14C3F890
:10BC70005015D2F83014C3F85415D2F83414C3F860
:10BC80006015D2F83814C3F86415D2F83C14C3F820
:10BC90006815D2F84014C3F86C15D2F84424C3F8E0
:10BCA0007025254B1B78062B7FF405AF264B1B68B0
:10BCB0001B077FF400AF54E7314A1F49D368097866
:10BCC00023F080730629D360EBD11F4B1B681C0740
:10BCD0007FF4F1AE29E72B4B0122C3F80425D3F8FA
:10BCE0000024002AFBD04FF0102315222549C3F869
:10BCF0000022D1F80034002BFBD04FF01022152188
:10BD0000204BC2F80412D3F80024002AFBD00022F2
:10BD10001C49C3F80425D1F80034002BFBD0BFF335
:10BD20004F8F0649184BCA6802F4E0621343CB6098
:10BD3000BFF34F8F00BFFDE7E00F00F000ED00E024
:10BD4000405D00200090D003E40F00F0E80F00F009
:10BD500074C007400DF0ADBA58020010E40E004068
:10BD6000440200103C050040105600408856004038
:10BD70001856004014560040A005004000C0004086
:10BD8000F0ED00E000E001400400FA0548DF7047F4
:10BD900010DF704761DF7047FCF740BE2DE9F047C8
:10BDA000DFF8BC902C4ED9F80040DFF8B8802B4F5C
:10BDB000DFF8B4A0B4FA84F482B06409337803F0F5
:10BDC000FF057BB901A8FFF7E1FF05280DD000288A
:10BDD0002FD0F3F7B1FB5CB13378012403F0FF05FA
:10BDE000002BEFD002B0BDE8F087002CFAD101257E
:10BDF000337803F0FF04002BF4D13A68B8F8003030
:10BE0000ADF80430104601A9FFF7C4FF05280BD098
:10BE1000D0B91046D9F800309847002DCED03378ED
:10BE20000125002BE9D0DDE7002DD5D002B0BDE81B
:10BE3000F0870198FEF776FDDAF800304BB10198F3
:10BE40009847002CC8D1D3E7F3F776FB002DE6D155
:10BE5000B4E7002CC0D1CBE7257E00202C7E00204B
:10BE60001C7E0020187E0020287E0020014B1878C0
:10BE7000704700BF247E002000292ED011F0030F50
:10BE80002BD138B51A4C1B4D21601B491B4C2A8005
:10BE90000B602368DB0708D50123C4F880301849FC
:10BEA000FFF776FF30B1236038BD1549FFF770FF0B
:10BEB0000028F9D1134B01221A70FEF745FD0F4AF5
:10BEC00092F81633C3F34113012B08D90E4B98682F
:10BED00040B94FF48003136038BD0720704742F229
:10BEE000020038BD1A6842F480021A60002038BD92
:10BEF0002C7E0020187E0020207E002000E100E043
:10BF000099BD0200247E0020307E0020034618B137
:10BF1000024A0020136070470E2070471C7E0020EC
:10BF200008B5094B1B6833B1984700B908BDBDE897
:10BF30000840F3F701BB054B1B78002BF6D0BDE89A
:10BF40000840FFF72BBF00BF207E0020247E00208A
:10BF5000094B9A6842B9094B4FF48002C3F880201C
:10BF6000074B01221A7070471A6822F480021A6087
:10BF7000034B01221A707047307E002000E100E080
:10BF8000257E00200E4B1A7802B970470D4A00201A
:10BF90004FF480011870C2F8001192F81633C3F301
:10BFA0004113012B08D9084B986808B911607047F4
:10BFB0001A680A431A60704742F20200F3F7BCBAEB
:10BFC000257E002000E100E0307E0020014B187843
:10BFD000704700BF257E002030B50024A24201D169
:10BFE000002007E0035D01340D1915F8015CAB4238
:10BFF000F4D0581B30BD10B5431E0A44914200D105
:10C0000010BD11F8014B03F8014FF7E7F8B500BF79
:10C01000F8BC08BC9E467047F8B500BFF8BC08BC29
:10C020009E467047C05C0020FFFFFFFFFFFFFFFF41
:10C03000FFFFFFFFFFFFFFFF000000000000000008
:10C040000000D60107010000320000004585020013
:10C050004900000065850200430000009D85020044
:10C0600062000000456F020063000000896F02005B
:10C0700064000000CD6F0200650000001D7002002A
:10C08000660000008970020069000000C5700200AF
:10C090006800000019710200600000008571020054
:10C0A00067000000D9710200B0000000898402001E
:10C0B000B1000000BD840200B2000000F184020063
:10C0C0008B000000AD7802006C000000697A02006D
:10C0D0006D000000A17A020070000000DD7A02000D
:10C0E00071000000157B02006E000000517B020011
:10C0F0006F000000BD7B02008C000000CD720200CA
:10C100008D000000157302008A00000031730200E8
:10C1100086000000A177020085000000C9780200B7
:10C12000720000006973020073000000C573020012
:10C130007400000001740200750000001D7402000C
:10C14000760000005D740200770000009974020020
:10C1500078000000CD740200790000000175020033
:10C160007A0000003D7502007B000000757502003A
:10C170007C000000F57502007D000000B175020032
:10C180007E000000417602007F0000008176020000
:10C19000800000005977020086000000A1770200AD
:10C1A00087000000F5770200880000003578020063
:10C1B00089000000797802008200000059790200AD
:10C1C000810000009579020084000000D57902000A
:10C1D000830000001D7A02008E0000001179020029
:10C1E00094000000897C020095000000D17C0200D0
:10C1F00096000000117D020097000000517D0200B2
:10C2000099000000917D02009A000000E17D02008B
:10C210009B000000297E02009C000000757E020049
:10C220009D000000C57E020098000000017F020012
:10C230009E000000497F0200A0000000BD7F0200B8
:10C24000A1000000A9800200A20000000D800200F1
:10C25000A3000000F5800200A40000005981020044
:10C26000A5000000B1810200A600000005820200C6
:10C27000A70000005D820200A8000000A182020069
:10C28000A9000000F1820200AA0000004983020018
:10C29000AB00000005840200AC000000B583020082
:10C2A000AD00000041840200FFFFFFFFFFFFFFFF22
:10C2B000FFFFFFFFFFFFFFFF000000000000000086
:10C2C0000000D6010701000000F0040000D00900C2
:10C2D00000B013000050270000003B0000A04E00FB
:10C2E00000F0750000509D0000F0EB0000903A0156
:10C2F00000E0D70133000000230000001B00000015
:10C3000017000000150000001500000014000000D8
:10C3100014000000130000001300000013000000D0
:10C32000E0620020D061002010000000100000003A
:10C330000100000008640020F862002010000000E6
:10C3400010000000010000000800000006000000CE
:10C3500005000000070000000100000000000010C0
:10C3600001000007FFC1FBE84C90728BE7B35189D5
:10C3700063AB232302841872AA612F3B51A8E537CF
:10C3800049FBC9CA0C18532CFD45E39AE6F15DB090
:10C39000B61BB4BE2A50EAE90E9C4B5E5724CCA1D2
:10C3A000B759B887FFE07D742648B9C5F3D9A8C44A
:10C3B000B1D5911101420C39D5B0979D28D4F29B8B
:10C3C000A4FD6465068C2996FEA2714DF3F82E58E3
:10C3D000DB0D5A5F1528F57407CE25AF2B12E6D07A
:10C3E000DB2CDCC37FF03E3A13A4DCE2F96C54E2B0
:10C3F000D8EAC8880021869C6AD8CB4E146AF94DC9
:10C40000D27EB23203C6144B7FD1B8A6797C17AC6A
:10C41000ED06ADAF0A947ABA03E792D7150973E82F
:10C420006D16EEE13F781F9D09526EF17C362A7140
:10C430006C7564448010434E35EC65270AB5FC26C4
:10C44000693F599901638AA5BF685CD33CBE0BD68E
:10C450007683D657054A3DDD8173C9EB8A8439F46A
:08C46000360BF700000000009C
:08C46800D82FFF7F0100000046
:10C4700000000000000000000000000000000000BC
:10C4800000000000000000000000000000000000AC
:10C49000000000000000000000000000000000009C
:10C4A000000000000000000000000000000000008C
:10C4B000000000000000000000000000000000007C
:10C4C000000000000000000000000000000000006C
:10C4D000002000400000000000200040000000009C
:10C4E000330000000100017E0101010800800040CE
:0CC4F0000090D00325F4010001F40100CD
:040000032000BA71AE
:00000001FF
